:020000040000FA
:1000000000F80202C17500005D330000C940000025
:1000100000000000000000000000000000000000E0
:100020000000000030490100784901005D33000004
:1000300000000000000000005D330000297C00008B
:10004000E93200005D3300005D330000E17500001F
:10005000BD4D00009D700000ED320000E133000056
:1000600025170000611600005D33000061330000B9
:10007000914D000035880000617500008D7500000D
:100080005D3300005D3300005D3300003D7F000004
:100090005D7F00005D3300005D3300005D330000D4
:1000A000817F00008B7F0000EB320000B173000005
:1000B0005D3300000571000000000000000000003A
:1000C0000348854600F08AFE0048004785C50000C9
:1000D00000F8020230B50B46014600202022012420
:1000E00009E00D46D5409D4205D31D469540491B6C
:1000F0002546954040191546521E002DF1DC30BDB5
:1001000070B500242546002801DA01244042002968
:1001100001DA01254942FFF7DDFFAC4200D0404241
:10012000002C00D0494270BD03460B439B0703D00F
:1001300009E008C9121F08C0042AFAD203E00B78AC
:100140000370401C491C521EF9D27047D2B201E024
:100150000270401C491EFBD270470022F6E710B522
:1001600013460A4604461946FFF7F0FF204610BD25
:10017000CAB2401E4178401C8A4202D00029F9D1FF
:1001800000207047421C0178401C0029FBD1801AD6
:10019000704730B504460020034600E05B1C9342E4
:1001A00003D2E05CCD5C401BF8D030BD30B50546D5
:1001B0000020034600E05B1C934205D2EC5CC85C67
:1001C000201A01D1002CF6D130BD00000FB400B5CB
:1001D0008DB009900B9010A900200091C0430A90A7
:1001E00000200C9006480690064807906A4609A829
:1001F0000F9900F05BFC0DB008BC04B0184700007C
:10020000CD0A0000ED0A0000FFB5002083B0009089
:1002100050680190916914460026976804988847B1
:1002200005460C990698084305D009E0A169761C9B
:10023000049888470546216A284688470028F5D152
:10024000681C03D00198C00704D017E00020C04309
:1002500007B0F0BD2068011D2160006800900DE02E
:100260000198C00704D1009805700098401C0090C8
:10027000A169761C7F1E049888470546002F1CDD67
:10028000681C1AD0069800280FD0E817C00E401935
:1002900041118A0006994009511840012A1A09683B
:1002A000012090400142DBD107E00C980028D7D113
:1002B000216A284688470028D2D0E16904988847F7
:1002C0000C98002807D1002E05DD0198C00702D147
:1002D000009800210170A068B84204DD0C98002845
:1002E00004D0002F02D00120C043B1E73046AFE771
:1002F00070B5064610F0ACFE046805460A220021DF
:10030000304600F05FFC2C6070BDF8B502464A40F4
:10031000D40F42004B0052085B089A4202D20246B8
:10032000084611464A0023D0C30D4A00DDB2120E22
:10033000AD1A202D35DA49020126490AF6058A1937
:10034000002C00D0524220214F1B1146B9402A41B7
:100350001018C20D9A4221D0002C17D0012D08DCB4
:10036000DA05801AD20F8019D207DBB200F06AFCDE
:10037000F8BDDA05801A012340001B06C01880185A
:100380005A428018CA0F1043490007E04908C207C3
:100390001143DA05801A80194008801800F04AFCE1
:1003A000F8BD61000122511A001BF7E70122D207B4
:1003B0005140AAE70122D2075040A6E7024670B595
:1003C0004A40D30FDB0740002DD04A002AD0010E4F
:1003D000140E000212020919400A520A8418E5019B
:1003E00004465443000A120A2E045043A419421929
:1003F000200CC543AA18120C0125AD03521C52193A
:1004000012047F39240400D0521C104301D4400050
:10041000491EC2B20C06C0092018401C4008802AA0
:1004200002D003E0002070BD40084000002900DA3F
:100430000020184370BD70B502464A40D50F4000F9
:100440004A00ED0740085208002814D0002A12D0B4
:10045000C40DD30D41020120C0055202490A520ABF
:10046000E41A091812187D34914201D3641C00E08B
:100470004900002C01DA002070BD0023914201D315
:10048000891A0343400849000028F7D100290AD0FF
:10049000914202D10121C90705E0914201D2012117
:1004A00001E00121C943E005C018401900F0C2FB7A
:1004B00070BD0000F0B507460846584087B0C00F31
:1004C000049048000E46590040084908BC1A88416B
:1004D00005D2384631461E4617460B46024658009E
:1004E000400810434CD0300D039040055900400D9A
:1004F000490D0590401A0290402872DA1803012134
:10050000000B09050843019004980092002805D0CB
:1005100001995242002088410092019002984021A6
:100520000A1A0199009800F087FA05460C466B46B6
:1005300007CB00F0A2FAC0197141039A0E0D0023F7
:10054000D71756401A467A40164344D0049A002AD8
:100550002DD0029A012A039A15DC1205C01A914186
:1005600001263605001C7141D20F059ED20700936B
:10057000019202962A46234600F0AAFB07B0F0BD7E
:1005800038463146FAE71605224A0F46B218C01A15
:10059000B74101210905001C4F4100187F41114658
:1005A00018187941E20F10436D19644113E0E20716
:1005B0006D0815436408C2071443039A0126120507
:1005C000C01A91413605001C7141CE0740083043E6
:1005D0004908C01851412A46234600F06CFBCDE77C
:1005E000FFE7049801224000C117121A00238B4133
:1005F00004983146C417381AA141EEE730B40124FB
:10060000E407634030BC55E730B40124E40761409F
:1006100030BC4FE70000E0FFF0B51FB488B00B9985
:100620000998002448400999C00F490049080991D8
:10063000C0070B990090490049080B910999089847
:10064000A64608431CD00B990A98084318D009986D
:1006500001244000420D4800410D09982405000383
:10066000000B204309900B980003000B20430B90D4
:1006700050181C494018002201901446104605E00D
:10068000002001460DB0F0BD032801DA034600E06A
:1006900003239C46C11A0AAE0AE05F0008ADED5B79
:1006A0004F00F75B7D430027AA187C41491C5B1E65
:1006B0006145F2DD410004AB5A522104120C0A4399
:1006C000240C401C0828DFDB01980290009970463A
:1006D00001910090059B049A0799069800F0F8FA9A
:1006E000D0E700000DFCFFFFF0B50C465C4085B084
:1006F000E40FE40703944C00002664085900944674
:10070000490802460296224321D062460A431ED07F
:100710006200570D4A000E032303550D01240246C3
:100720002C492405781B1B0B360B4018234326430A
:10073000614600901C46501AB44103D30098401CF7
:10074000009002E0921800985B41002803DA002034
:10075000014605B0F0BD0020012109050746864687
:1007600011E064461D46141BB54106D36546521B75
:10077000B341744607430C43A646CD0740084908D9
:10078000284392185B4105460D43EAD110461843B1
:1007900013D06046194650407140084306D0604669
:1007A000101AB34106D20122002306E000220123E1
:1007B000DB0702E00122D243531000987446010582
:1007C000381C6141029C039D0019694100F073FAD5
:1007D000BFE70000FD0300000122D207002800DB74
:1007E000101A002900DB511A814201D801207047FC
:1007F000002070470122D207002800DB101A0029D0
:1008000000DB511A814201D201207047002070475D
:100810000122D207002800DB101A002900DB511A40
:10082000814201D301207047002070470122D20786
:10083000002800DB101A002900DB511A814201D97F
:1008400001207047002070470122D207002800DBFA
:10085000101A002900DB511A814201D10120704792
:100860000020704710B5002904DB0C460121C907A0
:100870004042A141002B04DB1C460123DB0752420E
:10088000A34142404B401A4301D0002010BD01203B
:1008900010BDC217C10F504010B54018CA079623AB
:1008A000002100F0CFF910BD10B5002296231146AB
:1008B00000F0C8F910BD00000EB5054902910021F5
:1008C00000910A460B46019100F002FA03B000BD08
:1008D00033040000C20F410040020123400ADB053F
:1008E000D207090EC0187F2901DA00207047962927
:1008F00003DC9623591AC84001E096398840002A43
:10090000F4D040427047410040020122400AD20523
:10091000090E80187F2901DA00207047962903DC30
:100920009622511AC8407047963988407047000097
:1009300070B5CD0F4A0009030123090B1B051943AC
:100940000B4BED070024520D9A4201DA002070BDD6
:10095000074B34339A4203DC9A1A00F07DF802E028
:100960000449511888402C43F1D0404270BD00002A
:10097000FF030000CDFBFFFFC20FD207400040087D
:100980000BD0C10D0723DB01C91840020905400A3D
:100990001143C208400711437047002001467047C9
:1009A000CB0FDB07490010B5490802460A4307D0C0
:1009B0000A0D07240903E401090B121B002A01DCBC
:1009C000002010BDC900440F0C43C100E018D2053F
:1009D000801800F02FF910BDF0B51FB406460020B6
:1009E00082B005464024019100901BE00199224607
:1009F0000F46304600F030F8049A059B801A994162
:100A000010D310461946224600F016F8361A8F41C8
:100A10000197224601200021009F00F00DF83818B0
:100A20004D4100902046641E0028DFDC019B0098A9
:100A30002946324607B0F0BD10B5202A04DB014636
:100A4000203A9140002010BD914020239C1A03467B
:100A5000E3401943904010BD10B5202A04DB08463E
:100A6000203AD040002110BD0B46D340D040202476
:100A7000A21A91400843194610BD10B5202A06DB82
:100A8000CB170846203A1041C1170B4306E00B462E
:100A90001341D0402024A21A91400843194610BDAA
:100AA00002681378511801601846704710B5D1607C
:100AB000044951610449116200211161114600F09D
:100AC000ADF910BDA10A0000090E00004268002A1D
:100AD00008D001680B78491C002B03D0521E06C0B9
:100AE000184670470121C160881E70474268002A7D
:100AF0000BD0C3680168002B07D183688B4204D0F8
:100B0000491E521C06C0002070470020C043704799
:100B10000FB400B589B00A460DA9009100230C99C5
:100B2000002ACB60234B0693234B079301D0042369
:100B300000E00023214A0292214A089201930246D2
:100B40006B46002000F095FB09B008BC04B01847C4
:100B5000F0B585B007460020C04301901E46002036
:100B600015460C460091029104903B466A46314678
:100B700004A8FFF7CDFF049902466018002D05D0A8
:100B8000002901D0034600E023462B6000290ED047
:100B9000002A02DD0099814209D0001B01900094D7
:100BA0003B466A463146029404A8FFF7B1FF05B000
:100BB000F0BD0000CD0A0000ED0A0000FFFFFF7F3E
:100BC000090E0000F7B5009C0F4600262578641C2E
:100BD000002D05D000F014F90068405DC007F5D184
:100BE0002B2D02D02D2D18D0641E39462046029A96
:100BF00000F06AFC002F04D03968A14201D10099AD
:100C000039607105022400290BDA4042002803DD17
:100C100010F01EFA0460A007FEBD0120800206430A
:100C2000E3E70028F8DA10F013FA04600048FEBD8C
:100C3000FFFFFF7F002904DA401C490001D1400872
:100C40004000704770B40024050C05D11024000446
:100C500002D1002921D01124050E01D1000208344F
:100C6000050F01D10001241D850F01D18000A41CB6
:100C7000002801DB4000641C002908D020252E1B21
:100C80000D46F540A14000D001212943084301064B
:100C90001B1B000ADB1D02D5002070BC7047DB0562
:100CA000181880180029F8DA401C4900F5D170BCEA
:100CB00040084000704710B5002B08DA0024401CA3
:100CC000614192185B411A4301D14008400010BDB8
:100CD000F0B51FB482B005460C0003D0084610F0F2
:100CE0009FF902E010F09CF9203002460090214666
:100CF0002846FFF7A1FE049B059A04460F461843B9
:100D00001143084314D0184610431BD000984021CB
:100D10000A1A18460599FFF79FFE05460E46009AE7
:100D200005990498FFF788FE084305D0012004E0E8
:100D30002046394607B0F0BD0020C11705430E43D9
:100D40002C43374300990E986305401A7905E40A4D
:100D500000220C43FD0A0A3002D500200146E9E7D3
:100D60000105101969410C9C0D9D00196941FFF79F
:100D7000A2FFDFE74A0009030123090B1B05194302
:100D80000A4B10B5520D9A4202DA0020014610BDFE
:100D9000064B34339A4203DC9A1AFFF75DFE10BD0E
:100DA000034BD218FFF748FE10BD0000FF03000000
:100DB000CDFBFFFF10B5002904DB0124E40740420E
:100DC0008C412146002B04DB1C460123DB075242E9
:100DD000A341994200D1904210BD0000064C01256C
:100DE000064E05E0E36807CC2B430C3C98471034D3
:100DF000B442F7D3FFF768F974430100944301004C
:100E000000487047F419010010B50446FFF7F8FFD9
:100E10000068005DC007C00F10BD0000F3B58DB0C5
:100E200000200A9001200B90002608460C300C464A
:100E300009906269012109989047051E2ED0252D41
:100E40002DD0216A8847002818D0626901210998AD
:100E50009047216A88470028F7D1411E62690998A6
:100E6000904700E0761CA1690D988847216A884761
:100E70000028F7D1E1690D988847DAE7A1690D9854
:100E800088470746A84201D1761CD2E7E1690D9850
:100E900088477F1C02D10A98002877D049E10027B3
:100EA00062693D463946099890472A280CD1626903
:100EB000012109989047012506E00A214F433F1878
:100EC000303FEBD410200543626901210998904717
:100ED000014630390A2903D29B498F42DEDCECE718
:100EE000E90600D4994F6C280AD04C2810D0682805
:100EF00024D06A282ED074280CD07A280AD00DE08D
:100F000062690121099890476C2823D004211CE0D4
:100F1000202005436269012109989047A760656018
:100F200065284FD026DC582839D01ADC452849D00E
:100F300012DC252834D04128B0D143E06269012178
:100F400009989047682802D008210D43E6E7012060
:100F5000C002DEE70220DCE7462833D047282CD148
:100F600030E05B2870D061282CD063286CD06428D6
:100F700023D161E06F284FD009DC662822D0672892
:100F800020D0692826D06E2817D12EE0CDE0702819
:100F90004DD073286FD075284ED078280DD154E0ED
:100FA000A1690D9888470546252800D16CE7E169BD
:100FB0000D9888476D1C00D16DE7BAE00A224CE01D
:100FC0000A2252E0012023466A46C0430D9900F0F0
:100FD00050F9A3E02846402108436060A807234653
:100FE00001D5002239E000223FE0E80700D020E7E9
:100FF0002068011D21600068290501D5067018E7E9
:10100000290701D5068014E7A90703D5F117066063
:1010100041600EE706600CE7284640210843606007
:10102000A807234601D5082217E008221DE04849F9
:1010300028460840606016E028464021084360606A
:10104000A8072346BCD5B9E715E028464021084348
:101050006060A80707D5234610220120C0430D99E0
:10106000C046C0465AE0234610220120C0430D99D5
:10107000C046C04652E000210C910B460091632807
:1010800002D05B2807D043E0E80601D40120A0602D
:10109000012000903CE062690121099890475E2898
:1010A00005D101200C900146626909989047216999
:1010B000002906D10B4601AA8F00491CD3510829EB
:1010C000FADB002835D0216900290ED1C117C90EDD
:1010D00009184A11930001AA9A1849094901411AAD
:1010E0000120136888400343136062690121099855
:1010F00090475D28E5D10C98002808D0002001AB6E
:1011000081005A58401CD2435A500828F8DB01ABE2
:1011100001202246C0430D99FFF776F800280ADA2D
:10112000401C06D10B98002803D00020C0430FB00C
:10113000F0BD0A98FBE7E90702D10A99491C0A9118
:10114000361800200B9074E6CCCCCC0CFFFFFF7F50
:10115000F1F7FFFFFFB5087889B01546FF2805D0E5
:10116000491C2D2804D00022002407E000240BE0B5
:101170000122F9E70A235C430419491C0878FF2877
:10118000F8D1002A00D06442002004902A78014659
:101190002D2A01D02B2A0FD16D1C2D2A02D000221E
:1011A000049209E00122FBE700260A2233466D1C67
:1011B00000F0DDF9381871412F78FF2FF4D10C9A27
:1011C000A218069202460A4304D0FF23069A9133DE
:1011D000DA4205DA002109980A4606C00DB0F0BDD2
:1011E0000024B74AB54D2646079200F00DFA02904A
:1011F00006980391002801DA474200E007463905C6
:101200000020AF4A001C51410191009012E0F80704
:1012100007D022462B4630460799FFF7FDF90646D0
:10122000079122462B4610461946FFF7F5F904466A
:101230000D467F10002FEAD10698019B0028009AE6
:101240000399029806DAFFF74FFA3246079BFFF739
:101250004BFA05E0FFF7E0F93246079BFFF7DCF9B0
:10126000049A002A02D00122D2075140099A03C2EF
:10127000B4E7FFB591B0002009900025ED432E2082
:101280009E685C681F460190B9696D1C129888477A
:101290000090396A88470028F6D10098401C0AD08F
:1012A0000D20C0018443002E12DD00982B2809D0A8
:1012B0002D280DD103E00020C04315B0F0BD012062
:1012C00080020443B9696D1C12988847761E00900D
:1012D00003A9600501D52D2000E02B206A4610737C
:1012E000491C0CA80F9102900AE0B9696D1C129874
:1012F000884700900120400204431398761E056041
:10130000002E02DD00983028EFD001990098884225
:1013100045D18020044308E00998401E099001202F
:10132000400204431399681C0860B9696D1C761E5D
:101330001298884700903028EED030E0019988421A
:1013400005D1200603D480200443761E1DE00098BA
:101350000FF04CFF002825D0012149020C430098D2
:1013600007AA0F9903323038761E914208D20870CE
:101370000F98401C0F90200607D50998401E03E0E7
:10138000200602D40998401C0990A00502D51399A3
:10139000681C0860B9696D1C129888470090002E7F
:1013A000CCDC59E0002E57DD0098652801D0452897
:1013B00052D1A00550D5032000028443B9696D1CA9
:1013C000761E129888470090002E0CDD2B2804D042
:1013D0002D2808D1FF2001300443B9696D1C1298F3
:1013E0008847761E0090E00501D52D2100E02B21D5
:1013F000029801700298401C0290019025E00120A3
:10140000400204430EA902980131761E88420ED292
:101410000098029930380006000E087003D1029936
:10142000019881420AD90298401C029006E0E0052A
:1014300001D5244801E0234840420990B9696D1C58
:1014400012988847009013980560002E04DD0098DC
:101450000FF0CCFE0028D2D1F969129888470F9975
:10146000FF200870029903AA087000200A900B90D0
:101470000CA90AA8099BFFF76DFEA00502D4012064
:10148000C0431AE72420044209D0E00713D138688A
:101490000B9A0A99031D3B60006806C00BE00B998C
:1014A0000A98FFF77DFA0146E00704D13868021D6B
:1014B0003A60006801602846FFE600000000144022
:1014C0000000F03FF1D8FFFFF7B582B0029C002783
:1014D0002078641C15460197302802D0002D15D0C5
:1014E00015E020780127641C782804D0582802D001
:1014F000002D09D00BE0002D01D0102D07D10027C1
:1015000010252078641C02E0082500E00A2500264A
:10151000009610E00099012769430818020C29463B
:1015200080B2714300908E183804864201D30120A6
:1015300001902078641C294600F056F80028E9DA6A
:101540000398002805D0002F01D0641E00E0029C03
:1015500004600198002806D00FF07AFD0221016096
:10156000C81E05B0F0BD009930040843F9E7F0B596
:101570001FB486B000200090019002900698069952
:1015800080B204900798090C0204001411430790DC
:101590000027089D099806913E463C460390039813
:1015A000A9B20204000C039004982D0C1543484383
:1015B00000212246FFF740FAC719714110340E4648
:1015C000402CECDB3846029AFFF736FA009A019B72
:1015D00080180090594102980191103002904028E3
:1015E000CCDB00980BB0F0BD3A2800D23038202375
:1015F00002469A43412A01D310463738884201D324
:101600000020C043704700000EB5054A0292002238
:10161000009213460192FFF75BFB03B000BD000090
:101620003304000030B58C180278401C13071B0FE0
:1016300001D10378401C120906D10278401C03E056
:1016400005780D70401C491C5B1EF9D101E00B7040
:10165000491C521EFBD1A142E6D3002030BD000040
:1016600010B52148016A8A0715D44A0715D4C9075D
:1016700032D01E498A89002A15D0531E8B81826878
:101680008C6904C48C610A691B040DD0002A22D124
:101690000121016010BD022100E00421C161134855
:1016A0008021416110BD0A69012A09D10268012324
:1016B0009A430260C361FF20683099300C4A106081
:1016C00001204861CA69002A05D0886909898B0010
:1016D000C01A904710BD10BDFF226832054806A110
:1016E00009A30DF067F9C04608D0014098950102A2
:1016F00080E200E0502901004144435F49525148D3
:10170000616E646C65720000556E65787065637417
:1017100065642041444320696E746572727570740B
:101720000D0A000070B582B000230193444801689F
:101730008A6A4C6813252540132D02D1CB689B077C
:10174000DB0F4361930772D453070AD4D30711D137
:10175000130724D5048F838E1C1B102C0EDD102341
:1017600010E0042088620220032142A20EF07EF9DC
:1017700002B070BD0120886202B070BD048F1B1BD7
:101780001C0610D0DBB20024058FC66A75192D5DCA
:101790000D74641CA342F7D1048FE3180387D206AB
:1017A00007D400212FE04B6A0824A3434B62D206E2
:1017B000F7D5CB68C28E448F141B5B04DB0EA342AB
:1017C00001D3438FD31ADAB2002A16D0097D438F92
:1017D000046BE1540199012A10D001231C468901B0
:1017E00045582D7D41184E8F9B19096BCD54641CB3
:1017F000E3B201999A42F2D800E000218B01C318AC
:101800005C8FA2185A878A0181184B8FCC8EA34215
:101810000BD301230B61805800224262CA6B002A5D
:1018200003D03A31098801A8904702B070BD022068
:101830008862044804A1084A08A30DF0BBF8C0461A
:1018400084900102692901004145535F4952514882
:10185000616E646C65720000CE0200004145532049
:10186000696E707574206F766572666C6F770D0A9D
:1018700000000000414553206F7574707574207529
:101880006E646572666C6F770D0A0000F0B581B00A
:1018900001243F2900D993E003468068456B2D68F9
:1018A0008E0001A7BE59B746E7190000031A0000D1
:1018B000DF190000DF190000C1190000C119000084
:1018C000C1190000C1190000C1190000C1190000B0
:1018D000C1190000C1190000C1190000C1190000A0
:1018E000151A0000311A0000C1190000C1190000CA
:1018F000C1190000C1190000C1190000C119000080
:10190000C1190000C1190000C1190000C11900006F
:10191000C1190000C1190000C1190000C11900005F
:10192000C1190000C1190000C1190000C11900004F
:10193000C1190000C1190000C1190000C11900003F
:10194000C1190000C1190000C1190000C11900002F
:10195000C1190000C1190000C1190000C11900001F
:10196000C1190000C1190000C1190000C11900000F
:10197000C1190000C1190000C1190000C1190000FF
:10198000A9190000A9190000A9190000A91900004F
:10199000A9190000A9190000A9190000A91900003F
:1019A000A9190000A9190000434800690024022871
:1019B00009D001280DD0002802D103CA05F0E4F9AE
:1019C000204601B0F0BD03CA05F0D0F9204601B0B1
:1019D000F0BD03CA05F0EEF9204601B0F0BD0229C2
:1019E00031D0022430E0344D00242C616C619849E0
:1019F000354A01F027FE6869401C6861204601B045
:101A0000F0BD01F059FE284602F0C6F80024204639
:101A100001B0F0BD284909690C234B432749CA5836
:101A2000C918496801F00EFE0024204601B0F0BD3F
:101A30000024204605F076F90128C1D11E48303037
:101A4000204900241CE001241B490F690C26314663
:101A500079431A4A51188968214208D000247D1C14
:101A600015490D614C61052D10D3154906E0124949
:101A70004869401C4861032812D3294900241846AC
:101A8000224602F039F8204601B0F0BD6E430B4902
:101A90008A598919496801F0D5FD204601B0F0BD89
:101AA0000E20009000240A222846214602F014F855
:101AB000204601B0F0BDC046C8990102F8190100E6
:101AC00000210100E02001006A340100B0B50429C2
:101AD0000FD804468068C0467944097949008F448C
:101AE000020A0E1C1700104910A201F0ABFD0020E5
:101AF000B0BD0120B0BD01F0DFFD0020B0BD00256C
:101B00000321284605F01EF9064920462A4602E030
:101B100003490022204601F0EFFF0020B0BDC0467F
:101B2000F02001007021010088130000415445306D
:101B30000D0A0000B0B582B001240A2910D88368CC
:101B40007944097949008F440E2905050B0B0B0BCD
:101B50000B0B1A00194909680024224601F0CCFF3A
:101B6000204602B0B0BD506814490860144915A25F
:101B7000184601F067FD0024204602B0B0BD0024E5
:101B8000019403CA09A201AB02F0D4F80228E7D1FC
:101B9000019805F02BF9204602B0B0BD184601F0BF
:101BA0008BFD0024204602B0B0BDC0462B435351EC
:101BB0003A2025642C252A0D0A000000289A0102EB
:101BC0008813000041542B4353510D0A00000000BC
:101BD000B0B582B00546002405F002F901280DD108
:101BE00008498C60E86B426853684B60009401922E
:101BF0006A4601F081FF204602B0B0BDE4432046B2
:101C000002B0B0BDBC930102B0B50546881E0228E3
:101C10000AD3A868012913D0002915D10C490DA2B7
:101C200001F010FD0020B0BD0220014605F08AF849
:101C3000064900242846224601F05EFF2046B0BD3A
:101C400001F03AFD0020B0BD0120B0BDC020010070
:101C50008813000041542B4346554E3D300D0A0079
:101C600080B5E0B00320C10168460FF0C1F9064815
:101C70000078002804D003206A4601460DF0F6FEE5
:101C8000002060B080BDC04669990102F0B597B0F0
:101C900008201490642013902548109002200E9084
:101CA0004B20C0011690234D284614301290012776
:101CB0000F97B802119003200EA906F023FA002610
:101CC000F443002802D0204617B0F0BD0C3528465A
:101CD00001F070FF0028F6D180200C9016490B917E
:101CE0000A9016480990164808901648079016481A
:101CF00006903920059015480490154803900D95DD
:101D0000144D03A9284601F007FD0028DBD10095FA
:101D100001970F4C104911A2124B204601F0A0FE72
:101D20001149204601F0D0FE3446204617B0F0BDE0
:101D300074BF01028896010274C30102F4C3010258
:101D4000E52D0000452E0000B52D00008022010089
:101D5000F899010284C8010260200100414952370C
:101D60003830450080210100611C000010B5034897
:101D7000002404700EF0CAFD204610BDD29E010260
:101D800080B501F04BF9002080BD0000F0B58DB0AA
:101D90000E4600270C970B970A9709970897079705
:101DA00006970597029080680490406B0068019048
:101DB00004F0B2FF04465BA105220392FEF7F6F998
:101DC0005A4D00281ED05AA105222046FEF7EEF9F2
:101DD000002817D058A105222046FEF7E7F9002871
:101DE0000FD059A105222046FEF7E0F9002809D0BE
:101DF00057A105222046FEF7D9F9002807D156A59C
:101E000000E04FA505A820212A4602F065F8012030
:101E10003F2E00D936E0C0467E4436797600B7447E
:101E20003340474A57313131313131313131653009
:101E30003131313131313131313131313131313192
:101E40003131313131313131313131313131313182
:101E50003131313131311F1F1F1F1F1F1F1F1F1F26
:101E6000BE48416A04290CD1039A426287620C2061
:101E700050433D490A580818416805AB049801F0E1
:101E8000E1FB38460DB0F0BDB44C00206062A062AA
:101E9000CD49364A049801F0D5FBA06A401CA062E7
:101EA000EFE7049801F008FC019801F075FEE8E7FF
:101EB000AA48406A05E0A949486A01220243032A68
:101EC0001CD1A649421C4A628F62062ACFD30BE07E
:101ED000A2494A6A012013460343052BD2D1501C64
:101EE00048628F62062803D31E490DE09B48406A72
:101EF0000C2141431C4842584018BDE7886A401CE9
:101F00008862032805D316490022029801F0F4FDE7
:101F1000B7E70E20009000210A220198029B01F0F1
:101F2000DBFDAEE734363030300000009234010083
:101F300034363030320000003436303031000000AA
:101F4000554E494E455400003436303036000000BE
:101F5000343630303300000043544E455400000006
:101F600060200100B0200100341A01000534010096
:101F700070B5022956D30F2907D1784C217A01294F
:101F800005D1002222728F494AE0012070BD866887
:101F900001F036FE002004F0CDFE012803D1002020
:101FA000032104F0CFFE0025284604F0BBFE0128E3
:101FB00004D130346A490022204631E0304600F036
:101FC000EFFD00282ED03046FFF702FE002829D072
:101FD00004F0C2FE012807D15F498D60F06B4268B2
:101FE000E26252684A601AE0022004F09BFE012877
:101FF00008D159498D61F06B4268E26252684A61CA
:1020000010310CE0022004F095FE01280AD152495B
:102010008D62F06B4268E26252684A6220312A4661
:1020200001F06AFD002070BD10B582B003460120AA
:10203000272931D87944097949008F442C132D2D53
:10204000162D2D2D2D2D2D2D2D2D2D2C2D2D2D2DD8
:102050002D2D2D2D2D2D1C2D2D2D2D2D2D2D2D2DC1
:102060002D2D2D2905F046FB15E0DF4900221846ED
:1020700001F042FD0FE00020019003CA08A201AB6D
:1020800001F058FE012806D1019805F04DFC02E050
:10209000024801210172002002B010BDC89901025E
:1020A0002B51495552433A2022636C6F7365642269
:1020B0002C25640D0A000000B0B502294AD30F296F
:1020C00014D18568002004F035FE012803D10020DA
:1020D000032104F037FE0024204604F023FE0128EB
:1020E00006D1D94830301E49002231E00120B0BD70
:1020F0002846FFF76DFD00282CD004F02DFE0128A6
:1021000008D115498C60E86B4268CF4BDA6252689F
:102110004A601CE0022004F005FE012809D10E49A6
:102120008C61E86B4268C84BDA6252684A611031D0
:102130000DE0022004F0FEFD01280BD106498C625F
:10214000E86B4268C04BDA6252684A62203122462C
:1021500001F0D2FC0020B0BD50900102C8990102EC
:10216000E020010080B5022905D3042905D19E494C
:10217000002201F0C1FC002080BD012080BDC046CE
:10218000B0B50546881E02280AD3A868012913D0D5
:10219000002915D10C490DA201F054FA0020B0BD60
:1021A0000220032104F0CEFD0649002428462246E1
:1021B00001F0A2FC2046B0BD01F07EFA0020B0BDC7
:1021C0000120B0BD002101008813000041542B43C1
:1021D00046554E3D310D0A0010B50F290BD001298F
:1021E0001DD000291DD1FFF7C1FD0020022104F000
:1021F000A9FD002010BD0446002004F093FD012835
:1022000003D10020022104F09DFD002004F092FD86
:10221000012804D104490022204601F06DFC002071
:1022200010BD012010BDC046F0200100F0B581B006
:102230000124322928D805468768786B0668C0468D
:102240007944097949008F442F3F1919191F1F1F1D
:102250001F1F1F1F1F1F221F1F1F1F1F1F1F1F1F8B
:102260001F1F1F1F1F1F1F1F1F1F1F1F1F1F1F1F7E
:102270001F1F1F1F1F1F1F1F1F1F26001E49002477
:102280002846224601F038FC204601B0F0BD1B482C
:10229000017800291FD0184900242846224601F061
:1022A0002BFC204601B0F0BD0024FC6239693846A1
:1022B00088470028FAD011480470FC62FFF756FDE9
:1022C0000E20009001220EE0304601F065FC002453
:1022D000204601B0F0BD01210170FFF751FD0E2035
:1022E000009000240522304621462B4601F0F4FBE5
:1022F000204601B0F0BDC046802001002C9A0102AA
:1023000010B586B0034601203B2900D956E0C046EF
:102310007944097949008F445050515133515151FA
:10232000515151515151515151515151515151519D
:10233000515151515151515151515151515151518D
:1023400051515151515151515151515151391D1DFD
:102350001D1D1D1D0020059003CA02AA009218A28F
:1023600005AB01F0E7FC022827D1039A029817A1D8
:10237000FDF71CFF002820D1059805F0D5FA1CE0D8
:10238000B5490022184601F0B7FB16E00020029084
:102390000590049003CA05AA019204AA00920DA216
:1023A00002AB01F0C7FC032807D1049A05990298F3
:1023B00005F082FB029805F0FBFA002006B010BD84
:1023C00025642C2025700D0A00000000434C4F535B
:1023D000454400002B524543454956452C25642C65
:1023E00025643A0D0A256500D0200100012901D895
:1023F0000020704701207047B0B50546881E0328AD
:102400000BD2104604F0B0FC0F48C16A00242846E5
:10241000224601F071FB2046B0BDAC6801290BD00B
:1024200000290ED104F07AFC0346084908A2204690
:1024300001F008F90020B0BD204601F03DF9002070
:10244000B0BD0120B0BDC046C8990102881300008C
:1024500025730D0A0000000070B582B001240F2919
:102460003DD803468568686B0668C046794409799B
:1024700049008F4407141E343434342F3734343435
:102480003434434E6648002404708461C4610121E1
:1024900001716649664A284601F0D4F81FE02846D3
:1024A00001F00AF9304601F077FB0024204602B023
:1024B00070BD5B48002404718269042111430278D5
:1024C000002A2ED0052958D1016A491C016259D22F
:1024D000624961E0524B18780024002831D0204630
:1024E00002B070BD4E4B1878012816D103CA1833BC
:1024F00051A201F01FFC002002B070BD484800242A
:1025000084610121017100784849002812D1484AAC
:1025100011E0434E307900281BD00024204602B041
:1025200070BD052932D10024012101708461C4618C
:1025300001713E493F4A284601F084F8204602B026
:1025400070BD03CA183340A201F0F4FB204602B06C
:1025500070BD002004F0EEFB012803D10020032110
:1025600004F0F0FB0024204604F0DCFB012816D127
:1025700030362D49002430464BE000210162C1690C
:10258000491CC1610E20009000241CE0C169491C57
:10259000C161652915D330490024184639E0284621
:1025A000FFF716FB00289AD004F0D6FB012812D1C1
:1025B0001C4900248C60E86B4268F26252684A60F1
:1025C00027E00E20009002223046214601F084FAD6
:1025D000204602B070BD022004F0A4FB012809D1FE
:1025E000104900248C61E86B4268F26252684A61CB
:1025F00010310EE0022004F09DFB012800D06EE7B0
:10260000084900248C62E86B4268F26252684A62B0
:102610002031224601F070FA204602B070BDC0465B
:10262000C899010250900102E020010088130000C7
:102630002E340100393401002B43475245473A20DC
:10264000252A2C25640000002B435245473A2025BB
:102650002A2C256400000000D020010090200100F9
:10266000B0B584B001243B2900D937E013460546B4
:102670008068C0467944097949008F444B5532320D
:102680002F2F2F2F2F2F2F2F2F2F2F2F2F2F2F2F5A
:102690002F2F2F2F2F2F2F2F2F2F2F2F2F2F2F2F4A
:1026A0002F2F2F2F2F2F2F2F2F2F2F2F2F2F2F2F3A
:1026B0002F2F1D1D1D1D1D1D0024039403CB01AADA
:1026C00000921C4A03AB01F035FB022806D1029AA6
:1026D000019819A1FDF76AFD00280FD0204604B02B
:1026E000B0BD1848006805F01FF9174900242846B6
:1026F000224601F001FA204604B0B0BD114800683E
:1027000005F012F910490022284601F0F5F920469B
:1027100004B0B0BD0B490B601E210CA200F092FF6B
:102720000024204604B0B0BD00F0C6FF00242046BF
:1027300004B0B0BD92350100434C4F5345204F4B80
:1027400000000000309A0102A020010041542B43F8
:102750004950434C4F53453D25640D0A000000008D
:10276000F0B589B0044601203B2900D9AAE01646FD
:10277000A7687A6B1568C0467944097949008F4487
:10278000536AA071A1A1A1A1A1A1A1A1A1A18AA106
:10279000A1A1A1A1A1A1A1A1A1A1A1A1A1A1A1A129
:1027A000A1A1A1A1A1A1A1A1A1A1A1A1A1A1A1A119
:1027B000A1A1A1A1A1A11D1D1D1D1D1D00270897DF
:1027C00003CE06AA0092414A08AB01F0B3FA0228F0
:1027D00077D13F4805680898854272D1079A069ECE
:1027E0003CA130460592FDF7E1FC002847D03DA111
:1027F0003046059AFDF7DAFC002840D03CA130466F
:10280000059AFDF7D3FC0028314E5AD1284605F031
:10281000A5F87068401C706003283CD303207060EA
:10282000306805F023F836E029480660304605F0A8
:1028300071F805902648006805F040F80490244897
:10284000006805F047F80499019102900598012865
:1028500027D02EA026E0384600F02EFF284601F0B3
:102860009BF92EE01A4D286805F078F86868401C3E
:10287000686003280FD300226A6022490DE0144EDD
:102880007760284605F080F8306805F0BBF900282D
:1028900001D01B4900E00C490022204601F02CF930
:1028A0000FE019A000901A491AA23846334600F0EA
:1028B000C9FE0E2000900021B4222846234601F0D4
:1028C0000BF9002009B0F0BDA020010092350100F5
:1028D00000970102414C524541445920434F4E4E0E
:1028E00045435400434F4E4E454354204F4B000048
:1028F000434F4E4E454354204641494C0000000092
:102900004021010060200100544350005544500014
:102910008813000041542B43495053544152543DB5
:1029200025642C222573222C222573222C25750D3B
:102930000A000000B0B582B014468A1E022A12D3E3
:102940008568012917D000291CD1204604F0A8FF72
:1029500000901E210EA22846234600F073FE00249C
:10296000204602B0B0BD09490024224601F0C4F857
:10297000204602B0B0BD284600F09EFE002420464E
:1029800002B0B0BD0124204602B0B0BD502101000C
:1029900041545E4845415254434F4E4649473D31AC
:1029A0002C25642C25750D0A00000000F0B583B0BD
:1029B00014468A1E022A1CD38568012921D00029C9
:1029C00026D1164F3C60204604F05CFFFDF7DAFB91
:1029D0000646386804F056FF7108009101901E21E8
:1029E0000FA22846234600F02DFE0024204603B007
:1029F000F0BD09490024224601F07EF8204603B0CC
:102A0000F0BD284600F058FE0024204603B0F0BD7B
:102A10000124204603B0F0BDA0200100349A010239
:102A200041545E4845415254424541544845583D01
:102A300025642C25752C25730D0A0000F0B585B092
:102A4000044601203B2900D988E0A568794409792A
:102A500049008F444257825E8383838383838383C9
:102A60008383838363838383838383838383838356
:102A70008383838383838383838383838383838326
:102A8000838383838383838383831D1D1D1D1D1D7A
:102A90000020049003CA02AA0092314A04AB01F05C
:102AA00049F9022859D12F4885680498854254D1A4
:102AB000039E029F2CA138463246FDF777FB002883
:102AC0003DD02BA138463246FDF770FB002844D19B
:102AD000284604F029FF29493BE0224CA260104619
:102AE00004F004FF002838D001F08DFAE0600028DF
:102AF00033D0A36840680090234924A2284600F000
:102B0000A1FD2AE017480021C160284600F0D4FD4D
:102B100023E01448806804F007FF19E000F03CFE51
:102B2000012804D10F48C16803C900F03DFF0D48DA
:102B3000C0680CC81349284600F0C4FD0DE02846C3
:102B400004F0D4FE0028074907D0C96801F031FA23
:102B50000B490022204600F0CFFF002005B0F0BD59
:102B6000923501000097010253454E44204F4B001F
:102B700053454E44204641494C000000D0200100FE
:102B8000A0200100204E00008813000041542B4378
:102B9000495053454E443D25642C25750D0A0000CF
:102BA000F0B583B0074601F02BF80026304604F05C
:102BB000A7FE032835460BD10421284605F012F85C
:102BC000F86B51492A4600F097FF304603B0F0BD3C
:102BD00002970024204604F093FE0428254609D1DC
:102BE0000298C06B49492A4600F086FF26463046C7
:102BF00003B0F0BD0027384604F082FE05283D46AC
:102C000009D10298C06B40492A4600F075FF3E4644
:102C1000304603B0F0BD01970125284604F070FE50
:102C20000328029FC8D00125284604F069FE042825
:102C3000D6D00125284604F063FE0528019FE0D088
:102C40000225284604F05CFE0328029FB4D002252A
:102C5000284604F055FE0428C2D00225284604F078
:102C60004FFE0528019FCCD0254C2068401C032135
:102C7000FDF746FA0D46084604F042FE0628029F7C
:102C800008D1284604F032FE002803D001F0BBF939
:102C900000282AD1681C0321FDF732FA0D460846A8
:102CA00004F02EFE062808D1284604F01FFE002856
:102CB00003D001F0A8F9002817D1681C0321FDF703
:102CC0001FFA0D46084604F01BFE0021CE430628DD
:102CD00000D07AE7284604F009FE002800D174E706
:102CE00001F091F9002800D16FE72560F86B0549E4
:102CF0002A4600F001FF0026304603B0F0BDC04672
:102D0000389A0102602101002021010030210100D8
:102D1000B0B582B001220F293ED803468068446BCB
:102D20002468C0467944097949008F44071F252744
:102D3000343535353535353535350A1527490022D1
:102D400004E02649CA68092A20D8521CCA601649DC
:102D5000164A00F077FC1EE0002003F0E3FF012894
:102D600019D11E4830300E49002212E000F0A4FCB8
:102D7000204600F011FF0EE00D4908E00E20009003
:102D800000210122204600F0A7FE04E005490022B0
:102D9000184600F0B1FE0022104602B0B0BDC04699
:102DA000E0200100C020010088130000453401002C
:102DB0007020010080B5032005F08CF980BD000073
:102DC0000648416B0020002905D0054A914203D0F6
:102DD00049680029FAD1704701207047C89901025B
:102DE000B0200100B0B514460D460846114600F06B
:102DF00088FF01281ED1285D00281BD1002C0FD090
:102E00006019401E00780A280AD17B480078002803
:102E100010D003200A4A01462B460CF027FE09E099
:102E200075480078002805D00320054A01462B4646
:102E30000CF01CFE03202946224605F037FAB0BDEF
:102E4000CE330100F0B585B0054604A80024047017
:102E5000E743002D12D0EA68002A0FD0686A0028E4
:102E60000CD0A86A002809D0401EE96A814200D32C
:102E70008EE004A928469047002803D03C4620460F
:102E800005B0F0BD564EE86A411CE962696A049AD1
:102E90000A54E86A696A002202920A54E86A092818
:102EA00006D1696A09224D48FDF773F900283ED022
:102EB0003078411E022908D800F0A2FEB168401AFD
:102EC0004849884264D8464E30780A2820D00128E4
:102ED00023D16E6A3A213046FDF74AF9002847D0DF
:102EE000019002980390E96A03AB30463EA200F0DD
:102EF00021FF02284CD10398002849D00A21384AE2
:102F0000117001990818696A401AC01C50602FE0BE
:102F10007068E96A81422BD13AE004A800780A2857
:102F20000FD00D2814D101202863E86A1AE001208F
:102F3000307000F065FEB0603078411E0229BBD9C8
:102F4000C3E7296B012904D102202863E86A03E062
:102F5000296BE86A022905D1022817D10298E86294
:102F6000286305E0012803D1686A00783E280FD065
:102F7000A86AE96A401E81420AD2EA6804A9284682
:102F800090470028164E00D17DE777E70298286326
:102F9000E96A686A00F0B5FE012819D1E86A0028DC
:102FA0000CD06B6AC018401E00780A2806D112485F
:102FB000007800280CD0032010A206E00E4800780C
:102FC000002805D06B6A032010A201460CF04EFDCC
:102FD00003480470204605B0F0BDC046112D010025
:102FE00088960102DC0500002B52454345495645B1
:102FF0002C252A2C25643A00699901025B41542052
:10300000526563765D202573000000005B4154200B
:10301000526563765D2025730D0A000010B50C24FF
:103020000021204603F000FF054806F0D0FB0121F7
:10303000204603F0F9FE034806F0C9FB10BDC04668
:10304000DC050000B80B0000B0B50F2001F018FE41
:10305000194D6870287033282AD120243721204642
:1030600001F05AFE2120032101F056FE22204021CA
:1030700001F052FE2320082101F04EFE3020AA214B
:1030800001F04AFE0D4802210187322001F044FE82
:103090003320012101F040FE5F21204601F03CFE7B
:1030A0000F2001F0EDFD28700A2006F097FBB0BD5F
:1030B00002480021C187B0BD2C96010256A801022A
:1030C000F0B585B04A4E30788149097881423DD1CA
:1030D000707A20283AD14748022101607A4B0120BA
:1030E000187200245C82B27A5A727079B17909023E
:1030F000081801909882D8813F48323035460B3508
:103100000292570029463A46FDF70EF8B9190B31DD
:103110003A4E30463A466C4FFDF706F803A801993F
:1031200001807978002914D035483230027843780C
:103130001B029A1803AB1B88934204D0801C641CAA
:10314000A142F3D10C463C82312904D9002005B0BC
:10315000F0BD00243C820298002811D05B48026830
:1031600000202B786F783F02FB189A420AD0AD1CE2
:10317000B61C401C029B8342F3D1534F029D16E0C4
:10318000002514E0C5B2284600F03EF84E4F3C8AB8
:10319000A000318809B21B4A115079788C4206D1BF
:1031A000491C79706000164A1018FA894286CAB222
:1031B000787A854207D1A3B2934204D100F024F873
:1031C000002005B0F0BD0028C0D1FB8904AC2380ED
:1031D0000906F3D00A4932310B784C782402E318FF
:1031E00004AC24889C42B1D0891C521EF4D1E5E77E
:1031F000D4D1010290950102FC980102A0D10102F4
:103200005A98010258DE0102F0B581B02D4C2121FF
:10321000009161722C4FB8702C4909886170FA894D
:1032200062717B6B3B622A4D2D782570090AA17073
:10323000110AA17127494143C81827494518BD63A0
:103240000AF0D6FB40190BF02FF806460D4623482E
:10325000007D0AF0B5FE224909882222A15482B2DB
:10326000D20B801802B2D0175210B2186841130E58
:10327000009D6355130C202563553B6FA3761D0AF3
:10328000E5761D0C25771B0E637723462233090A4A
:103290005970A277134DBA66F8662A606860100A02
:1032A000E0770AF00FFC7862BB6B282101222046F0
:1032B0000DF010FEF870388A29180020087201B04D
:1032C000F0BDC0466AD20102689701028C990102E2
:1032D00068990102C0F30000200C0100389001023F
:1032E0006E990102E097010270477047B0B582B055
:1032F000194C2068056801A90020087007E0904774
:103300000198401C01A90870C0B2082822D20122ED
:1033100011048140294209D02268516080002018A0
:10332000826A002AECD001A80121E8E71302834059
:103330002B4201D0022104E082402A42E0D0032146
:10334000134622685360800020188268002AD7D074
:1033500001A8D4E702B0B0BDC8920102FEE70000A8
:1033600010B509480168CA6920231343CB6102697B
:10337000032A08D1012293050C689C430C6051027A
:10338000C26E0A43C26610BD3C93010281B010B503
:1033900081B00393002807D0C16A002904D003AB91
:1033A0000093C46A0021A04701B010BC01BC01B069
:1033B0000047000080B5024608480068002807D092
:1033C00091B2120C03889A4203D040690028F9D1C7
:1033D00080BD002200F0ECFA80BDC04680C801022A
:1033E000F0B581B05C4C2068856BE80707D0E168D8
:1033F000002904D000208847206801218163A807A4
:1034000007D52169002904D00120884720680221BE
:103410008163680707D56169002904D002208847C5
:10342000206804218163280707D5A169002904D0F9
:1034300003208847206808218163E80607D5E169F1
:10344000002904D004208847206810218163A80641
:1034500007D5216A002904D005208847206820214B
:103460008163680607D5616A002904D00620884771
:10347000206840218163280607D5A16A002904D06D
:10348000072088472068802181630126E80507D549
:10349000E16A002904D03702082088472068876342
:1034A000A80507D5216B002904D077020920884799
:1034B00020688763680507D5616B002904D0B702CF
:1034C0000A20884720688763280507D5A16B002953
:1034D00004D0F7020B20884720688763E80407D5EB
:1034E000E16B002904D037030C20884720688763EC
:1034F000A80407D5216C002904D077030D20884744
:1035000020688763680407D5616C002904D0B7037D
:103510000E20884720688763280407D5A16C0029FE
:1035200004D0F7030F20884720688763E80307D596
:10353000E16C002904D03704102088472068876395
:10354000A80307D5216D002904D0750411208847F0
:103550002068856301B0F0BDCC930102F0B58DB059
:10356000002862D00446406800285ED0A068402849
:103570005BD8E56A002D58D007462046403000262B
:10358000039003E0019E4AE0039848E040210122B5
:103590000691FCF7DBFDAE4202963ED2002031469A
:1035A000019009900398069B3E46002EEAD0606A7F
:1035B0000491405C07900998401C05900021042765
:1035C00008916518EA5C012A17D10A966268D31936
:1035D0001B1F1B68099E9E5D0798864208D1059DAA
:1035E0005B5D002B0A9E22D00898401C089003E0E7
:1035F000403500222A70A668069B0837491CB14254
:10360000DFD308980028BFD00499491CE06A8142A2
:10361000059809900398C8D301E003983E463746C1
:10362000E56A029E761CAE42B0D30DB0F0BD616A71
:103630000B91E16A0C91D1590BAA204600F09CF83D
:103640000DB0F0BD81B0B0B583B00D460446079310
:1036500007AB02938069E1690DF0CAFC20626548FE
:103660000078002803D1216AA06900F09FF96369FE
:10367000A169226A204698470146A06B002905D01F
:1036800069460C600021224B0A460CE000F084FAE7
:103690007D2081002846FCF71DFD0246A06B69468F
:1036A0000C6000211B4B00F0D3FA002003B0B0BC2B
:1036B00002BC01B00847C04680B5806B00F06CFAD0
:1036C000002080BD70B582B00D46044646691146A3
:1036D0001A46B0470146A06B002907D069460C6026
:1036E00000210B4B0A4600F0B3FA0EE000F054FA4A
:1036F0007D2081002846FCF7EDFC0246A06B694660
:103700000C600021034B00F0A3FA002002B070BD52
:10371000FD3700001338000070B50D4604468021C7
:1037200000F0C0FA2868E06368686060A868A0607C
:10373000E868E0602869206168696061A869A06143
:10374000E86900262662E061286A6062686A26638A
:10375000E662A062A86A60632046383000F02AFA68
:10376000002802D0F643304670BD21480168216030
:103770000460304670BDC04670B514460D4606461E
:10378000881E032802D8B06B00F006FAF06B2946B9
:10379000224600F00DF970BD16480178012048401E
:1037A0007047C04670B512480468002C1FD0114EF7
:1037B00011A5216920468847002815D130780028B6
:1037C0000DD1E16A606A00F09CFA0146606A012945
:1037D00003D0E16A00F0E8F8284600F0E3F820465C
:1037E000FFF7BCFE0020E0622468002CE1D170BD30
:1037F0007CC8010274C801020D0A000010B504461D
:10380000806B00F0C9F9E06B0521002200F0D0F8D0
:1038100010BD10B50446806B00F0BEF9E06B0421CA
:10382000002200F0C5F810BDF0B581B00091064649
:10383000C7680468A01C3946FCF74CFC002570687A
:10384000814201D1ED430BE0601C3946FCF742FC9C
:10385000316032695143B06808180099FCF764FC84
:10386000284601B0F0BDB0B50124002505604460D4
:1038700008300EC0B0BD70B50E460446C168006881
:10388000401CFCF727FC00256068814202D1ED4313
:10389000284670BD22695043A16841183046FCF7A4
:1038A00043FCE1686068401CFCF714FC616028463A
:1038B00070BDB0B5002400280DD0054600688842D0
:1038C000FDD3401A286068684018E968FCF702FCDC
:1038D00069602046B0BDE4432046B0BDB0B50024C9
:1038E00000280ED00546006840182860EA6890421B
:1038F000FDD8A86840181146FCF7ECFBA9602046EB
:10390000B0BDE4432046B0BDF0B583B016460246D4
:103910000027F843002E22D01C46002B1FD00D4656
:10392000D168136899421AD9CB1AAB4217D392685F
:10393000019252198A423A4607D9019A8A1A02928A
:10394000029A52199342029A09D3029201981018CE
:10395000FCF7C0FB3160029840192060384603B084
:10396000F0BD406870478068704702460020002A1A
:1039700004D0106050609060D1607047C0437047C1
:10398000002803D001684842484170470120704731
:10399000002805D00168C068411A48424841704774
:1039A00001207047002070470020704700207047BA
:1039B000F0B583B014460D4606464088012818D15C
:1039C000306900280CD0A900405801782D2910D06A
:1039D000F368716809686A461160506010A205E0DA
:1039E000F36870680068694621C115A23046FFF788
:1039F000CDFC7768FB683046294622469847012867
:103A000008D00AE0C36830462946224698477F68B6
:103A1000012802D178680028F4D103B0F0BDC04677
:103A200046534D3A252D38732053544154453A2579
:103A30002D323873204556454E543A25730D0A00F1
:103A400046534D3A252D38732053544154453A2559
:103A50002D323873204556454E543A25750D0A00CF
:103A6000F0B581B0002828D01E460C460546079BBD
:103A70000698009000206862A862E86210490988F0
:103A80006B8029800F4B1F686C60009BAB602B46DE
:103A90000C33C4C3A861E8612862481C0849088047
:103AA00008480560002C08D06C60002128460A46B2
:103AB000FFF77EFFA468002CF6D101B0F0BDC04630
:103AC00004CC010280C8010202460020002A01D075
:103AD000D1627047C043704710B582B004AC2488EF
:103AE0001B881B041B196C462360024B00F0B0F8C6
:103AF00002B010BDB5330000F0B597B01646029184
:103B000005464268002A30D001966A6001210024EF
:103B1000284616462246FFF74BFF3046029FBE421C
:103B200032D003A85021FCF718FB32467268002FF0
:103B30000CD003AF029811C74068083F824209D0F9
:103B4000394608313C4600280F46F4D1002A019E30
:103B5000DBD10AE0019E38686860002128463246C1
:103B6000FFF726FF7F68002FF5D102988468002CAC
:103B700008D06C60002128463246FFF719FFA46880
:103B8000002CF6D117B0F0BD00212846019E324628
:103B9000FFF70EFFE9E70000014600201F2901D9C9
:103BA000C043704718224A43344901238B50891877
:103BB0008860704710B50021CC4300280BD00A4A1A
:103BC0001368002B09D01832491C2029F8D306D1DC
:103BD00006A0FFF7E7FE204610BD01231360016039
:103BE0000024204610BDC04604C9010274696D65F9
:103BF000722049442069732066756C6C0D0A0000C0
:103C0000264800687047C04670B520241B4D234EDF
:103C10002868022817D13068A968EA68401A9042DB
:103C200011D96969002907D02879002807D0022016
:103C300028603068A86004E00120286003E00120CB
:103C40002860286988471835641EE1D170BDC046D8
:103C5000F0B5044600201F2C01D9C043F0BD059DDE
:103C600018266643054C0227A751A41921710B4958
:103C700009682646083626C66361F0BD04C90102FC
:103C800006480168491C0160054841680268002334
:103C9000521C02604B4143607047C046B0AC010209
:103CA000B8AC010280B5FCF758FA80BDB0B5027817
:103CB000002A24D0441C0021084601E0573A08E0BD
:103CC00023460001D5B2302D0C4611D3392D02D830
:103CD000303A14460CE0412D0C4609D3462D01D84C
:103CE000373AF6E71446613CE4B2062CE6D30024EA
:103CF000E2B280185C1C1A78002AE1D1B0BD002025
:103D0000B0BD10B50246012000290DD00023D45CBF
:103D1000202C02D37F2C04D307E00D2C01D00A2CD9
:103D200005D15B1C8B42F2D310BD002010BD0020DA
:103D300010BD000081B0F0B584B009930023039357
:103D4000002800D1C2E0002A00D1BFE009AB0393F4
:103D50001678002E00D1A8E05623DB430093002301
:103D60001D46002900D1A2E0252E3FD1971C527894
:103D70001446643C0023142C43D8C0467C44247968
:103D80006400A7440A99A3A3A3A3A3A3A3A3A3A3E3
:103D90004CA3A3A3A3A3A3A35F000297039A131D9D
:103DA0000393126801920122002317461E460478ED
:103DB000FF0703D02D2C01D1164607E02746303FE0
:103DC000092F09D80A275F433B19303B491E401C85
:103DD00000270029EBD13946029A019C002C03D020
:103DE000012E00D15B4223606B1C06E00378B342D6
:103DF0005BD1491E521C401C2B461678002EAFD1B9
:103E000064E02A2A62D13A780378934204D0491EAA
:103E1000401C0029F8D100216B1C3A46EDE7039ABB
:103E2000131D03933E7812680023C45CB44233D060
:103E3000491E5B1C0029F8D13C46C7180021002A06
:103E40002ED12EE00297039A131D039312680023CC
:103E5000009E0778302F18D33A2F02D234462734E9
:103E60000BE0612F03D3672F344606D30DE03C46A9
:103E7000413C052C09D8344620341B011B19DB19A1
:103E8000491E401C0029E4D10021029C002A00D0D8
:103E900013606B1C2246B0E73C46C718002A00D0CE
:103EA00009C26B1C22463846A7E700230EE0252EE8
:103EB0000BD15178652908D103990A1D039209682D
:103EC000002900D008606B1C00E02B46184604B0A7
:103ED000F0BC02BC01B0084781B010B581B00C46FF
:103EE000039303AB00930DF083F8A04200D3601E50
:103EF00001B010BC02BC01B0084770B504460020F8
:103F0000002A1BD0002C19D0002B17D014600120E0
:103F1000022B13D32578002D10D0641C01208D4274
:103F200005D1651E00262E7085005451401C984214
:103F300004D2661C2578002D3446F0D170BDB0B592
:103F400004467821FCF714F9002805D158212046B1
:103F5000FCF70EF9002828D04278002A23D0841CD0
:103F60000021084623460001D5B2302D0C4613D35C
:103F7000392D01D8303A0EE0412D0C460CD3462D98
:103F800001D8373A07E01446613CE4B2062C01D36D
:103F9000002401E0573A1446E2B280185C1C1A78FB
:103FA000002ADFD1B0BD0020B0BD2046FCF7A0F94B
:103FB000B0BD70B504460026F043002C0DD00D4670
:103FC00000290AD0204610300121FFF772FCA968B1
:103FD00020342046FFF76DFC304670BD70B50446B6
:103FE0000026F043002C0DD00D4600290AD02046B3
:103FF00010300121FFF772FCA96820342046FFF73A
:104000006DFC304670BD70B50024002814D0054604
:10401000064610363046FFF7B3FC01280CD0284680
:104020002030FFF7ADFC012806D02C683046FFF7A2
:1040300098FC0C2141436418204670BDF0B583B054
:1040400000250295019500281FD00C46064607461C
:1040500010373846FFF79CFC002816D13046203038
:1040600002AA01AB2146FFF74FFC00280DD13568AD
:104070003846FFF778FC0C214143B068029A1018CB
:1040800068506D186C600198A860284603B0F0BDB8
:1040900070B505460C2058430024904211D2121AE4
:1040A000461829606860AE60EA60284610301946FC
:1040B000FFF75BFCE96820352846FFF756FC2046F1
:1040C00070BDE443204670BD04217046084204D010
:1040D000EFF30983EFF3088203E0EFF30883EFF3D4
:1040E00009829BB004A8F0C044464D4656465F4640
:1040F00008A8F0C01846F0C86846F0C018690C90CF
:10410000202018440D9058690E9098690F90D86936
:104110001090EFF310801190EFF314801290094982
:1041200008681390084908681490084908681590B1
:1041300007490868169017931892704619906846B8
:104140000AF052FE04ED00E00CED00E010ED00E09E
:1041500014ED00E0F0B581B003260024304621467E
:1041600007F094FA04252846214607F08FFA012724
:10417000304639463A4607F061FA30462146324623
:1041800007F0ACFA284639463A4607F057FA0221BA
:104190002846224607F0A2FA01B0F0BDF0B589B07A
:1041A00008900425284607F031FA0A27384605F01A
:1041B00015FB284607F03AFA0324204607F02EFAAA
:1041C00007900526304605F009FB284607F01EFA41
:1041D000384605F003FB284607F028FA204607F08A
:1041E0001DFA0690304605F0F9FA284607F00EFA57
:1041F000384605F0F3FA284607F018FA204607F08B
:104200000DFA0590304605F0E9FA284607F0FEF968
:10421000384605F0E3FA284607F008FA204607F08A
:10422000FDF90490304605F0D9FA284607F0EEF97A
:10423000384605F0D3FA284607F0F8F9204607F08B
:10424000EDF90390304605F0C9FA284607F0DEF98B
:104250003846019705F0C2FA284607F0E7F92046EC
:1042600007F0DCF90290304605F0B8FA284607F06E
:10427000CDF9384605F0B2FA284607F0D7F92046BE
:1042800007F0CCF90746304605F0A8FA284607F0B3
:10429000BDF9019805F0A2FA284607F0C7F92046B3
:1042A00007F0BCF90446304605F098FA284607F0B6
:1042B000ADF90699481E81410A460799481E814179
:1042C000480080188000059A511E8A41510040180C
:1042D000049A511E8A4180188000039A511E8A4117
:1042E00051004018029A511E8A4180188000791EA0
:1042F0008F4179004018611E8C41061908980028EA
:1043000003D0032007F082F902E0032007F08EF9C2
:104310000A24204605F062FA0425284607F086F9AB
:10432000204605F05BFA284607F070F9F0B209B0B4
:10433000F0BDF0B589B008900324002120460A465C
:1043400007F07CF90427384607F060F90626304666
:1043500005F044FA384607F069F9204607F05EF99F
:1043600007900525284605F039FA384607F04EF93A
:10437000304605F033FA384607F058F9204607F082
:104380004DF90690284605F029FA384607F03EF91F
:10439000304605F023FA384607F048F9204607F082
:1043A0003DF90590284605F019FA384607F02EF930
:1043B000304605F013FA384607F038F9204607F082
:1043C0002DF90490284605F009FA384607F01EF941
:1043D000304605F003FA384607F028F9204607F082
:1043E0001DF90390284605F0F9F9384607F00EF953
:1043F000304605F0F3F9384607F018F9204607F083
:104400000DF90290284605F0E9F9384607F0FEF864
:10441000304605F0E3F9384607F008F9204607F082
:10442000FDF80190284605F0D9F9384607F0EEF876
:10443000304605F0D3F9384607F0F8F8204607F083
:10444000EDF80646284605F0C9F9384607F0DEF8CB
:104450000898821E501E82410121204607F0EEF886
:104460000799481E8141069A501E8241500040180B
:10447000059A511E8A4191000818049A511E8A41DA
:10448000D1000818039A511E8A4111010818029A96
:10449000511E8A4151010818019A511E8A41910109
:1044A0000143701E8641F0010843C0B209B0F0BD5F
:1044B00070B50446042007F0A9F860B2002803D4C0
:1044C000032007F0A3F802E0032007F0AFF80A2565
:1044D000284605F083F90426304607F0A7F8284659
:1044E00005F07CF9304607F091F8284605F076F99A
:1044F000600603D4032007F089F802E0032007F0E8
:1045000095F80A25284605F069F90426304607F093
:104510008DF8284605F062F9304607F077F828460E
:1045200005F05CF9A00603D4032007F06FF802E061
:10453000032007F07BF80A25284605F04FF90426EA
:10454000304607F073F8284605F048F9304607F082
:104550005DF8284605F042F9E00603D4032007F091
:1045600055F802E0032007F061F80A25284605F017
:1045700035F90426304607F059F8284605F02EF99B
:10458000304607F043F8284605F028F9200703D401
:10459000032007F03BF802E0032007F047F80A2564
:1045A000284605F01BF90426304607F03FF8284658
:1045B00005F014F9304607F029F8284605F00EF901
:1045C000600703D4032007F021F802E0032007F07E
:1045D0002DF80A25284605F001F90426304607F093
:1045E00025F8284605F0FAF8304607F00FF8284677
:1045F00005F0F4F8A00703D4032007F007F802E061
:10460000032007F013F80A25284605F0E7F80426EA
:10461000304607F00BF8284605F0E0F8304606F083
:10462000F5FF284605F0DAF8E00703D1032006F08D
:10463000EDFF02E0032006F0F9FF0A24204605F012
:10464000CDF80425284606F0F1FF204605F0C6F80F
:10465000284606F0DBFF204605F0C0F870BD70B5B7
:104660000446042006F0D2FF60B2002803D40320E1
:1046700006F0CCFF02E0032006F0D8FF0A2528460A
:1046800005F0ACF80426304606F0D0FF284605F0C9
:10469000A5F8304606F0BAFF284605F09FF86006F8
:1046A00003D4032006F0B2FF02E0032006F0BEFFB1
:1046B0000A25284605F092F80426304606F0B6FF93
:1046C000284605F08BF8304606F0A0FF284605F096
:1046D00085F8A00603D4032006F098FF02E003202B
:1046E00006F0A4FF0A25284605F078F8042630468F
:1046F00006F09CFF284605F071F8304606F086FF6C
:10470000284605F06BF8E00603D4032006F07EFF90
:1047100002E0032006F08AFF0A25284605F05EF82D
:104720000426304606F082FF284605F057F830464A
:1047300006F06CFF284605F051F8200703D403204B
:1047400006F064FF02E0032006F070FF0A25284609
:1047500005F044F80426304606F068FF284605F0C8
:104760003DF8304606F052FF284605F037F860075E
:1047700003D4032006F04AFF02E0032006F056FFB0
:104780000A25284605F02AF80426304606F04EFF92
:10479000284605F023F8304606F038FF284605F095
:1047A0001DF8A00703D4032006F030FF02E0032029
:1047B00006F03CFF0A25284605F010F8042630468E
:1047C00006F034FF284605F009F8304606F01EFFD3
:1047D000284605F003F8E00703D1032006F016FF92
:1047E00002E0032006F022FF0A24204604F0F6FF30
:1047F0000425284606F01AFF204604F0EFFF28465D
:1048000006F004FF204604F0E9FF70BDF0B581B06A
:1048100003260025012430462946224606F00EFFD5
:10482000304606F003FF0626304604F0D7FF04208A
:1048300006F0FCFE304604F0D1FF032006F0EEFE49
:1048400000281BD0681CFA2D0546F6D304252846FF
:1048500006F0DCFE0326304606F0D8FE0A2738466E
:1048600004F0BCFF284606F0E1FE304606F0DEFE0E
:10487000384604F0B3FF204601B0F0BD032001210B
:104880000A4606F0DBFE042006F0C0FE00242046A7
:1048900001B0F0BDF0B581B00326002501243046FB
:1048A0002946224606F0CAFE304606F0BFFE06261E
:1048B000304604F093FF042006F0B8FE304604F0C2
:1048C0008DFF032006F0AAFE002820D0681CFA2DD8
:1048D0000546F6D30426304606F098FE0325284602
:1048E00006F094FE0A27384604F078FF304606F0BA
:1048F0009DFE284606F09AFE384604F06FFF2846D3
:104900002146224606F09AFE204601B0F0BD032063
:1049100001210024224606F091FE042006F076FED6
:10492000204601B0F0BD0000F0B583B01C460092F7
:10493000019106460325284606F078FE04273846EE
:1049400006F074FE284606F061FE0A20029004F08C
:1049500045FF384606F05AFEFE203040FFF77FFE46
:10496000FFF798FF5C4908610198FFF778FEFFF7B1
:1049700091FF59494861284606F058FE384606F02E
:1049800055FE284606F042FE029804F027FF3846FE
:1049900006F03CFE012006433046FFF760FEFFF7BD
:1049A00079FF4D498861002C38D0E0B2FFF7C1FC97
:1049B000009D2870042006F029FE012C1DD06F1CDC
:1049C000032006F023FE0A26304604F007FF0425E4
:1049D000284606F02BFE304604F000FF284606F07D
:1049E00015FE641EE0B2FFF7A4FC3870284606F0FE
:1049F0000DFE7F1CA0B20128E2D1032006F016FEB6
:104A00000A24204604F0EAFE0425284606F00EFE9D
:104A1000204604F0E3FE284606F0F8FD0424204674
:104A200006F0F4FD0325284606F0F0FD0A26304680
:104A300004F0D4FE204606F0F9FD284606F0F6FD07
:104A4000304604F0CBFE03B0F0BDC046F0B583B0F5
:104A500000AC0EC407460324204606F0E7FD0425FB
:104A6000284606F0E3FD204606F0D0FD0A26304633
:104A700004F0B4FE284606F0C9FDFE200740384683
:104A8000FFF7EDFDFFF706FF134F38600098FFF7C3
:104A9000E6FDFFF7FFFE78600198FFF7E0FDFFF706
:104AA000F9FEB8600298FFF7DAFDFFF7F3FEF86051
:104AB000284606F0ABFD204606F0A8FD304604F07F
:104AC0008DFE284606F0B2FD204606F0AFFD3046CA
:104AD00004F084FE03B0F0BDD495010270B5044625
:104AE0004D4E307001202040707003D1032006F03D
:104AF0008DFD02E0032006F099FD0825284606F00A
:104B000095FD284606F082FDA007C00F707003D106
:104B1000032006F07BFD02E0032006F087FD082558
:104B2000284606F083FD284606F070FD6007C00F9A
:104B3000707003D1032006F069FD02E0032006F047
:104B400075FD0825284606F071FD284606F05EFD35
:104B50002007C00F707003D1032006F057FD02E05C
:104B6000032006F063FD0825284606F05FFD284671
:104B700006F04CFDE006C00F707003D1032006F074
:104B800045FD02E0032006F051FD0825284606F009
:104B90004DFD284606F03AFDA006C00F707003D107
:104BA000032006F033FD02E0032006F03FFD082558
:104BB000284606F03BFD284606F028FD6006C00F9B
:104BC000707003D1032006F021FD02E0032006F0FF
:104BD0002DFD0825284606F029FD284606F016FD7D
:104BE000E009707060B2002803D4032006F00EFDC7
:104BF00002E0032006F01AFD0824204606F016FD08
:104C0000204606F003FD0724204606F00FFD20464F
:104C100006F0FCFC70BDC046D095010202488069D8
:104C2000811E4842484170474C96010280B5FDF70D
:104C30002DF8002801D00020C04380BD80B5FEF7CC
:104C4000BFF880BD10B504480F2100242246FEF7AE
:104C5000AFFE204610BDC046F8990102B0B507244A
:104C600000252046294606F011FD012120462A464E
:104C700006F0E4FC022120462A4606F02FFDB0BDD6
:104C8000F0B581B007460324204606F0CFFC04258A
:104C9000284606F0CBFC204606F0B8FC0A26304633
:104CA00004F09CFD284606F0B1FC3220FFF700FC22
:104CB000FFF7ACFDF8B2FFF7FBFBFFF7A7FD2046BF
:104CC00006F0B4FC284606F0B1FC204606F09EFC37
:104CD000304604F083FD284606F098FC3320FFF7A9
:104CE000E7FBFFF793FD0020FFF758FA0746284639
:104CF00006F08CFC204606F089FC304604F06EFD80
:104D0000284606F093FC204606F090FC304604F05E
:104D100065FD384601B0F0BDF0B581B000910746A1
:104D20000324204606F082FC0426304606F07EFC72
:104D3000204606F06BFC0A25284604F04FFD30465D
:104D400006F064FC3220FFF7B3FBFFF75FFDF8B21B
:104D5000FFF7AEFBFFF75AFD0098FFF7A9FBFFF73F
:104D600055FD304606F052FC204606F04FFC284622
:104D700004F034FD304606F059FC204606F056FC9F
:104D8000284604F02BFD284604F028FD01B0F0BDB4
:104D900080B5074801210170064802680A43026095
:104DA00005480268002A02D000200146904780BDD5
:104DB0000ACC01021C1000500CCC0102F0B599B0D5
:104DC000F548017BC67A427B0E92F44C221F136891
:104DD000F34A1268069242780C9202790592C76AE9
:104DE00004931F4001200F907A0200D5BCE03A02E4
:104DF00000D5BFE0FA0102D50F98020622605025C7
:104E000008968A191826BB0102D50F98430623601D
:104E10004123079569430A96354655431426FC02FB
:104E200010D50F98040538463746DC4E3460DA4C0E
:104E3000A469B464D84CE4697464DA4C241D346009
:104E40003E46074690000B90D8040D9068180990D4
:104E50000E9B73430F988203B902D04D22D50F9851
:104E600041052960CC480E9616460246816929659F
:104E7000C169696509990D980143089800010818EE
:104E80000B994018C018C849098892794A4380187C
:104E90000A301C4604F082FF234632460E9EC0496B
:104EA00088672A600F98C404380300D52C60F80383
:104EB00002D50F98000428600F984104B80300D56C
:104EC0002960380400D4E4E1039402910E9308921F
:104ED0000D980B990C180A980C9941430C910F9856
:104EE000C0030B90286007F091FD002801D004F06A
:104EF00037FF0C98005B410B43D1099800190E99BC
:104F000040180599090140180E90E74D287B079B32
:104F10004343E97A0A010D9C2243D21841188B00C1
:104F2000D2180A9B4B43D1186A7B564389190E9EAF
:104F30002A791018DF4A1288424388181690306880
:104F4000C000800D10A9C882002511957079C00796
:104F50007ED110A80F998182069C00940020E8A2BF
:104F6000049B0AF083FD78E00F98820522603A02E4
:104F700000D43FE70F98C2052260FA0100D53BE755
:104F80003DE7072149030840032149038842089A65
:104F900000D07EE1069707F053F9002016900990A3
:104FA0001590C14CE07A217B08180A994143800092
:104FB0000D9A10434118627B0E9672438A186178ED
:104FC000A379079E7343D718FA683F263240637867
:104FD0009A420C976ED105960A9A4A4380580F213F
:104FE0000A0702400398401EC04B1B68DB090340C0
:104FF000981810900F98C0020B90B868800767D47B
:105000002C46283C09F0A8FC05462068000609D576
:10501000C3208401786A400704D409F09DFC401B3A
:10502000A042F7D905980002B96849080140B34881
:1050300003688268B868C40C20202040DB0700D0D9
:1050400095E0002310221D461C460E9E0B9FB1E0EA
:1050500010A88582B0681190069C701D924B19793A
:10506000E20707D1491C1971D97A1A798A4202D309
:105070001D7100E0D97001784278120251188278CF
:105080001204891803229143017035715878401C2D
:105090005870D87A197B08185978884200D85D7002
:1050A000D879401ED871596B002901D010A88847C3
:1050B0007E4DEDE010A80B998182F868304063784E
:1050C000009000207CA20F990AF0D0FC0E9E94E084
:1050D000388A874A024010A8C2822022BA5C93070D
:1050E000DB0F3C68C3720F9B1A4082726205D20CC0
:1050F0000D9B1A431692FA68130E0372BB69FC6982
:105100007C4D2D682D0C05745204920F4272119340
:105110001394654CA07B002809980E9E0B9F5FD0CE
:1051200075480068007A0328099859D00C98007DCA
:1051300008400928099853D1C320840109F00CFCC8
:1051400005460C98406A41070BD45949096809067D
:10515000890F06D109F000FC401BA042F1D90C9840
:10516000406A41030898884310A9888237E0D20733
:105170000E9E0B9F03D108230022154619E00C9BBD
:105180009A68029C224211D19A68520C02249443DC
:105190000022134615460DE010D1010228A0005050
:1051A0003CA10050FC1F00000CD10102042500228C
:1051B000134614460843104318432843204310A9BC
:1051C000888238420BD10C9B198A494A0A4010A99F
:1051D000CA8219684905C90C0D9A11431691324CBF
:1051E0002921615C002908D03037B84205D010A9C8
:1051F00008461130123108F0F9FEE77A2A48047B9C
:10520000E519294800790E9027484078401C294626
:10521000FAF760FF88000D9A1043189007996143D0
:105220003801104340182049497B4E4380191C2106
:10523000694340180E9909191B4B1E4A12884A43AC
:1052400080181790099A0C998A60987B002800D0E2
:105250004A629879401C9871187B99798142069F1F
:1052600000D39A715978491C5970D97A081859781D
:1052700088420E4D00D85A70187A401E18722820A5
:10528000185C002804D0996B002901D010A8884729
:10529000089A174202D00F98000328601C4804495E
:1052A000486019B0F0BDC04610D1010228A00050DE
:1052B0003CA100500CD1010248572045542069649C
:1052C0007820256420616E6420455420696478202C
:1052D000256420696E2052582064657363206D69CF
:1052E000736D617463680D0A00000000382000408F
:1052F000FF030000943000403894010260400040F9
:105300004D4143204556542025782025780D0A002C
:10531000FFFFFF03F0B5A5B01E460C9208910024D4
:10532000239422A90C8016A90C8024A909250D809C
:10533000598C0D91FAF7CEFE2A99012900D0DFE0B1
:105340003189012900D0DBE0318C012900D0D7E080
:105350000D99002900D1D3E0224607962C990B9194
:105360002B99069180B205900F9415A805809000A6
:105370000E900C990C582E460025204629461746BB
:10538000FBF72AFA0028119636D12C200A97784389
:105390000899081817A90A4668C868C2E8C8E8C288
:1053A000E8C8E8C2079F119880B280000E5822AD6D
:1053B000019523A8009020463946059A069B04F0E3
:1053C0001BFA0F98401C0F90288800282DD03B8A8C
:1053D000239913AC039416A8029014A8019015AE5B
:1053E000009617A824AA04F0E1FB258830881190C4
:1053F0000120149E0A9A05E013A8058014952E46F4
:1054000028463A460E9F51000B9B119C5C5259183E
:1054100008830D84D81986600F981885521C0D9842
:1054200082426DD024A805889FE7099616A800251A
:105430000580149524A80688239812902F4610956D
:1054400003E06D1CA8B2B04213D8A8B2800017A91F
:105450000C5820461299FBF7CDF90028F1D1002F06
:10546000EFD115A8058016A8012707801494109481
:10547000E7E715A80288B01A012805D115A806800B
:10548000099F1497119628E010200799095E0129B9
:10549000119221DB551CA8B20C18109F0E9B099489
:1054A00003E06D1CA8B2844218DDAAB2B242F8D85B
:1054B000800017AA10581090394634461E46FBF754
:1054C0008BF933462646099C0028EAD115A80580A9
:1054D000109F14971195E4E7109F0E9B1C463E46C3
:1054E00038461299FAF7A7FFFBF7F4F905460528A5
:1054F00000D3052513A8058001200A9A274682E7D4
:1055000025B0F0BDF0B58BB00243159A149C139EE4
:105510002BD0054601A856C0129CD869196A09907B
:105520000A911E469F6B0123009309A807AA014612
:10553000059306F0F9F8716C3846FAF77CFF0746D8
:10554000E06A616BFAF777FF002D069613D00446E8
:1055500011980199012924D10921081A0421069AD8
:10556000515E884229D16425B1E00020308020704E
:1055700010700BB0F0BDB08800226425002829D03F
:10558000059269493846FBF751F90028049C039EAF
:105590006FD166493846FBF749F900281DD05A25D6
:1055A00067E03C25082800D191E05F492046FBF7E1
:1055B0003DF9002819D0502589E00A291DDB1D2955
:1055C0003BDC59493846FBF731F90022002854D01A
:1055D0005A253AE03346049C39E055493846FBF7F2
:1055E00025F9002821D0502543E050492046FBF7FB
:1055F0001DF900282ED0462569E03C25012866D0FB
:1056000049492046FBF712F90028D4D147492046E2
:10561000FBF70CF90028EED145492046FBF706F9C7
:10562000002854D1434920466EE042493846FBF7F2
:10563000FDF800281CD128251BE03B493846FBF724
:10564000F5F80022002832D05025049C069B0299D0
:10565000039E41E036492046FBF7E8F8002836D1A2
:1056600034492046FBF7E2F800282FD114252EE01C
:1056700037250299059A069B2EE005922B4938465C
:10568000FBF7D4F8002896D129493846FBF7CEF825
:105690000028B0D127493846FBF7C8F80028049CF9
:1056A000069B0299039E059A3BD11E2514E00592A4
:1056B0001E493846FBF7BAF800289CD11C493846E9
:1056C000FBF7B4F800281DD03C2500E02325049CFE
:1056D000069B0299039E059A25803270002008706F
:1056E000307800280CD118681349FBF791F800288E
:1056F00006D12088102803D30F3820800BB0F0BDCE
:105700000BB0F0BD0B493846FBF790F80028049C1D
:10571000069B0299039E059A01D11425DCE72325F7
:10572000DAE72D25D8E7C046CDCCCC3DCDCC4C3DDD
:10573000CDCCCC3C0AD7233C0000204070B588B0CB
:105740000C4606464088002820D0FBF7ADF80590AF
:1057500005A804A901252A4606F050FA3088B18828
:10576000081AFBF796F80390049903A807AA2B469A
:1057700006F004FA5249079D2846FBF757F800281F
:1057800008D0BF200006206008B070BD0020206057
:1057900008B070BD4B492846FBF72CF8002804D010
:1057A0003F200006206008B070BD47492846FBF73F
:1057B0003DF8002801D0002010E000212846FBF72A
:1057C00035F8002801D0022008E040492846FBF7C0
:1057D0002DF8002801D0042000E0062001957F214B
:1057E000C905029180003A49091801A806AA0223B6
:1057F00006F078F90698206008B070BDF0B587B063
:105800000C4605464768002638463146FBF71CF82B
:10581000002802D0266007B0F0BD049704A803A9B1
:105820000126324606F0EAF9A8682968FAF7BEFDB3
:105830000290039902A806AA334606F09FF9204970
:10584000069D2846FAF7F2FF002804D0BF2006067E
:10585000266007B0F0BD1B492846FAF7CBFF0028A9
:1058600004D03F200606266007B0F0BD1649284642
:10587000FAF7DCFF002801D0002010E000212846C4
:10588000FAF7D4FF002801D0022008E00F4928468B
:10589000FAF7CCFF002801D0042000E00620009594
:1058A0007F21C9050191800009490918684605AAA8
:1058B000022306F017F9059E266007B0F0BDC0462A
:1058C000CDCC0C3F295C0FBFCDCC4C3ECDCC4CBEDB
:1058D00040940102F0B587B00C4606467F27008849
:1058E000002801D0FD0503E0B08800282ED0334DFC
:1058F000FAF7DAFF03907088FAF7D6FF049003A84E
:1059000002A90126324606F079F9029904A806AAEE
:10591000334606F033F92A49069E3046FAF786FFE9
:10592000002802D03F20010641E026493046FAF720
:1059300061FF002802D0BF20010638E0224930462E
:10594000FAF774FF002805D0002024E00020206032
:1059500007B0F0BD1D493046FAF768FF002801D0B6
:10596000022018E01A493046FAF760FF002801D0FB
:10597000042010E017493046FAF758FF002801D0FC
:10598000062008E014493046FAF750FF002801D0FD
:10599000082000E00A200096F905019180000F49D7
:1059A0000918684605AA022306F09CF805992846BE
:1059B000FAF704FD206007B0F0BDC046000080BFCC
:1059C000000038433333733F0000C8420000704288
:1059D000000020420000A0410000C040609401028D
:1059E000F0B59DB015460B917F210391C9051C911F
:1059F00002911B9119A900248C8019941894179472
:105A0000598C0691198C0F91DE8B998B079199789F
:105A100005911F882B21CA432799914201DB7F0002
:105A200015E04022D243914211DC4922D2439142F7
:105A300002DB7908CF190AE05322D2439142EEDA11
:105A40005D22D243914201DBBF0000E0FF000A97D4
:105A50001396269E597E00290BD0002132460F4610
:105A6000D170917051701170121D7F1C5C7EA74225
:105A7000F6D30C9311952599149122990D911590B7
:105A800041088C4211D2FD4A2346A0008458345468
:105A9000270A451C7755250C871CF555240EC01C7C
:105AA00034545B1C9CB2A142EFD823981090012083
:105AB0000990009030463146149A159F3B4605F0F8
:105AC00041FE0D9800060890400E139D00D186E01F
:105AD00068000490002F3FD0002210461146144663
:105AE00006E01C461146159F401C82B2BA420ED2F7
:105AF00083B2AB42F8D09200149B9A5E0FB2BA42C6
:105B0000034600DC2346BA42EBDC0A46E9E7002FF5
:105B100025D0002210461146129206E0129311463B
:105B2000159F401C82B2BA4214D283B2AB42F8D065
:105B3000A5B2AB420CD09200149B9A5E0FB2BA424F
:105B4000034600DC129BBA42139DE7DC0A46E5E7F8
:105B5000139DE6E7129903E00024214600E00021AE
:105B6000129110980183C4828582049FF057FAF73E
:105B700090FE7921C9050E91FAF720FC1099C861B1
:105B800009980743F057FAF784FE0E99FAF716FCC6
:105B9000109F38622004C40B3057FAF77AFE0E9932
:105BA000FAF70CFC7862601C3056FAF772FE0E9C15
:105BB0002146FAF703FCB86212980004C70BF057AD
:105BC000FAF767FE2146FAF7F9FB109CE062781CB1
:105BD0003056FAF75EFE0E99FAF7F0FB2063119843
:105BE00005800C98407E410000278D4228463A46A9
:105BF000149E1ED30A9880B28AB29300F45E844247
:105C00000BDA491C8AB2AA42F6D9002728463A463E
:105C100081B2691A012910D01BE0F018119B19807C
:105C2000078808040FD0500040008019001F028828
:105C3000084681B2691A01290BD1A80030181199C0
:105C40000D80078826E00020024681B2691A0129EA
:105C5000F3D00A9989B2079B4B43BB421AD30699EA
:105C60008A4217D80599002914D0401C82B289189D
:105C700003E0401C82B291420CD983B2AB42F8D807
:105C80009200B35EBCB2A342F3DDB218119B188040
:105C90001788EEE712970B980580119800882B1A49
:105CA000002B16DD02210F9A1143032942D10E93D6
:105CB000411C421E10B281420EDA0E98032824DBEA
:105CC0000C98808C012820D019A818A9FFF736FD60
:105CD0001FE0002018902BE00026F443374608E030
:105CE000B8B2400019AD2B527F1C521C10B2814239
:105CF000E3DB13B2A3423346F2DD159B98423346F1
:105D0000EEDA8000149B1B5AEAE719A818A9FFF7DE
:105D1000E1FD149E139D0F9A012A13D0032A11D07E
:105D2000022A04D111980088281A02280ADA0020D1
:105D3000179034E0022A01D1022BB8DA0020189023
:105D4000012AEBD1681C691E0FB2B84208DA0C9820
:105D5000808C01281DD119A817A9FFF7BBFD1CE0F5
:105D60000022D343144608E0A5B26D0019AF7E535C
:105D7000641C491C0FB2B842E9DB0DB29D421646C5
:105D8000F2DD159DAF421646EEDABD00149E765B3D
:105D9000EAE719A817A9FFF7D1FC149E139D249FC9
:105DA000189C17992046FAF701FB0F99012900D892
:105DB000204638600D98002800D1CBE01199088862
:105DC000109FB8860888281AB880129880B2FAF70F
:105DD0006BFD7921CC052146FAF7F0FA2146FAF756
:105DE000EDFAB863119F3888002849D081008919DD
:105DF000091F0988129C0C191599884203D280004A
:105E000080198088041915984300534916AA304612
:105E100005F076FE169810994864FAF774FDA4B25E
:105E2000A04201D14D480FE0001BFAF73DFD1C9048
:105E30001CA81BA9012205F0E1FE2046FAF734FD5B
:105E400001461B98FAF7BAFA109908603988491B7D
:105E50004A1C92B2032A02D20021159F17E009B210
:105E60000229159F12DB3F210906FAF7DFFC002803
:105E700002990CD10998810709E0C04640210040F1
:105E80000020129C15998842B9D3BCE73449109878
:105E900001610898800E5DD0002F1CD000221146B1
:105EA000144610464B1B1DB2ED135B196B40139D3E
:105EB0001BB29200B25E53431818A418491C8AB250
:105EC000BA42EFD3FAF7F0FC06462046FAF7ECFCAC
:105ED000002C03D100E000260398C0051C901CA8EC
:105EE0001BA901252A4605F089FE1B9C2046314648
:105EF000FAF764FA014610988160002F119422D0BD
:105F000000242746264613951291B8B2FAF7CCFC26
:105F10001299FAF74BFA0546A0001499085EFAF7B1
:105F2000B8FC01461398C00785432846FAF746FA9D
:105F300001463046FAF7E9F906467F1CBCB21598CF
:105F40008442E2D300E0002611983146FAF736FA8F
:105F50001099C8601DB0F0BD54A601020000204198
:105F600000004040F0B58FB00692F74A09AF70CA02
:105F700070C770CA70C70328079320D88800F3A1A0
:105F80000858F649FAF7C1F90446F549FAF7BDF998
:105F90000D90F4492046FAF7B8F90C90F2492046E2
:105FA000FAF7B3F90B90F1492046FAF7AEF90A90E7
:105FB000EF492046FAF7A9F90990EE4969E004286B
:105FC00022D0062820D88800EBA10858EE49FAF71D
:105FD0009CF90446ED49FAF798F90D90EC492046F2
:105FE000FAF793F90C90EB492046FAF78EF90B90EB
:105FF000E9492046FAF789F90A90E8492046FAF774
:1060000084F90990FD4944E00838022821D8880025
:10601000FBA10858D149FAF778F90446FC49FAF788
:1060200074F90D90FB492046FAF76FF90C90FF20A8
:1060300081052046FAF769F90B90F7492046FAF7EF
:1060400064F90A90CA492046FAF75FF90990FE49B7
:106050001FE08800F1A10858F449FAF756F9044600
:10606000F349FAF752F90D90F2492046FAF74DF943
:106070000C90F1492046FAF748F90B90EF49204679
:10608000FAF743F90A90EE492046FAF73EF90990EB
:10609000EC4900942046FAF738F9EC4909680E906B
:1060A000EB480468EB4801684808EB4F05463D4063
:1060B0000022002D08922DD0CA01120E07D0280C04
:1060C000E90D12D14000E649085AE6490AE0C90341
:1060D000090E0CD0280AE90B10D14000E049085AFB
:1060E0008F2189004018E4300DE0DC490AE081B2DC
:1060F0007F2905D84800DA49085A04E0D94901E067
:106100008F218900401800B2FAF7C3FBD649FAF78D
:1061100055F902460292039507252606D34B1A68C5
:10612000002A089840D0791C8A420BD21102090E2D
:1061300013D0110C1F46D00D1FD14800C849085A72
:10614000C84907E01F46110E002A13D44800C4496D
:10615000085AC2494018E4301FE011041F46090ED6
:106160000ED0110AD00B12D14800BD49085A8F2118
:106170008900EFE7BE4808180FE0B84808180CE09F
:1061800091B27F2906D84800B549085A05E0B548BC
:10619000081802E08F218900501800B2FAF779FB45
:1061A000B149FAF70BF93B460590159F2C40F50EC7
:1061B0005B69B0491940089810D0DA02D20E34D089
:1061C000C80B3E210140A648405AA6494018E43079
:1061D00000B2FAF75EFBA449FAF7F0F80490149EB7
:1061E0006800A5A1085EFAF754FB0146A00009AAC1
:1061F0001058FAF78AF80146B8B20128089F0191B1
:1062000002D1022C0AD9A74F052C24D11898089046
:106210000C2D20D80B2D16D3A44918E00027022CF2
:10622000089718D08120C70515E01A04120E00D176
:10623000CAE0080AC90B00D0CDE040008849085ADE
:106240008F218900C2E7092D00D2C7E0964908983E
:10625000FAF75BF8089001200021B542034600D30D
:106260000B46052C00D308461799169A1A9C199DBF
:106270001843069B012B12D1079B402B22D10028EB
:1062800040D03846FAF741F801460198FAF73DF850
:1062900001460098FAF78AF8059A04998AE0079B64
:1062A000402B1FD1002838D03846FAF72EF8014687
:1062B0000198FAF72AF801460098FAF777F8059A54
:1062C000049977E0002833D03846FAF71EF80146E3
:1062D0000198FAF71AF801460098FAF767F8059A54
:1062E000049967E000285BD03846FAF70EF80146BB
:1062F0000198FAF70AF801460098FAF757F8059A54
:10630000049957E002981146FAF750F803990029CA
:1063100000D16748059A04994CE002981146FAF7B3
:1063200045F80399002900D16148059A049941E094
:1063300002981146FAF73AF80399002900D15C480F
:10634000059A049936E0C0467C1A0100000068C135
:10635000000088C166665EC1000084C100008441FF
:106360000000B44100004841000020400000F0C09F
:10637000000084C10000F841333323C1000050C144
:106380009A9929C19A9949C19A9949413333CB4184
:1063900066667641CDCCAC40333393C09A9949C1FF
:1063A00002981146FAF702F80399002900D14048F3
:1063B000059A049928601046F9F7F8FF0899F9F74B
:1063C000F5FF20600FB0F0BD99B27F2911D84800C9
:1063D0002349085AFCE623494018F9E6C120010682
:1063E0000898F9F792FF0890062D00D933E70020AE
:1063F00030E78F2189005818EAE6C0463333F3416D
:10640000000058C19A9961C19A9969C1000084C17C
:106410000000AC4100003841000008C1CDCC80C173
:10642000CDCC88C133338FC1333397C133339741D8
:10643000CDCC8C413333F3409A9919C0666646C17E
:10644000333397C1CDCCB4410000D4410C0000409F
:106450005030004068400040FFFFFF007C08000013
:10646000841E01005C050000919AF63C6420004007
:106470009C0B0000FFFF1F00FAFFFCFFFEFF000067
:1064800002000400060008000A000C000E001000C4
:1064900012001400160018001A001C001E00200034
:1064A00022002400000080BF0000A0C0000040C007
:1064B0000000DCC2F0B5FFB0ECB017460E460D9000
:1064C0000021E991E891DC919991989197919691A9
:1064D0001491139112919AA8F49DF39CF29A002EB4
:1064E00000D1E6E10B938030F09B11800995296083
:1064F0002546DBAC218095AC21800C952980DA9172
:106500007F24E405B994B894B794B694B594B49440
:10651000B394B294B194B094AF94AE94AD94AC945F
:10652000AB94AA94A994A894A794A694A594A4948F
:10653000A394A294A194A0949F949E949D949C94BF
:106540009B949A94046644668466C46604674467B0
:106550008467C467046444648464C46404654465F3
:106560008465C465046244628462C46204634463F3
:106570008463C463046044608460C46004614461F3
:106580008461C461B0090B250B2800D3AE011095BE
:10659000012B0B9D00D070E12B89012B00D06CE109
:1065A000298C00290E9200D18BE16B8C002B00D13D
:1065B000FAE1AA8C3021695C002900D188E10892B7
:1065C000109F5F431196304639460F93F9F782FDCD
:1065D0000590FAF75EF901462046F9F72CFF832172
:1065E000C905F9F7EBFE064696A8021D11988742E9
:1065F0000A9200D879E155A811909AA9069196AF10
:1066000015463A46059C234605F06CFA15A80F90EE
:1066100006992A46234605F065FA02230D9338466B
:1066200031463A4605F0AAFA012308930093E8AAF6
:1066300010923846394605F077F8E898DD901198C1
:10664000069D29463A46234605F04CFA0F982946FE
:106650000A9A234605F046FA384631463A460D9BDB
:1066600005F08CFA089B009338463946109A05F0DD
:106670005BF8E898DE9011982C4629463A46059D2D
:106680002B4605F02FFA0F9821460A9A2C462B46E6
:1066900005F028FA384631463A460D9B05F06EFA69
:1066A000089B009338463946109A05F03DF8E89863
:1066B000DF901198069D29463A46234605F012FAC6
:1066C0000F9829460A9A2346254605F00BFA3846C4
:1066D00031463A460D9B05F051FA089B0093384627
:1066E0003946109A05F020F8E898E0901198069C39
:1066F00021463A462B4605F0F5F90F9821460A9AAD
:106700002C462B4605F0EEF9384631463A460D9BAD
:1067100005F034FA089B009338463946109A05F084
:1067200003F8E898E1901198069D29463A462346D9
:1067300005F0D8F90F9829460A9A2346254605F010
:10674000D1F9384631463A460D9B05F017FA089BB9
:10675000009338463946109A04F0E6FFE898E29034
:106760001198069C21463A462B4605F0BBF90F9836
:1067700021460A9A2B4605F0B5F9384631463A4685
:106780000D9B05F0FBF9089B009338463946109A9B
:1067900004F0CAFFE898E390119821463A462B4648
:1067A00005F0A0F90F9821460A9A2B462C4605F0D1
:1067B00099F9384631463A460D9B05F0DFF9089BBA
:1067C000009338463946109A04F0AEFFE898E490FA
:1067D0001198069D29463A46234605F083F90F98FD
:1067E00029460A9A2546234605F07CF93846314663
:1067F0003A460D9B05F0C2F9089B0093384639468E
:10680000109A04F091FFE898E5901198069C2146B3
:106810003A462B4605F066F90F9821460A9A2B4610
:1068200005F060F9384631463A460D9B05F0A6F969
:10683000089B009338463946109A04F075FFE89893
:10684000E690119821463A462B4605F04BF90F98F1
:1068500021460A9A2B4605F045F9384631463A4614
:106860000D9B05F08BF9089B009338463946109A2A
:1068700004F05AFFE898E7907AE010880C9A1080AC
:1068800099919891DA9E08460F46099DF59CF9F773
:106890008DFD2860DC9827606060A6600C34DDA860
:1068A0000EC80EC42EC82EC42EC82EC47FB06CB025
:1068B000F0BDFF2010800021296020807FB06CB0E7
:1068C000F0BD002201233021695C002900D076E66A
:1068D000DDAA1ACF1AC23ACF3AC23ACF3AC20B2136
:1068E0003046F9F7F7FB054642E000200690059D8B
:1068F0000796089F1190069801460D9C0F9A4A43EF
:10690000D219109B5A43119BD218D200A358890068
:106910002E4655AD6B503546121DA25815AB5A5038
:10692000401C01B28E42E9DC55A89AAE96AC3146C5
:1069300022462B4605F0D6F815A831460A9A2B4672
:1069400005F0D0F8022320460799224605F016F9F3
:1069500001230093E8AA2046214604F0E5FE119B9E
:106960009800DDA9E89A0A505B1C0B2B1846C1D190
:10697000F19EDDA89AA9DCAA0B2305F0B3F8092142
:106980000E980F9101800B98C168DC9C2046F9F7A6
:1069900015FD0146A8B2E69F0F281BD808280DD385
:1069A0000846F9F7B2FC14E0FF2010800021099A94
:1069B00011600C9908807FB06CB0F0BD042803D33F
:1069C00081220846D10502E0412208461106F9F766
:1069D000F5FC01462B20C04386420D9704DB084698
:1069E000F9F793FC014603E04020C043864244DDB2
:1069F0000E9A0C9C0B98408A002811D00B98038AA1
:106A000095A80390DBA80290DAA801900094DDA875
:106A10000D4603F0CBF829462488DA9E099D68E0EC
:106A200011910F98208000273D46109705E00E98A1
:106A300004887F1CB8B2A04211D8B8B28000DDA98A
:106A40000C5820461199F9F7D5FE0028EFD1002DFA
:106A5000EDD10C98078001250F971094E7E7DBA88C
:106A600005800F9A90B2201A012811D10C98048049
:106A70000D9FDA973E46099D3AE04920C043864281
:106A800000DA8BE0FF2208469105F9F797FCA9E7A9
:106A900010200B990E5E012E00DA90E0551CABB26F
:106AA0001846A1B2AAB28A4217D805E00E990C88FE
:106AB000A1B2AAB28A4210D88000DDA90C582046A3
:106AC00010991F46F9F788FE3B46002805D10C981F
:106AD00005800B98068A0F95109430B2C1186D1C72
:106AE000A8B28142E2DC109EDA960F9C099D0D9FB0
:106AF00011993046F9F79FFCF9F7ECFE052800D311
:106B0000052095A90880A0B20E990988814218D95C
:106B1000401C611E0CB2A04218DA12A898A9FEF718
:106B20006DFE0E980188481C491E0CB2A04221DA65
:106B300012A899A9FEF762FE99999898099D0D9F50
:106B4000A4E600219891999108469FE600221346F9
:106B500008E09CB2A40012AF3D515B1C491C0CB272
:106B6000A042DADB8DB20A2D1546F2D8A400DDADC5
:106B70002D59EEE70022134608E09CB2A40012AFA4
:106B80003D515B1C491C0CB2A042D1DB8DB20A2DD9
:106B90001546F2D8A400DDAD2D59EEE75320C043D1
:106BA000864200DB1BE70E460B9881692046F9F709
:106BB00013FE00280C9C08D10B98808B07E014462C
:106BC000099D0D9F1199109E93E70B98C08BF9F7C3
:106BD0006BFE01463046F9F7F1FB119021E700000A
:106BE000F0B58BB01C4609930E46034600200A9070
:106BF00040480088224F05970AA904910394029205
:106C0000109C0194012500950B21414389B230333A
:106C10001C4A3046FFF74EFC3868079078680890A9
:106C2000B868069033480088334F00950194029766
:106C3000324E30363249334A3346FEF76BFB069804
:106C4000F8620798386308987863099800882E4995
:106C500005912E4904912E490391029701900096C7
:106C60002C4B284629462A46FEF74CFC43200106B9
:106C70000A98F9F7A3FBF9F72DFE0BB0F0BDC0465B
:106C80001CA6010214DE0102F0B589B00F9F0E9C14
:106C9000002815D01098079016480088164E012538
:106CA0000095019102960893144B30331449154A0C
:106CB000FEF730FB089BF76207983063746303E0CC
:106CC0000D484763C462002518880F4905910F4994
:106CD00004910F490391084902910190074830300F
:106CE000009001210B4B28460A46FEF70BFC09B029
:106CF000F0BDC046C8AC0102D8D20102849F010297
:106D0000D49E01024CD101024CA30102C0AC01028D
:106D10005CAC010264AC0102304870470048704727
:106D200008AD0102800037490918C86B0022CA6308
:106D30007047C046800033490918886C00228A6475
:106D40007047C04680B52F4AD369002B01D0126A24
:106D50009847002080BDC0460249087800220A708A
:106D60007047C04678C801020020704780B51829D6
:106D700005D803468A1E03481946F9F7D5F90020BD
:106D800080BDC046CCAC0102B0B50246002002294D
:106D900001D2C043B0BD8C1E0F2C07D8044D28462D
:106DA00011462246F9F7C0F900202855B0BDC0466B
:106DB000E8AC0102B0B502460020022901D2C0436E
:106DC000B0BD8C1E0F2C07D8044D28461146224614
:106DD000F9F7AAF900202855B0BDC046F8AC010269
:106DE0000849087800220A707047C046B0B50446CA
:106DF000044DAA68002A02D0E968204690472C6119
:106E00000020B0BD1097010280B5054842680020FF
:106E100001460AF035F80349C8710120887180BD28
:106E2000389001026897010270B5421E0F2A23D8DC
:106E3000082808D801209040934A137F00290BD0DE
:106E4000034313770DE00938012282408E48437FC7
:106E5000002904D0134303E08343137701E09343F5
:106E60004377894E747F357F402002212A4623468E
:106E7000FDF7ECFD7477357770BDC046F0B587B08F
:106E8000814C2146263105914878BF2606404E7038
:106E900026200690275C40250621039128463A4685
:106EA0003346FDF7D3FD0698275405984670667F54
:106EB000284604952E436677257F022102912A46B3
:106EC0003346FDF7C3FD0699605CEF270740675422
:106ED00066772577059D6E78049803993A46334680
:106EE000FDF7B4FD069827546E70207F10260643E8
:106EF0002677637F0093049F384602993246FDF758
:106F0000A5FD0698255CFE2101910D4025540098B1
:106F100060772677059E7378384603992A461F4680
:106F2000FDF794FD069825547770267F0120009088
:106F300006432677657F0498029932462B46FDF773
:106F400085FD0699605C202707436754657726779F
:106F5000059846780498039D29463A463346FDF73E
:106F600075FD0698275401980640059846700498C8
:106F700029463A463346FDF769FD06982754059899
:106F80004670667F009806436677227F0092049DD4
:106F9000284602993346FDF759FD0698275C7F2164
:106FA00001910F402754667700982077059E7378EB
:106FB000284603993A461D46FDF748FD0698275492
:106FC0007570207F802606432677637F0093049D9B
:106FD000284602993246FDF739FD0699675C2F4332
:106FE000675400996177267705994B780093284676
:106FF000039D29463A46FDF729FD06982754F726B2
:107000000098064005984670049829463A4633464B
:10701000FDF71CFD06982754059F7E70607F0825AC
:1070200005436577267F0498029932462B46FDF783
:107030000DFD657726770198C0437A780192104359
:107040007870069EA75DC3B2049D284603993A4610
:10705000FDF7FCFCA7556F20C64301980643059831
:107060004670F3B2284603993A46FDF7EFFC0698BE
:107070002754059846703034002128462246029B4A
:10708000FDF752FC07B0F0BDD495010280B50A4669
:1070900000210223FDF748FC80BD000080B51248A6
:1070A00001681F220A40026003200840022812D112
:1070B0000E480268D30D02D0FF231B06D2180C4BDA
:1070C0001A600C4A12680C4B1A6080680B4A1080D8
:1070D000000C0B4A10801A488268002A02D082688D
:1070E0000020904780BDC0467420004064400040AE
:1070F00060D101027830004064D10102EA9F0102B0
:10710000CED2010280B50D48016889070FD505214F
:1071100001600B48C178002908D00021C170C16806
:10712000002903D0C26841680020904780BD05480F
:1071300005A10B4A0BA307F03DFCC0462C04004000
:1071400028940102843701005048595F54494D4545
:10715000525F49525148616E646C657200000000D4
:107160008D0A0000556E65787065637465642069EA
:107170006E746572727570740000000070B504461C
:10718000401E012814D80320084011D13F2040039D
:107190000818050B281980280AD8164E31780120C6
:1071A0004840294603F05CFC641E6D1C002CF5D1A0
:1071B00070BDC04680B50020014603F099F9002853
:1071C00000D080BD0B480121017080BD70B516460E
:1071D0000C460546FF22F8F7B9FF05483118054867
:1071E0000278012050402A46234603F0E1FA70BDA0
:1071F00000E0070454A801020120000370470120A9
:1072000040037047F0B585B04A484B49016005F02E
:1072100019FB4A4DEA8A4A2149484252AC8A482120
:1072200044520021E983AB88C362AE7A0672AE890C
:10723000C68104824282AA8D028704938386EE8EE1
:1072400001241D2E264600D80E463E490E70511EC2
:107250008A415100C161210269803221695C417219
:10726000288B394908806C8C0F20224602407D21F2
:10727000C900260B4E43B6182205170F6422574348
:10728000F6192406270F0A246743F6192F4F3E806C
:10729000AE8C374607402B46350B4D43ED1937056D
:1072A0003F0F5743ED193606360F6643AD19284E8A
:1072B0003580DD8C2E4606402F0B4F43BE192F051F
:1072C0003F0F5743F6192D062D0F65437519214FB2
:1072D0003D801D8D28402E0B4E4330182905090F87
:1072E000514340182906090F614340181A4E308057
:1072F00003241AA220462146049B08F0B7FB0F483E
:107300004088C1B20091030A18A22046214608F025
:10731000ADFB0E4803880E480088398832880A4D34
:107320002D8800AE27C61AA22046214608F09EFBF3
:1073300005B0F0BD28960102D184000056A80102D4
:107340006099010274960102569601024E9601025E
:10735000509601025296010254960102C9E8B1B852
:1073600049443A202578202E0D0A0000B9CCBCFEF5
:10737000B0E6B1BE3A34472D475053B6A8CEBBCA8B
:10738000D6BBB7205625642E25642E200D0A00009A
:10739000B7FECEF1C6F7B5D8D6B73A2025642E256C
:1073A000642E25642E25643A25642E0D0A00000003
:1073B000F0B583B030480068C16B0901890F01D076
:1073C00003B0F0BDC16BC06B2C4D05404800400FB1
:1073D0000826029686400227384602F0E3F801901C
:1073E0007043C10B4A1B26485043F8F789FE0446F8
:1073F00007F022FA032123A238461F4F00912346AB
:1074000008F034FBF88A002817D00198400129467B
:10741000F8F760FE46431822324001200F2A014649
:1074200000D8002173095B181B4CA3420DD8194DDD
:10743000ED1A6D050F2A0CD80CE038680021C160E8
:10744000112002F09FF803B0F0BD5D1C6D050F2AFE
:1074500000D956422A0C029D2E4009018919A342E7
:1074600002D80098000400E0400408188018396829
:10747000086303B0F0BDC046B8940102FFFF1F00CF
:1074800040420F0052434F33324B2070706D202525
:10749000640D0A00FF070000FE7F000070B52E4952
:1074A000486017222D4B1EE01D68A5431D6000BFDC
:1074B00000BF00BF00BF00BF00BF00BF00BF00BFD4
:1074C00000BF00BF00BF00BF00BF00BF00BF00BFC4
:1074D00000BF00BF00BF00BF00BF00BF00BF00BFB4
:1074E000521E541C36D20446D440012525400D704E
:1074F0001E68802426431E6000BF00BF00BF00BF7F
:1075000000BF00BF00BF00BF002DCDD000BF00BF37
:1075100000BF00BF00BF00BF00BF00BF00BF00BF73
:1075200000BF00BF00BF00BF00BF00BF00BF00BF63
:1075300000BF00BF00BF00BF00BF00BF00BF00BF53
:1075400000BF00BF00BF00BF00BF00BF1D68A54354
:107550001D60B3E770BDC0461096010204200050C4
:10756000B0B582B0154908688269D2070CD00122F3
:10757000C2610D69002D07D000686C46214606F0F7
:1075800049FF00212046A84702B0B0BDB0B582B087
:107590000A490868026C92070ED5026C0123134356
:1075A0000364CD68002D07D000686C46214606F0C4
:1075B00031FF00212046A84702B0B0BDB8940102B7
:1075C00006480168032291430160016801220A43D1
:1075D000026000F035FB07F051F9C046280000407A
:1075E00080B50D490868002810D522480268042398
:1075F000032A01D01A4300E01A460A601E490A68AD
:10760000002A02D041680020904780BD03A00CA151
:107610009E2211A307F0CEF92C100140696E636C15
:107620007564652F647269766572732F6D6B5F7315
:107630006C6565705F74696D65722E630000000093
:10764000534C4545505F54494D45525F495251484E
:10765000616E646C65720000556E65787065637468
:10766000656420736C65657020696E7465727275EF
:10767000707400000C900102D4D20102B0B582B047
:1076800004460078002811D0094D01A90870286827
:10769000416A0029FCD101A901220020034608F01B
:1076A0006BFF611C607800280C46EED102B0B0BDC3
:1076B000F0940102F0B581B01C4615460E4607460F
:1076C000EFF3108072B6072003F0A0FFE120000165
:1076D00000BF401EFCD13846FFF7E0FE3046FFF702
:1076E000DDFE2846FFF7DAFE2046FFF7D7FE62B63A
:1076F00001B0F0BD10B5DC4C216806290FD801207F
:1077000002468A4058210A4209D020600020A06029
:107710002369002B03D06269002002219847D148D9
:107720002258062A12D801210B46934058221342B0
:107730000CD021502018002181600369002B05D056
:10774000AD20C0002258012002219847D948225874
:10775000062A11D801210B469340582213420BD020
:1077600021502018002181600369002B04D00348B8
:107770002258022001469847002010BDBC0A000094
:10778000F0B581B00024022803D9E443204601B0BB
:10779000F0BD17460B46094E464309488519284651
:1077A00018302A2107A2FCF797FB42202F52032012
:1077B00003498851204601B0F0BDC0465405000081
:1077C00088AD010225730000F0B585B0DD4D2C6851
:1077D000002C0CD0DA4FDB4CE659002E0CD0B54F04
:1077E000E659002E0DD00020C04305B0F0BD01AC1D
:1077F0000FC400272E4608E001AE0FC6E619012788
:1078000003E001AE0FC6E6190227CD4C30462146F3
:10781000FCF748FA022030607C432919029D4D6034
:10782000CF60039808610498486108464430CC3121
:107830000122560210233246FCF72AFCE1480019C7
:10784000B32189004118012D05D1B83001233246FA
:10785000FCF709F804E0743010233246FCF718FCFA
:1078600001980760002005B0F0BDC0460146002029
:10787000022901D9C0437047E04A4A43E049885091
:107880007047C046022806D8E4494143E4484018FE
:107890000249401870474B2080007047D404000014
:1078A000022802D94B2080007047DC494143DC4864
:1078B00040184D21090140587047C046032801DB9C
:1078C00003487047D5494143D548401818307047A0
:1078D00091350100022806DCD0494143D0484018C8
:1078E0004221405A704700207047C046032801DB00
:1078F00000207047C9494143C94840184430704787
:10790000022804DCC5494143C5484058704700205F
:107910007047C046022805DCC0494143C0484018B2
:107920004068704700207047B0B50024E14302284A
:107930000FD8BA4A4243BA4B9D58042D09D0991822
:1079400001220A600B69002B05D04A690221984781
:1079500021460846B0BD2046B0BDC04610B5002443
:10796000022801D9E04310BDAC494143AC4A07238A
:10797000535051180B69002B03D04A69002421464B
:107980009847204610BDC04610B50024022801D9F2
:10799000E04310BDA1494143A14A06235350511869
:1079A0000B69002B02D04A6901219847204610BD7F
:1079B00010B50024022801D9E04310BD9749414386
:1079C000974A51180B69002B02D04A690321984746
:1079D000204610BDF0B583B017460024E2430228CC
:1079E0001AD8002B18D00D468C4941438C484618B4
:1079F00070680128029312D1002F0AD0B8360024F3
:107A000029193046FBF737FF002825D1641CA7420F
:107A1000F6D1029807600022104603B0F0BD019233
:107A200074363046FCF7EFFA002811D0034642685E
:107A3000BA4209D2196828461D46F8F775FB2B464D
:107A4000686802990860019430461946FCF7B1FA5B
:107A5000019A104603B0F0BD02980460002210465F
:107A600003B0F0BD5405000088AD01026C48016808
:107A7000062909D06949415806290BD00D494158BA
:107A800006290ED0002070470121816063494158CA
:107A90000629F3D1064901224250064941580629D8
:107AA000F0D1AB2109010122425000207047C046AD
:107AB0005C050000A80A0000F0B581B00446002073
:107AC000C343022C02D9184601B0F0BD15460E463C
:107AD0001B4A62431B498F187968012910D1002D78
:107AE00028D01C460090B83738463146FBF79CFE3C
:107AF000002821D1761C6D1EF6D1009801B0F0BD92
:107B00000090743738462946FCF798FA00280CD0C4
:107B10000446006831462A46F8F706FB38462146F7
:107B2000FCF75CFA009801B0F0BD07A02146FBF716
:107B300039FF009801B0F0BD204601B0F0BDC0464D
:107B40005405000088AD0102536F636B65745B25BB
:107B5000755D2052656376204275666665722046C3
:107B6000756C6C0D0A000000F0B583B01546074631
:107B70000022D043022F19D8002D17D000AB07C325
:107B80000F4878430F490E18443630462946FCF713
:107B900055FA00280CD00446006801992A46F8F7E7
:107BA000C3FA30462146FCF719FA029803B0F0BD3B
:107BB00005A03946FBF7F6FE009803B0F0BDC046BD
:107BC0005405000088AD0102736F636B65745B251B
:107BD000645D2073656E64206275662066756C6CEA
:107BE0000D0A000002460020022A04DC0B4B53431E
:107BF0000B4AD1507047C0437047C046540500003F
:107C000088AD0102022801D9002070470349414391
:107C100003484018034940587047C04654050000C7
:107C200088AD0102CC04000080B504480168491CFD
:107C300001600069002800D0804780BD40DE01025D
:107C40000148024901607047809001020026B80394
:107C500010B59F480024846114300221024A234653
:107C6000FFF7B2FD204610BD657D000070B5B6B0CF
:107C7000FCF7E4FF012814D1FBF7C2FF2C4DA969E2
:107C8000022914D0002909D12978002939D0E969BD
:107C9000411A062902D300212970E861002036B07C
:107CA00070BD234800218161002036B070BD296A73
:107CB000421A20493B2A02D80A78002AEED02862CC
:107CC00000220A701C4908880A801C4B19881A80F7
:107CD000F8F700FA1A4908801A4880881A49097882
:107CE0000090019104ACC821184A194B204609F0B4
:107CF0004FF9024668692146FFF736FF002036B08B
:107D000070BD0126AE616B88A888E9882A8900AC1D
:107D100007C4B1020F4C10A22046FCF7DDF86869D9
:107D20006A892146FFF72CFD2E70002036B070BD09
:107D30004C96010238930102789601027696010270
:107D4000E89F010256A801026C990102C02C0100B3
:107D50003C9A010274C4010225752E25752E2575E5
:107D60002E257500F0B5C1B0032909D879440979E9
:107D700049008F4401070F155548816901290AD030
:107D800041B0F0BD524881690129F9D102218161D8
:107D900041B0F0BD4E4800218161017041B0F0BD9D
:107DA000002702974A4E70694A494B4A02ABFFF7D7
:107DB00011FE0028E4D1032048A2014607F056FE38
:107DC000444849A10922F8F7E4F9002840D0414885
:107DD00048A10A22F8F7DDF90028D1D13D482C212D
:107DE00035AA0C23FCF789F83698FBF75FFFB081C2
:107DF00080B2434989888142C2D13798FCF79FF805
:107E0000F0813898FCF79BF83082B389F0890090B4
:107E100003A8C8213BA209F0BBF80446308A002819
:107E20000FD03DA5F0893818400035490A5A03A8FB
:107E30000019294609F0C8F804197F1C308A8742C6
:107E4000F0D3706903A92246FFF78EFE41B0F0BD62
:107E500003A8C82131A21F4D2B4609F099F804460A
:107E60002C2135AA0C232846FCF747F83698FBF757
:107E70001DFFB08180B2224DA988814200D07FE7EA
:107E80003798FCF75CF8F08180B200280ED03028DB
:107E90000CD032280AD0706903A92246FFF764FE8D
:107EA0003898FCF74CF8F189490068521F490020C6
:107EB00008701F4908701F4A01211170EA8E1D2A9F
:107EC00000D801461C48017006F054FC41B0F0BDDA
:107ED0004C96010274C40102FF030000CAD5B5BD6F
:107EE000CAFDBEDD0D0A0000247365747061726105
:107EF0002C0000002472656164706172612C0000C6
:107F000056A80102247265706C79706172612C252B
:107F10003034782C256400002C25640024736574AB
:107F2000706172616F6B2C25730D0A00C2AC010287
:107F3000C4AC0102209401027496010280B582B0A3
:107F40000E4908680022C2600192CA68002A02D065
:107F5000016801A8904702B080BDC04680B582B0DC
:107F6000064908690022C26001220192CA69002AFA
:107F700002D0016801A8904702B080BD10930102B1
:107F800080B5002007F0B0FF80BD80B5012007F06C
:107F9000ABFF80BDF0B581B003F0C0FA164CE060D5
:107FA000A178002901D001B0F0BD21790029FAD1D2
:107FB0000121217100281BD08D02281AA16881425D
:107FC00016D0424E2F46A068305C21698847A068D1
:107FD000401CA060681EA168814201DD0020A060F5
:107FE000E168A068022F03D3691A7F1E8842EAD194
:107FF0000020207101B0F0BD1896010270B5B6B036
:108000001249088800250D80114A11881580F8F75B
:1080100061F8104908801048808810490978104E8E
:108020003278104B1B7800AC0FC404ACC8210EA2F0
:10803000134B204608F0ACFF0246357011484069EA
:108040002146FFF791FD36B070BDC046789601021B
:1080500076960102E89F010256A801026C9901027E
:10806000649901027396010225732C253034782C13
:108070002530327525252C25642C25640D0A000039
:108080003C9A01024C96010270B50E250024284648
:10809000214603F0FBFA0D20214603F0F7FA0124F4
:1080A000204607F029FE04262846314603F0EEFA62
:1080B0000920314603F0EAFA204601F0AFF8A202A7
:1080C0000249034B204608F015F970BD0CCD0102A2
:1080D0002D05010080B5032810D800290ED07C2280
:1080E0004243BF488018C268012A07D12030FBF7FD
:1080F000C2FB002801D00020C04380BD0020C04347
:1081000080BDC046F0B589B00022D543032800D910
:10811000ABE00C46002900D1A7E00095216A0727B3
:10812000534DA9420EDC574DA9421ADD564A9142E1
:108130002FDC4B22D501A9423ED0120291424BD1F5
:10814000042246E04B4A914217DD4B4A91422ADC19
:10815000E1221203914231D0494A91423CD10C2292
:1081600037E04B252E01B14233D06A01914227D02E
:10817000AA01914230D102222BE0E1225502A9420C
:1081800020D09502A9421FD0D202914224D10922C7
:108190001FE04B225202914218D0E122120291427A
:1081A0001AD1062215E0E1225203914210D0334A3F
:1081B000914211D10D220CE003220AE00A2208E0CC
:1081C000012206E0072204E0082202E0052200E086
:1081D0000B22D1002D4A57587C214143804A5050F0
:1081E00056182068B0606068F060A1683161E2688C
:1081F0007261002505950323049303950295019769
:108200000695079501231B020893012807D0002833
:108210000AD18818009A8018B161F06104E03046F4
:1082200020300123FBF71FFB206970636069B06396
:10823000E069B067A069F063706801A907F086FF84
:108240002068012806D830464030234610330ECB34
:10825000FBF71EFF6068012807D1301D70360068EB
:1082600001220B4B314608F045F8284609B0F0BD15
:10827000FFC10100FF0F0E00FF1F1C0080841E00C5
:1082800040420F007F250000FF950000C01A01004A
:1082900045050100B0B50C467C214843504A1518ED
:1082A0002846FBF7FFFC6C600020B0BDF0B583B042
:1082B0000024E743032800D98EE00E46002900D1B0
:1082C0008AE01546002A00D186E07C2141434448DB
:1082D00041188868022832D001283AD000282BD1D2
:1082E000EFF31080C00702D1EFF3108072B6029155
:1082F0000846403001902946FBF7A0FE002863D0D5
:10830000014601980F46FBF769FE386831462A4658
:10831000F7F70AFF0198FBF776FEEFF31081C90724
:1083200003D1EFF3108172B662B602994D6806C8A8
:108330002C4B284608F020F9204603B0F0BD4868D1
:10834000002431462A46234608F016F9204603B099
:10835000F0BDEFF31080C00702D1EFF3108072B6CA
:1083600002910846403001902946FBF767FE00283D
:108370001ED0014601980F46FBF730FE38683146A3
:108380002A46F7F7D1FE0198FBF73DFEEFF3108187
:10839000C90703D1EFF3108172B662B602994D6836
:1083A00006C8104B284608F0E7F8204603B0F0BD99
:1083B000EFF31080C0070FD1EFF3108072B662B6F2
:1083C0003C46204603B0F0BDEFF31080C00703D158
:1083D000EFF3108072B662B63C46204603B0F0BDA3
:1083E00084BD010249080100B0B582B0602833D0D5
:1083F000622843D0642854D101A82F490180EFF3AB
:10840000108072B600242046214602F071F82B4DF0
:10841000002805D1012002030020294601F0C2FFF7
:10842000103501AA02232046294602F099FC62B6C3
:1084300023A0FFF723F964201B490C5206F09AF998
:108440001A4801F0CBF9BFF34F8F19481949016061
:10845000BFF34F8F00BFFDE76020134900220A528F
:1084600006F088F9114801F0B9F9BFF34F8F1048B1
:1084700010490160BFF34F8F00BFFDE762200A493A
:1084800000220A520A8006F075F9084801F0A6F9A0
:10849000BFF34F8F064807490160BFF34F8F00BFFE
:1084A000FDE702B0B0BDC04656A80102A08601009B
:1084B0000CED00E00400FA05AAAA000000D00204B6
:1084C000BDF8C8EBC9FDBCB6C4A3CABD0D0A000007
:1084D000F0B5D1B0A9490A78002A26D0A64EF28B71
:1084E000002A22D1A64DAA68082A00D992E093005A
:1084F00001A4E3589F46C0461D8500001586000074
:1085000015860000258600004F8600005986000071
:1085100063860000338600006D860000552800D079
:10852000BDE00120A86051B0F0BD4978002900D11C
:10853000B9E0934D6A7997498854A979A871E9718E
:10854000521C6A710A2800D0ADE00D2900D0AAE0C3
:1085500003A8019037A800902C4628348D488E49F6
:108560001DAB2246F7F732FEE8608CA105222046BB
:10857000F7F70FFE002837D1864C2046F7F702FEAA
:10858000821E88482146F7F7CFFD1DA8002421460A
:1085900009F0E0F9A861E96137A8214609F0DAF9A4
:1085A00028626962A869E96922462346F8F75AF900
:1085B000002802D17C4800F0F3FC03A8F7F798FEEE
:1085C0002861002810D079480470794804707948EF
:1085D000048079480078002805D0FFF70FFD774820
:1085E000047008F093F92C616A489621F7F7B5FDFD
:1085F0001DA864242146F7F7B0FD37A82146F7F7F8
:10860000ACFD03A82146F7F7A8FD00206871E880BB
:1086100051B0F0BDAA2838D1012A36D10220A86075
:1086200051B0F0BD0421A9600021A970687051B05B
:10863000F0BD2979534A5054481C28716978491F64
:10864000C0B281422FD10820A86051B0F0BD0522F0
:10865000AA60887051B0F0BD0621A960A87051B021
:10866000F0BD0721A960287051B0F0BD6A78062AD4
:1086700002921AD3531F0025424A2C46575DE41933
:10868000A4B26D1C9D42F9DB10E0032807D1022A39
:1086900005D10120E8700320A86051B0F0BD002092
:1086A000A870A860687051B0F0BD00242018029A2C
:1086B000821888781118324FBD7849193C78091909
:1086C000FA78002A00D0C91CC9B2FF2935D1012887
:1086D00009D0022831D11E2D36D1FFF7D5FC01205B
:1086E000F08351B0F0BD284A94710320107190704E
:1086F000AA2050705520107068085071651DD57003
:10870000400031181646D01D2246F7F70DFD301DEA
:10871000E11CEAB2D21C037892B2D218401C491E66
:10872000F9D1A019D143C171090A0172093401209C
:1087300000233146224607F01FFF0020B870B860C2
:108740003871787051B0F0BD70190E4E3146224626
:10875000F7F7EAFC3078012802D12846FFF744FEFB
:1087600006F008F8BFF34F8F084809490160BFF3CE
:108770004F8F00BFFDE7C04656A8010218900102C6
:10878000C0980102A8CC0102D29A01020CED00E0CF
:108790000400FA0510CC01025D2C0100474E47474A
:1087A000410000003C9A0102C1AC01022094010288
:1087B00073960102C2AC0102749601027296010224
:1087C00010B582B008F02AFB154C607A08F022F947
:1087D00014498A88684682800A8849880904891869
:1087E000009104F0E9F8607A052804D002220E49CD
:1087F000092805D003E001220B49092800D0891877
:108800004979207A2246093208F0C8F9607C05F0DF
:10881000E9FB0648064903F07BFB02B010BDC046E9
:1088200038900102941A0100EC9F01027DFC0000C7
:10883000B1E6000080B582B0002001900448C26813
:10884000002A02D001A80021904702B080BDC04696
:1088500080950102F0B583B000242046FEF7AAFC03
:10886000FEF7CDFC274EB060FEF7C6FC7060264FC9
:108870000BE001A8C1888088084319D101A840886D
:1088800024180834B068844235D201AD0821284646
:108890002246FEF79BFC28880028EAD0B8422AD05E
:1088A00001AD0421284600F037FFA9888842E5D0B1
:1088B0003460B06884420CD201AD022128462246C1
:1088C000FEF784FC2888B84203D0A41CB068844218
:1088D000F2D370682118491E4042084030600DD024
:1088E0000024254601202946FEF748FC03CE4D19F9
:1088F000083E8542F6D3346003B0F0BD00243460F6
:1089000003B0F0BD7C960102FFFF0000F0B585B01A
:108910001F4604920646C8170C1844400A2C0391BF
:1089200014D301250A212046F7F7D4FB6D1C632CD4
:108930000446F7D804998D4200D329460A9C002F9B
:1089400009D00398002808D4002207E001250499E3
:108950008D42F2D2F2E7002205E0012204232340F7
:108960009B081343FA1A0223234004980028029418
:1089700012D1002B10D0F468002C62D40398002888
:1089800025D40298400734D57068B5686F1C8742BB
:108990002FD830682B2423E0E407ECD1002A0AD139
:1089A000E9E7376820203855B560F068441CF4606A
:1089B000521E002CDFD49142DDD27768B468651C6A
:1089C000BD42EED9F468521E002CF4D5D3E74042E4
:1089D00003907068B5686F1C87420AD830682D24F0
:1089E0004455B760F068441CF4600025ED43A8428C
:1089F00027DB002B1CD00120029B1840049B18434E
:108A000016D1002A03D113E0521E002C0ED491423D
:108A10000CD27068B3685D1C8542F5D8306830248C
:108A2000C454B560F068441CF460EDE7002C08D431
:108A30000092029801900A2230460399049B00F0AC
:108A400003F805B0F0BD0000F0B587B01F4615462D
:108A50000290012406919142009407D301240698C4
:108A60002946F7F737FB641CA842F9D20D980C9AF7
:108A7000BC42039700D3039400990140002A00915F
:108A800009D00029029C25D12021800705D4084661
:108A9000002F11D004E0029C1CE03020002F0BD0EE
:108AA000084609E023685854A260E168491CE16067
:108AB0003246721E00290DD4039991420AD21646FD
:108AC0006368A1684A1C9A42ECD9E1683246721E7A
:108AD0000029F1D5E068002859D40590012401E06F
:108AE0007F1E6C43022FFBD2069821461646F7F7ED
:108AF000F1FA3246A842F4D2029880680490069FA8
:108B00000195069738462146F7F7E4FA049D691C5B
:108B1000029F7A68914206D9069F059A019D0592A7
:108B2000002A0ED516E01B4A125C3B685A55B96004
:108B3000FA68521CFA600491069F019D0592002A72
:108B400008D460433F1A20462946F7F7C3FAAC42DF
:108B50000446D6D200980028029C059B049D16D09E
:108B6000002E14D0701C01E0002B10D4401E03997D
:108B700081420CD2691C62689142F5D82268202398
:108B80005355A160E268531CE3600D46ECE707B063
:108B9000F0BDC0469C1D0100F0B583B0019002916C
:108BA000002923D00025144F2E460AE01548081846
:108BB000410F4018C0103873761CB0B20299884239
:108BC00014D2019800884B24210100B200F01CF857
:108BD000400061014018F88201B2084881422846ED
:108BE000E9DB07488142E1DD6420E4E7052001215B
:108BF000FEF71AF903B0F0BD60990102E40C000021
:108C0000041000001CF3FFFF074A904201DD054AF3
:108C1000801800B24143C817400D0818C00A00B2BE
:108C20007047C04600F0FFFFFF07000010B5007856
:108C3000012819D1AC480269012A04D1614A13689C
:108C40000124A3431360032905D080214161C26937
:108C5000002A05D107E001214161C269002A02D042
:108C600001898069904710BDFF222E32024803A17E
:108C700007A305F09FFEC046502901006164635FB1
:108C8000646D615F63616C6C6261636B0000000026
:108C9000556E657870656374656420646D612063EA
:108CA00068616E6E656C0D0A00000000F0B58DB055
:108CB0000D460124EFF31081214002D1EFF3108320
:108CC00072B6894E73690F2B06DD102B37D0402BFF
:108CD0002FD0802B2DD005E0002B2AD0012B01D1E5
:108CE00010237361B5813581B061F261002900D133
:108CF00062B63179002929D00294304C05A90A4680
:108D000004950390E8CCE8C2E8CCE8C2029C204677
:108D100000F0D4FD2A4800902A4D2946083120460B
:108D2000039A049B00F03AFE2C60002420460DB00C
:108D3000F0BD0029FAD162B620460DB0F0BD022484
:108D40000029F3D162B620460DB0F0BD317800297C
:108D500007D01C48072181610460002420460DB023
:108D6000F0BD3269B3891749002B15D0B569308938
:108D7000012A02D0002A03D003E09FB2874200D12B
:108D80000C604F68FF07FCD08F6880C55B1E1F0416
:108D9000EED10023B381B561012A02D10A68A24352
:108DA0000A607461F2690024002ABFD0B369318976
:108DB0008800181A904720460DB0F0BDDC1D010058
:108DC0002D8C000008D00140F0B581B0002856D0AD
:108DD0000446424EF068800754D41325284600F01C
:108DE000D9FB284605F008FB27686168012538464D
:108DF0002840CA07920F1018227C1207120E801802
:108E0000627C1207120D8018A27C1207120C8018C7
:108E1000627D13071B0AC018120912068018306001
:108E20007D2006020029304600D12D48E3681A0A49
:108E30007D2A1A4629D22B4EB3422AD200292BD0A2
:108E4000002A2946254E00D01146F7F743F9401E67
:108E500080B2706024480761E27C0270237D037158
:108E6000224F3E686902A468012C1BD02C022643C5
:108E70003E60002B1ED00121184A116329E0012019
:108E800001B0F0BD022001B0F0BD3246154EB34234
:108E9000D4D333460029D3D11A46002A29460F4E8F
:108EA000D2D1D2E73F242401A6437618F0363E60A3
:108EB000002BE0D1002A0CD0FF2212020C4B1C68C0
:108EC00094430122D203A2181A60304A1160304A3A
:108ED000116001214161002001B0F0BD00D00140CE
:108EE0000026B80380841E00989501022C060040DD
:108EF00008E400E070B5002801D0012070BD0C46E8
:108F00001625284600F046FB284605F075FA002C89
:108F100005D01B48183014222146F7F705F92821FF
:108F20001748415C002915D04168002916D4032256
:108F30000B469343144A9C588D07ED0EFF26AE4016
:108F4000B4439C501F220A40012191400F4A1160F6
:108F50000F4A116001210161002070BD8A07D20E05
:108F6000FF2393400F220A40083A03218A43054910
:108F700054589C43545001210161002070BDC046EB
:108F8000849001021CED00E000E400E080E200E0DB
:108F900000E100E05A21014A50527047849F0102CB
:108FA000F0B581B004460078414241412170244827
:108FB0000078C001234909788901014322480078DB
:108FC00040010843214909780901014320480078FC
:108FD000C00008431F4F3978890001431E4D28788F
:108FE000400008431D4E31780143C8B2FBF776FDBF
:108FF0007D20C00000F0F2FB207841424141217009
:109000000F480078C0010F490978890101430E48D3
:109010000078400108430D490978090101430C48D3
:109020000078C0000843397889000143287840005F
:10903000084331780143C8B2FBF750FD01B0F0BDE1
:10904000D29E01027296010221940102D4E601022D
:10905000C1AC0102D39E0102D2D10102C6AC010211
:10906000B0B5764DA8600224002120460A4602F0E1
:10907000E5FA01210522204602F030FBAA6803210F
:10908000204602F053FAB0BD70B55621D448B42240
:1090900042525C2100234352414AC28783873924CC
:1090A00044874049C18683863F4D45863F4D0586AE
:1090B0003325C58583854485C18483847A2444848B
:1090C0000384C3830383C3820382394C4460836077
:1090D000C360836503463E33364C250CDD829C829B
:1090E000160C5E821A826422DA8157229A816722E4
:1090F0005A815E221A81DD809C805E80090C018786
:1091000001853D21490441834182090C818381828B
:1091100070BDC04670B55621B148B42242525C21A0
:10912000002343521E4AC2878387392444871D493E
:10913000C18683861C4D45861C4D05863325C58515
:1091400083854485C18483847A2444840384C383CF
:109150000383C3820382164C44608360C3608365CB
:1091600003463E33134C250CDD829C82160C5E8236
:109170001A826422DA8157229A8167225A815E22FA
:109180001A81DD809C805E80090C018701853D216C
:10919000490441834182090C8183818270BDC046AC
:1091A0006C00630024002F00C7FF0000B7FF000021
:1091B0004C3737376200640070B58A484C21016033
:1091C00001252C02601C00F065F9322000F006FB3E
:1091D00000F04EF9284600F055F9284600F064F8F2
:1091E00000F040F90C4800F055F9002630463146B1
:1091F00000F060FA2846314600F05CFA204600F0A4
:1092000049F9022000F046F94834204605F04AFBAF
:1092100005F0A8FB70BDC0460102000010B5044671
:10922000072106F081FA0548446010BD10B50446D8
:1092300006F07AFA0148446010BDC046409601022B
:1092400070B505200425294602F020FA06242046A0
:10925000294602F01BFA01263046294602F016FA8A
:109260000E20294602F012FA11200025294602F0AC
:109270000DFA2846314602F009FA022128462A460C
:1092800002F02CFA0920214602F000FA0A202146B9
:1092900002F0FCF970BD0000024801680122914310
:1092A000016070475800004002490A68024082424B
:1092B000FBD1704704600040B0B5494D2868810774
:1092C000484C0ED528797F21084022688A4310181F
:1092D000206023680B4002200321434A06F0C6FBAE
:1092E000286880040ED55E20285C7F2108406268D3
:1092F0008A431018606063680B40022003213B4AD8
:1093000006F0B4FB172000F045F939480168022245
:109310000A4301218A4302603648374901603748D1
:109320000021C17181791F2529408171817A427C98
:10933000837C1B029A18C37C1B04D218037D1B0676
:10934000D2182F4B9A4218D1427B837B1B029A186A
:10935000C37B1B04D218037C1B06D218294B9A42EC
:109360000BD1C27A037B491E122906D8190289182B
:10937000254A914201D1202101720178CA0602D109
:109380001022114301701C3C20682021884320607A
:109390001E481F49016041680029FCD503F03AFAD4
:1093A0000446022003211BA2234606F05FFB0A208D
:1093B000C441032C05D8022003211DA206F056FB50
:1093C000FEE71848C1680F229143C1600168164A40
:1093D0000A40026019200001144948600D60B0BDC8
:1093E000EC9F0102480000409829010082290100F9
:1093F000040200400C060040AF6B100A6B000140F5
:109400004D383650312E32360734000000600040AF
:10941000FE1C0080436869702049443A202530389A
:10942000780D0A00C8600040FEFFC3FF0C04004036
:109430004F6C642063686970206D6F64656C20698F
:1094400073206E6F7420737570706F727465642012
:10945000627920746869732053444B2121210D0ADD
:109460000000000080B5172000F08CF8002080BDBF
:1094700010B51724204600F08DF8204604F0BCFFFC
:10948000002010BD0121C907014301480160704758
:109490000060004010B5C1B2000AC2B202290CD06F
:1094A000012913D0002930D1911E7F4802291BD2F7
:1094B0000121032A2AD0490429E07B484168002A77
:1094C0001FD00246203A1143416010BD7648016822
:1094D000D31E022B10D3012A29D0002A41D1012208
:1094E00092079143016010BD002A16D1012149075E
:1094F00002688A43026010BD0123042A1FD05A0467
:109500001EE0012292079143416010BD0904194AEF
:109510007F32C36A13405918C16217498A6992079A
:10952000FCD50121490702680A43026010BD0522EB
:10953000120791430246203A0A43026010BD1A0402
:10954000836A0C4C1C40A21882620B4A131F002431
:109550001C600A4B0A4C1C600D235B0214681C4300
:109560001460054A93695B06FCD505221207114376
:10957000016010BD80FFFCFF1402004004010040A8
:10958000FF0F000001218140474802688A430260C2
:109590007047C04601218140434802680A43026087
:1095A0007047C04610B5052811D8C04678440079E8
:1095B00040008744020E192434393B490A68086880
:1095C000C0003CD53A4820390A425DD03BE000203B
:1095D00010BD35490A680868C00035D534480B46C7
:1095E000203B1A4237D134E02F490A680868C0008E
:1095F00036D52F480B46203B1A424CD135E02A493C
:109600004C680120C0030A680B46203B1C421AD05C
:109610000C68E4003BD5264C1A423CD03AE0224884
:1096200000680120C00310BD1F490A680868C00017
:109630001ED51F480B46203B1A4220D11DE01B4877
:1096400020390A4220D010BD18480B46203B1A4250
:1096500001D10120C00349688900890FC84010BDAD
:1096600012480B46203B1A4215D10120C00312E0DC
:109670000E480B46203B1A4201D10120C003496825
:109680000903890FC84010BD0120C00310BD074C5D
:109690001A4200D020464A689200920FD040496892
:1096A0000901890FC84010BD20000040006CDC0299
:1096B0000026B80304282CD8164AC04678440079FE
:1096C00040008744020A121A210003200007136891
:1096D00083438807800818181AE00320800613685F
:1096E000834388070009181812E0032080041368D8
:1096F00083438807000B18180AE0FF200002136854
:1097000083430802181803E01068FF2398434018A9
:109710001060704724000040B0B5002200290CD032
:10972000074B047895B22D0A65406C001C5B120251
:109730006240491E401C0029F3D190B2B0BDC04622
:109740009C1B0100002841D000BF00BF00BF00BF2C
:1097500000BF00BF00BF00BF00BF00BF00BF00BF11
:1097600000BF00BF00BF00BF00BF00BF00BF00BF01
:1097700000BF00BF00BF00BF00BF00BF00BF00BFF1
:1097800000BF00BF00BF00BF00BF00BF00BF00BFE1
:1097900000BF00BF00BF00BF00BF00BF00BF00BFD1
:1097A00000BF00BF00BF00BF00BF00BF00BF00BFC1
:1097B00000BF00BF00BF00BF00BF00BF00BF00BFB1
:1097C00000BF00BF00BF00BF401EBDD1704780B5C5
:1097D0007D21C9004843FFF7B5FF80BD00280AD0AE
:1097E00030B407252C02CD25641960434009123896
:1097F000001FFDD830BC7047F0B583B01F46164639
:109800000D460146E8680291F6F7D8FD04460F2E92
:1098100011D8082E04D320462146F6F776FD09E03C
:10982000042E02D38120C10501E04120010620461B
:10983000F6F7C4FD04460999089E2B20C0438742D1
:1098400005DB20460F462146F6F75FFD0DE03F2081
:10985000C04387420BDA4920C04387420CDBFF201C
:109860000F4681052046F6F7A9FD39460446688A69
:109870000880346003B0F0BD01915320C04387429B
:1098800006DB20462146F6F740FD0446688A10E0D4
:10989000A8690299F6F7BCFF002801D1A88B00E067
:1098A000E88BF7F701F801462046F6F787FD0446F6
:1098B000002001990880346003B0F0BDF0B581B09C
:1098C00005460120072D66D80C46002963D04A4F73
:1098D00038680169C90736D105263046FFF75AFEB8
:1098E000304604F089FD03CF03690122134303616D
:1098F000002918D403200B4683438E481E5888073E
:10990000C00EFF278740BE43402787403743894822
:109910001F501F200840824087480260874802602D
:10992000354800680FE08A07D20EFF2696400F23C5
:109930000B40083B03218B437D495F58B7434026CA
:1099400096403E435E5069014018012109024218C9
:10995000E369DB069B0CA569ED00EDB2EB185360E3
:1099600062685207520B23685B075B099A18A36869
:109970005B079B0CD218E3685B075B0DD218236969
:109980005B01DBB2D21863699B07DB0ED218802320
:1099900013434350002001B0F0BDC046F0B581B084
:1099A000002A23D005460835134C2668F668EE4099
:1099B000F50702D0022001B0F0BD069D8600A61971
:1099C000B560400124682018009301231D02461948
:1099D00077680724A7437760F16032610099B1602E
:1099E000415919434151002001B0F0BD03A00AA123
:1099F00074220DA304F0DEFFC8920102696E636C4D
:109A00007564652F647269766572732F6D6B5F6420
:109A10006D612E6300000000646D615F7472616EA1
:109A20007366657200000000496E76616C6964209F
:109A30007472616E7366657220647374206164640D
:109A40007200000000015849085840687047C0463D
:109A5000F0B581B005460120012D4CD80C460029F7
:109A600049D0002D03D0012D04D10F2000E00E209D
:109A7000FFF790FDA668012E04D0002E4FD1E0899B
:109A800000284CD12901294843580020D860F50707
:109A9000AD0F27686668B607360F76192569EA079D
:109AA000920EB618022F04D0012F03D101221643C3
:109AB00000E040361D4F9E60E2681A6079188D60A4
:109AC0006269CA604968002917D403220B46934390
:109AD000184A9C588D07ED0EFF26AE40B4438026F1
:109AE000AE4026439E501F220A4001219140124A57
:109AF0001160124A116001B0F0BD8A07D20EFF2436
:109B000094400F230B40083B03218B4308495D58C9
:109B1000A543802494402C435C5001B0F0BD08A0C4
:109B20000FA1492212A304F045FFC0461093010281
:109B30001CED00E000E400E080E200E000E100E075
:109B4000696E636C7564652F647269766572732FD4
:109B50006D6B5F6475616C5F74696D65722E630017
:109B60006475616C5F74696D65725F6F70656E00BE
:109B7000636F6E66696720697320696E76616C69D0
:109B8000640000000001084A1058016081688022CA
:109B90000A4382607047C046000103490858816843
:109BA000802291438160704710930102F0B58DB01F
:109BB000019315460E460A901298002408900480DE
:109BC000149F3C80139809900460159804900480B9
:109BD000FF2081053046F6F7F1FB029030460396F0
:109BE0003146F6F792FB2B463D46069027460795F1
:109BF0000B9311E01180188880002858099908609B
:109C00000120079D28800520049908807F1CBCB294
:109C10001888844200D9A0E028880028F6D1A00046
:109C20000A9D2E5830460699F6F7E4FD002817D015
:109C300030460399F6F7DEFD00280B9B079DE5D122
:109C4000089A1780099D2E601888011B012934D1BC
:109C50001080198889000A9A51582960059035E0CA
:109C6000089A1780099806600B9B1988081B012821
:109C7000C0D00C96019825187E1CB0B28542BFD387
:109C800089B2B2B28A420ED880000A990C58204696
:109C90000C99F6F7A1FD0B9B002804D109980460EC
:109CA000089806800C94761CB0B28542A8D3198817
:109CB00089B2B2B28A42E7D9F5E70C9601996218E7
:109CC0007D1CA9B216468A4205972CD2059884B20B
:109CD000A5000A9E7259002C104609D0A819001F31
:109CE000016810460C92F6F710FB0C9A062C07D868
:109CF0000446A81941681046F6F707FB0C90204669
:109D0000079D0299F6F784FD00280B9B07D10C985C
:109D10000299F6F76FFD0B9B002800D076E7012033
:109D20002880032070E780B2AAB282420FD8880050
:109D30000A990C5820460C99F6F74EFD0B9B00280B
:109D400005D1099804600898058005950C946D1C50
:109D5000A9B28E42BAD31888E5E70DB0F0BD000075
:109D60000A490A680A4802400A60FD214900094A76
:109D70001268515C002908D007490A6C02400A6445
:109D8000012000060A6882430A6070470004004010
:109D9000FFFFFF7F38940102200000400020704741
:109DA000F0B583B00D4604467C26464350488719DB
:109DB000F869396AF6F78EF9A84200D892E0019561
:109DC00002940121EFF31080084002D1EFF31082DA
:109DD00072B63C4610343B690025062B0CD80A4667
:109DE0009A40D3065B0F06D161231A4275D00D4607
:109DF000002803D003E00225002800D162B6002D20
:109E000002D0284603B0F0BD00943C4620343848C8
:109E100080591021C1613E46143604F09DFD05466F
:109E20003868C069C00605D504F096FD401B31882E
:109E30008842F5D90621029D284600F00BFF2068D4
:109E400001994143B869091838688160172179562A
:109E50003C461734002909D5C16920220A43C26152
:109E60000121F966890502680A4302600521284636
:109E700000F0F0FE207840B200250028C1D42B4825
:109E800000687D24E100F6F725F96101414302985D
:109E900000F0B2FE04F060FD04463868C069C007F7
:109EA00005D004F059FD001B31888842F5D904F033
:109EB00053FD04463868C169890706D504F04CFD96
:109EC000001B31888842F5D938680121009A116059
:109ED00053498161284603B0F0BD03212160002869
:109EE0008CD08CE7034804A1084A09A304F062FD62
:109EF0003C930102C8290100666C6173685F626C63
:109F00006F636B5F65726173650000005D02000046
:109F1000626C6F636B20696478206973206F76656B
:109F2000722072616E67650D0A00000054DE010246
:109F3000F0B583B002907C214143934A5418E56EFA
:109F4000EAB2511E02291FD229040126090E18D097
:109F500001960092022100F07DFE2746143704F09E
:109F6000FBFC06462068C169890606D404F0F4FCAF
:109F7000801B39888842F5D92068007DC007019E82
:109F800008D0304603B0F0BD032A36D10092280431
:109F9000000E36D020466C302D0C0021019101605E
:109FA0002746143704F0D8FC06462068C069C0076D
:109FB00005D004F0D1FC801B39888842F5D904F023
:109FC000CBFC06462068C169890706D504F0C4FCAD
:109FD000801B39888842F5D9206811498161E9B22E
:109FE0000120002911D003290099019E00D00620EC
:109FF0002061226F002A0ED1C3E70026304603B04D
:10A00000F0BD0126304603B0F0BD0099019E2061ED
:10A01000226F002AB5D002A89047304603B0F0BDA9
:10A02000000093EB70B5002801D0012070BD7825A9
:10A03000CD4E705D00280ED000240921204600F08E
:10A0400009FE0F20FFF7CAFB1520FFF79BFA745596
:10A050003461204670BD042070BDC046F0B581B0AB
:10A060000C460078484EF16881422CD1032C54D123
:10A07000706EB16E884261D900240621204600F03E
:10A08000E9FD3068F16D81602046214600F0E2FD77
:10A09000354660352CCDF0683168B48C414F00975F
:10A0A0005B1BA34200D81C46A3081431FFF776FCC3
:10A0B000B06E0019B066306E00193066F06D001990
:10A0C000F06501B0F0BDB168814255D1032C45D196
:10A0D000F08CF16D0918F165316E09183166B16EB9
:10A0E0000818B066716E814238D9002406212046D6
:10A0F00000F0B0FD3068F16D81600121204600F074
:10A10000A9FD316EB068F38C3268264C009414328D
:10A110009B08FFF743FC01B0F0BD30681021C1611E
:10A1200004F01AFC05463068C069C00616D504F074
:10A1300013FC401BB18A8842F5D90FE0306810212A
:10A14000C16104F009FC05463068C069C00605D548
:10A1500004F002FC401BB18A8842F5D90120C107F6
:10A16000326813688B431360F16E22040A430002C5
:10A170001043F06601B0F0BD4D200201034804A178
:10A18000844B04F017FCC0463C930102C82901002F
:10A19000666C6173685F646D615F63616C6C626162
:10A1A000636B00005DA00000F0B581B000786E4DDB
:10A1B000AA68824200D0D0E001263002032942D1B1
:10A1C0006A6DAA66AB6DAC6AA418EB652C66AB6CC5
:10A1D0005B1CAB646B6E934235D95E30FFF7FEFAC1
:10A1E000686CA96C02293AD3814238D1E88C696D38
:10A1F000081868650020062100F02CFD2868E96D2C
:10A2000081602F6D04F0A8FB04462868C069C00770
:10A2100005D004F0A1FB001BA98A8842F5D904F0FF
:10A220009BFB04462A68D069800706D504F094FB9E
:10A23000001BA98A8842F5D92A687420285C012865
:10A2400041D0F10440E0F2072B681C6894431C6085
:10A25000EA6E090411430143E96601B0F0BD022929
:10A26000FBD38142F9D2E88C696D09186965A96D43
:10A270000818A8650020062100F0ECFC2868E96DAC
:10A280008160EF8C04F068FB04462868C069C00751
:10A2900005D004F061FB001BA98A8842F5D904F0BF
:10A2A0005BFB04462A68D069800706D504F054FB9E
:10A2B000001BA98A8842F5D92A687420285C0128E5
:10A2C00022D0F10421E03105334B3B4059180128DD
:10A2D00002D01920400601E00720C00608182F49C7
:10A2E00040185060002F0DD004F036FB04462A6859
:10A2F000D069800706D404F02FFB001BA98A88428E
:10A30000F5D92A682B6D1FE03105234B3B40C91856
:10A31000012802D01920400601E00720C0060818D5
:10A320001E4940185060002F0DD004F015FB044664
:10A330002A68D069800706D404F00EFB001BA98AA6
:10A340008842F5D92A68EB8C296EA868144C0094D1
:10A350001432FFF723FB01B0F0BD044804A10C4AFE
:10A360000C4B04F027FBC0463C930102C8290100B6
:10A37000666C6173685F646D615F77726974655F55
:10A380006E62797465735F63616C6C6261636B00AC
:10A3900072040000AF290100FF3F00000080800030
:10A3A000A9A10000F0B587B004460126880E14D09C
:10A3B0001546002A11D00F468120C004401B884258
:10A3C0000BD37C206043F04908180590818C3846F7
:10A3D0000691F5F77FFE002902D0304607B0F0BDA8
:10A3E00028460699F5F776FE0029F6D1059880698A
:10A3F0003E1A30460699F5F76DFE0746039670192A
:10A400000190069E3146F5F765FE0546C01B049097
:10A410000598006A02903146F5F75CFE0499814286
:10A420000FD20026BD42D8D92046394600F018FB8D
:10A430002046FFF77DFD0028FAD17F1CAF42F3D301
:10A44000CBE700900398029D2946F5F743FE0646A8
:10A45000284670430399081A019800D0761C2946B3
:10A46000009D7543F5F736FE05900299414301982A
:10A47000401A03900699F5F72DFE0490AF420BD2D7
:10A480002046394600F0ECFA2046FFF751FD00283F
:10A49000FAD17F1CAF42F3D305988642069D009FF8
:10A4A0000CD220463146FFF77BFC2046FFF740FDEB
:10A4B0000028FAD1761C05988642F2D30398A84268
:10A4C00003D20026304607B0F0BD0598474300256B
:10A4D000E919204600F0C4FA2046FFF729FD0028BC
:10A4E000FAD16D1C002604988542F1D375E7C04669
:10A4F000F0B585B0002803D00124204605B0F0BD9A
:10A500007822A14FB85C002803D00024204605B073
:10A51000F0BD0492002905D0384614300CC90CC097
:10A520001CC91CC00020F86615242046FFF732F82D
:10A53000204603F061FF38681021C16104F00CFA75
:10A5400004463868C169C90607D504F005FA001B3E
:10A55000B98A8842F5D9386800E0B98ABA7D12070D
:10A56000120B5218F97DCB07DB08D2188B07DB0FD3
:10A570005B05D218CB06DB0FDB05D2184B07DB0FD0
:10A58000DB06D2188B06DB0F5B07D2180907C90F51
:10A5900089071143016000240A21204600F05AFB7C
:10A5A0003220FFF71BF90821204600F053FB04F08E
:10A5B000D3F905463868C169890606D404F0CCF998
:10A5C000401BB98A8842F5D93868017D0A46C23AEB
:10A5D0005342534174257B550904027D12025118E0
:10A5E000007D0B180220032668A2314605F03EFAD2
:10A5F000785D0128039619D1F87D02900026062186
:10A60000304600F027FB0721304600F023FB0121F4
:10A6100002988143785D012847D138688901017526
:10A6200006757521795C012938D048E000200321A6
:10A6300000F010FB04F090F906463868C1698906FD
:10A6400006D404F089F9801BB98A8842F5D93868A4
:10A65000007D46080122F87D014631431640C907B6
:10A6600001D0304036D002950025062128460192BF
:10A6700000F0F0FA07210095284600F0EBFA019867
:10A6800046400298385C012813D13868B101017541
:10A69000009901757521795C012910D1143076215A
:10A6A000795C4A424A41510008E038680675490021
:10A6B00003E0386800990175710014300170374863
:10A6C00000687D21C900F5F705FD282141430020E0
:10A6D00000F092FA7720385C012803D10220002193
:10A6E000FEF7E8FF04F038F906463868C069C0078D
:10A6F00005D004F031F9801BB98A8842F5D904F0FD
:10A700002BF906463868C169890706D504F024F993
:10A71000801BB98A8842F5D93868D04981611720F1
:10A720003856002829D57868002816D40146039A9F
:10A7300091431C4A8B588507ED0EFF26AE40B3436C
:10A740008026AE401E438E501F21014001208840CC
:10A7500015490860154908600FE08107C90EFF22FE
:10A760008A400F230340083B039883430C481D583D
:10A77000954380228A402A431A5001200499785434
:10A780003861204605B0F0BD3C9301026A656465FE
:10A79000635F69642025780D0A00000054DE010221
:10A7A0001CED00E000E400E080E200E000E100E0F9
:10A7B000F0B593B07C270A9047439348C619980791
:10A7C00004D0F07D4024044000D017E10125880E1C
:10A7D0002ED0002B2CD08120C004C01A884227D351
:10A7E00009920122EFF31084144002D1EFF310809C
:10A7F00072B6304610300590306900250628089161
:10A80000069310D8079414468440E106490F04D1FA
:10A8100061210C4203D0154604E0022502E002212A
:10A82000059B1960079C002C00D162B6002D02D058
:10A83000284613B0F0BD344617347348C059102170
:10A840000491C1613746143704F086F80546306834
:10A85000C069C00605D504F07FF8401B39888842DE
:10A86000F5D92078400665D40297B78C069C20461F
:10A870003946F5F72FFC079039464143601A03909B
:10A8800035462435A74200D894E0039800281CD010
:10A8900006210A9C204600F0DDF9288807994843E4
:10A8A000089940183168886000272046039C394683
:10A8B00000F0D0F9079B099A28885843C0193168DD
:10A8C000097D11547F1CA742F6D330680499C161F9
:10A8D00004F042F80446029D3068C069C00605D500
:10A8E00004F03AF8001B29888842F5D904F034F8BE
:10A8F00004463068C069C00705D004F02DF8001B7D
:10A9000029888842F5D904F027F804463068C169DF
:10A91000890706D504F020F8001B29888842F5D95C
:10A9200030680121059A1160B249816100252846ED
:10A9300013B0F0BD03200025089FF7650999316623
:10A9400006997166B566F0660120C00731680A682D
:10A9500002430A6006210A9C204600F07BF9306819
:10A9600087602046294600F075F93A4F0BAA0A92F3
:10A970001BCF1BC21BCF1BC2B48CF0680A99FEF719
:10A980009DFFF0683168344A0092069A944200D3E1
:10A990001446A3081431099AFFF700F8B06E0019A5
:10A9A000B066306E00193066F06D0019F06528460B
:10A9B00013B0F0BD002404E0641C0798844200D367
:10A9C00063E706210A9800F045F928886043089952
:10A9D00040183168886000270A98394600F03AF933
:10A9E00028880028099AE7D0604310183168097D4B
:10A9F000C1557F1C28888742F6D3DDE7034804A1B0
:10AA0000064A07A303F0D6FF3C930102C8290100C0
:10AA1000666C6173685F726561640000C603000064
:10AA200054686520444D412072656164206C656EF8
:10AA30006774682073686F756C6420626520746841
:10AA400065206D756C7469706C65206F6620340DBF
:10AA50000A0000003C1E01005DA00000000093EB16
:10AA6000F0B583B00D4604467C264643514887190D
:10AA7000F869B98CF5F72EFBA84200D894E001954F
:10AA800002940121EFF31080084002D1EFF310820D
:10AA900072B63C4610343B690025062B0CD80A469A
:10AAA0009A40D3065B0F06D161231A4277D00D4638
:10AAB000002803D003E00225002800D162B6002D53
:10AAC00002D0284603B0F0BD00943C4624343948F7
:10AAD00080591021C1613E46143603F03DFF054602
:10AAE0003868C069C00605D503F036FF401B3188C1
:10AAF0008842F5D90621029D284600F0ABF820884F
:10AB000001994143B869091838688160172179565D
:10AB10003C461734002909D5C16920220A43C26185
:10AB20000121F966890502680A430260042128466A
:10AB300000F090F8207840B22C4600250028C0D4C0
:10AB40002B4800687D21C900F5F7C4FA20492D3152
:10AB50004143204600F050F803F0FEFE04463868FA
:10AB6000C069C00705D003F0F7FE001B318888429A
:10AB7000F5D903F0F1FE04463868C169890706D5A6
:10AB800003F0EAFE001B31888842F5D938680121BC
:10AB9000009A116017498161284603B0F0BD032176
:10ABA000216000288AD08AE7034804A1084A09A343
:10ABB00003F000FF3C930102C8290100666C617339
:10ABC000685F736563746F725F65726173650000BF
:10ABD0002B020000736563746F72206964782069CA
:10ABE00073206F7665722072616E67650D0A0000D2
:10ABF00054DE0102000093EBF0B583B001917C229A
:10AC00000290424353498C182546143503F0A4FEA4
:10AC100006460221029800F01DF803F09DFE07464B
:10AC20002068C169890606D403F096FEC01B2988F6
:10AC30008842F5D92068007DC00708D06420FEF75F
:10AC4000CDFD03F089FE801B01998842E1D903B054
:10AC5000F0BDC046F0B585B0049104467C20604349
:10AC60003C490F183D46143503F076FE0646386819
:10AC7000C069C00705D003F06FFE801B2988884299
:10AC8000F5D903F069FE06463868C069800705D526
:10AC900003F062FE801B29888842F5D91421049BA9
:10ACA0005943DC2060432C4A10180390029140184D
:10ACB000018A8268C47C7426BE5D012E0DD101918B
:10ACC000012B02990CD0012B0DD07526BE5D012EF3
:10ACD0000ED0019E072B0ED10EE00E4602990BE01E
:10ACE0000222012BF1D138247526BE5D012EF0D150
:10ACF0000326072B00D0019E184B334024069207F1
:10AD0000D20A1219D218039B5958C907490C521874
:10AD10004168CB071B0CD218837C5B075B0BD218F6
:10AD2000C0684007000A10183A685060002E0ED024
:10AD300001290CD103F010FE04463868C069800771
:10AD400005D403F009FE001B29888842F5D905B017
:10AD5000F0BDC0463C930102841F0100FF3F00008C
:10AD6000F0B59DB00D460126890E2FD0002B2DD0B9
:10AD700011928121C9041093C91AA94226D3012135
:10AD8000EFF310840C4002D1EFF3108272B67C22F4
:10AD90000F904243E74814928718384610303B69B9
:10ADA0000026062B0DD80A469A40D3065B0F07D122
:10ADB00061231A4200D16FE30E46002C03D003E05A
:10ADC0000226002C00D162B6002E02D030461DB003
:10ADD000F0BD0290BD650021139179651098401E69
:10ADE00012904019B964B9690D916E1A1199B9623E
:10ADF000FD6238637E63F98C0E913046F5F76AF98F
:10AE00000446B863129830180E9E3146F5F762F981
:10AE1000109B011B4A1CF86339647A64139A002959
:10AE2000194608D0704359190D9BC91A0A1A744360
:10AE3000581B80190119384648300E903846443066
:10AE40000D90384640300B903846263005903846F5
:10AE500058301390384654301290F9643A6514987B
:10AE6000B44908581021C16138461430149038464E
:10AE7000503004903D464C3503F06EFD0446386872
:10AE8000C069C00606D503F067FD001B1499098848
:10AE90008842F4D9F87D40060C9500D574E2012370
:10AEA0000E9803600D98016800290F9800D1CDE23B
:10AEB0003A4674320A92DA0407921A050992192264
:10AEC000520606920722D206089216E09A480068B7
:10AED0007D21C900F5F7FEF8109941430F9C2046EB
:10AEE000FFF78AFE20460C9D0E9A11684B1C1360DA
:10AEF0000D9909688B4200D9A8E20B9A1268012AC1
:10AF000055D0002A00D0A8E02E6812990C68139939
:10AF10000D6806211091FFF79DFE38688560119835
:10AF2000051903F019FD04463868C069C00706D04A
:10AF300003F012FD001B149909888842F4D903F02C
:10AF40000BFD04463868C169890707D503F004FD85
:10AF5000001B149909888842F4D938680A990A783C
:10AF6000012A089900D00699012A099A00D0079A67
:10AF70003346724C234013430B4371490B434360E8
:10AF8000002EA3D003F0E8FC04463868C0698007AF
:10AF900006D403F0E1FC001B149909888842F4D917
:10AFA0003868297801756D1C761EFAD18EE7012B61
:10AFB00000D0C7E02E6812990C6813990D6806211D
:10AFC0001091FFF747FE386885601198051903F066
:10AFD000C3FC04463868C069C00706D003F0BCFC57
:10AFE000001B149909888842F4D903F0B5FC044683
:10AFF0003868C169890707D503F0AEFC001B1499B6
:10B0000009888842F4D938680A990A78012A089987
:10B0100000D00699012A099A00D0079A3346474C76
:10B02000234013430B4346490B434360002E69D032
:10B0300003F092FC04463868C069800706D403F028
:10B040008BFC001B149909888842F4D93868297848
:10B0500001756D1C761EFAD154E0012B00D0C9E0B9
:10B060002E6812990C6813990D6806211091FFF74C
:10B07000F1FD386885601198051903F06DFC0446F0
:10B080003868C069C00706D003F066FC001B14993D
:10B0900009888842F4D903F05FFC04463868C16926
:10B0A000890707D503F058FC001B149909888842CA
:10B0B000F4D938680A990A78012A089900D00699C3
:10B0C000012A099A00D0079A33461C4C23401343A7
:10B0D0000B431B490B434360002E13D003F03CFC91
:10B0E00004463868C069800706D403F035FC001BAD
:10B0F000149909888842F4D93868297801756D1C3B
:10B10000761EFAD10C4800687D21C900F4F7E2FFF1
:10B11000109941430F9C2046FFF76EFD20460C9D81
:10B120002A68139B196889181960129B1968891875
:10B130001960D9E63C93010254DE0102FF3F000092
:10B14000008080008B4200D0CEE604990E681299F0
:10B150000C6813990D6806211091FFF77BFD386884
:10B1600085601198051903F0F7FB04463868C0693B
:10B17000C00706D003F0F0FB001B14990988884231
:10B18000F4D903F0E9FB04463868C169890707D59B
:10B1900003F0E2FB001B149909888842F4D938684F
:10B1A0000A990A78012A089900D00699012A099A71
:10B1B00000D0079A3346D44C234013430B43D34962
:10B1C0000B434360002E00D180E603F0C5FB04462C
:10B1D0003868C069800706D403F0BEFB001B1499D1
:10B1E00009888842F4D93868297801756D1C761E63
:10B1F000FAD16BE6129A1268119CA618139A156878
:10B200008B425FD104990C6806210391FFF722FD60
:10B210003868856003F0A0FB05463868C069C00740
:10B2200006D003F099FB401B149909888842F4D991
:10B2300003F092FB10900C9D3868C169890708D50E
:10B2400003F08AFB1099401A149909888842F3D9AF
:10B2500038680A990A78012A089900D0069910914D
:10B26000012A099A00D0079A2346A7490B401343A5
:10B2700010990B43A5490B434360002C14D003F0F5
:10B280006BFB10903868C069800707D403F064FB3B
:10B290001099401A149909888842F3D9386831788E
:10B2A0000175761C641EFAD19A4800687D21C90098
:10B2B000F4F710FF039941430F9C2046FFF79CFCD5
:10B2C000204611E605990C8806210391FFF7C2FC80
:10B2D0003868856003F040FB05463868C069C007E0
:10B2E00006D003F039FB401B149909888842F4D931
:10B2F00003F032FB10900C9D3868C169890708D5AE
:10B3000003F02AFB1099401A149909888842F3D94E
:10B3100038680A990A78012A089900D0069910918C
:10B32000012A099A00D0079A234677490B40134314
:10B3300010990B4375490B434360002C14D003F064
:10B340000BFB10903868C069800707D403F004FB3A
:10B350001099401A149909888842F3D938683178CD
:10B360000175761C641EFAD16A4800687D21C90007
:10B37000F4F7B0FE039941430F9C2046FFF73CFCD5
:10B38000204605990A88CCE65E4815A90A4678C881
:10B3900078C278C878C20125E8073A681368034381
:10B3A0001360B868FEF78AFA02200026139C216811
:10B3B000BA6AF9653A6610997966BE66F8660C98BD
:10B3C0000068129A1168091811600E9B19684A1CCE
:10B3D0001A60226810182060002900D0F6E4109549
:10B3E0003846603013903C465C3438460830129042
:10B3F00006210F98FFF72EFC3868216881600C98B1
:10B400000068119003F0A8FA04463868C069C007C4
:10B4100006D003F0A1FA001B149909888842F4D9D8
:10B4200003F09AFA0446109D3A68D069800707D560
:10B4300003F092FA001B149909888842F4D93A68FB
:10B440007420385C01282DD0E9042CE003F084FA44
:10B4500004463868C069C00706D003F07DFA001BB7
:10B46000149909888842F4D903F076FA04463868BA
:10B47000C169890707D503F06FFA001B1499098881
:10B480008842F4D938680121029A11602249816109
:10B49000002630461DB0F0BD04210160002C00D113
:10B4A00091E491E42905119C174B23405918012878
:10B4B0000C9D02D01920400601E00720C0060818A4
:10B4C000124940185060002C0ED003F045FA044693
:10B4D0003A68D069800707D403F03EFA001B14993C
:10B4E00009888842F4D93A682B6813980168129841
:10B4F0000068074C00941432FEF750FA30461DB035
:10B50000F0BDC046FC1D0100FF3F00000080800030
:10B51000A9A1000054DE0102000093EB3920C00015
:10B520000149096808587047C8920102F0B503291B
:10B5300020D8C0467944097949008F4401080F1585
:10B54000012181404F4B1B685963D96212E00121F0
:10B5500081404C4B1B681963D9620BE0012181408B
:10B56000484B1B68596304E001218140454B1B682F
:10B570001963996283004349CB18DA608A68002A0C
:10B5800029D14A68002A16D4032314469C43174B3A
:10B59000E5589607F60EFF27B740BD438027B74012
:10B5A0002F43E7501F23134001229A40104B1A608B
:10B5B000104B1A600FE09307DB0EFF259D400F2410
:10B5C0001440083C03229443074AA658AE43802502
:10B5D0009D403543A5500122824008680262886878
:10B5E00010438860F0BDC0461CED00E000E400E0C0
:10B5F00080E200E000E100E010B501242046FDF704
:10B60000C9FF204602F0F8FE002010BD0121814054
:10B610001C48006842688A434260704719490968BB
:10B620000968C140012008407047C046012181409F
:10B630001448006842680A4342607047012907D0F5
:10B64000002910D1012181400F4802680A430FE010
:10B65000012181400B4800684368002A0DD00B434C
:10B6600043600161704701218140074802688A43B5
:10B67000026004480068416170478B434360016188
:10B680007047C046CC93010208010040124A0728C7
:10B6900009D880000F2383408140194010689843E7
:10B6A0000843106070470F280AD8800020380F2305
:10B6B0008340814019405068984308435060704768
:10B6C000800040380F2383408140194090689843A0
:10B6D000084390607047C04634000040F0B543070F
:10B6E000DC0E0726A640C3089D000E4BEF187D68B0
:10B6F000B5433E1D002908D0356001228240012952
:10B700000CD1186810431860F0BD01218140186801
:10B7100088431860A24015433560F0BD1868904317
:10B720001860F0BD0C01004010B582B014460A4606
:10B7300001460498009301900820234600F092F8F7
:10B7400002B010BDB0B584B014460A460146089850
:10B7500002250095019302900720234600F052F93C
:10B7600004B0B0BD70B500285BD031490A783149CA
:10B77000002A03D14A68012313434B60428803889F
:10B780001B049A180B46183B1A60828883891B0495
:10B790009B180C460C3C23600B46083B84681C60DD
:10B7A000446903232340057CAD00EB188569AD0790
:10B7B0002D0D5B19457C2D035B19C569AE07B60AD3
:10B7C0009B19867CB6059B190E1F3360036A122BEA
:10B7D00004D107240C60541EA2410AE0032C05D1B9
:10B7E000012D03D807220A60012202E006220A6026
:10B7F0000122114C002525700F2464012034C57CE2
:10B800006D0225401B069B0BD218C3791B07DB0E6C
:10B81000D21880790007C00D10184019143908603B
:10B8200070BD064806A1862209A303F0C3F8C046EE
:10B8300008CC0102181000500ACC01024136010068
:10B840006C73705F656E67696E655F72756E000020
:10B85000506172616D65746572206973206E756CDC
:10B860006C000000F0B58BB0109E34043ED00D4645
:10B87000D64C2140012701977F06B9423CD11146A1
:10B880002140B9423FD11C40BC4243D1119902AC86
:10B890000027E781E780668027802782A774E1740C
:10B8A0009908A181A908A1800A900997089707978C
:10B8B000900880B204902046FFF754FFAA48007811
:10B8C000002801D00BB0F0BDAB480168C90708D112
:10B8D0000168C90705D10168C90702D10168C90714
:10B8E000F3D07F48019901700BB0F0BDB8480D4905
:10B8F000AF22C14B03F05EF80095B5480949B0226C
:10B90000754B03F057F80092B1480649B122724BCB
:10B9100003F050F80093AE480249B2226E4B03F098
:10B9200049F8C04617360100F0B58DB00392139E5A
:10B93000340446D00A46A54C2140012502956F06E5
:10B94000B94244D103992140B94247D11C40BC427D
:10B950004CD11499129D04ACE1742949218200272D
:10B96000E781E780668027809908A1819108A180FE
:10B970000B95012D01D16121CF43A7740C900220BA
:10B980000A9009900398800880B206902046FFF73D
:10B99000E9FE75480078002801D00DB0F0BD76486A
:10B9A0000168C90708D10168C90705D10168C9073D
:10B9B00002D10168C907F3D04948029901700DB05E
:10B9C000F0BD83480D49FB228B4B02F0F3FF009240
:10B9D0007F480A49FC22404B02F0ECFF039800909C
:10B9E0007B480649FD223C4B02F0E4FF0093784877
:10B9F0000249FE22384B02F0DDFFC046243601002A
:10BA00008E8E0000F0B58BB0119E340447D00D46E9
:10BA10006E4C2140012701977F06B94245D111465E
:10BA20002140B94248D11C40BC424CD11299109FD0
:10BA300002ACE174294921820021E181E180668024
:10BA400021809908A181A908A1800997012F01D01F
:10BA5000712100E06121C943A1740A90032008907C
:10BA60000790900880B204902046FFF77BFE3E4886
:10BA70000078002801D00BB0F0BD3F480168C9072D
:10BA800008D10168C90705D10168C90702D1016859
:10BA9000C907F3D01248019901700BB0F0BD4C48B2
:10BAA0000C49D522544B02F085FF009548480949BE
:10BAB000D622094B02F07EFF009245480549D72265
:10BAC000054B02F077FF009341480249D822024B10
:10BAD00002F070FF333601006136010086860000F7
:10BAE0000ACC010210B582B014460A460146002075
:10BAF0000093019004202346FFF7B4FE02B010BD6E
:10BB000010B584B014460A46014600200090019307
:10BB1000029004202346FFF707FF04B010BD000089
:10BB200070B50D46064604242046FDF733FD204639
:10BB300002F062FC0B4805600B480670002E0ED028
:10BB40000A48016880220A437F218A43026001205B
:10BB5000000307490860074908600748046000209F
:10BB600070BDC0460CCC010208CC01020CE400E020
:10BB700080E200E000E100E01C100050B0B582B0AF
:10BB8000144602461148204001256D06A8420DD1F9
:10BB9000180413D01748016000200093019006207C
:10BBA00011462346FFF75EFE02B0B0BD0094FF22AF
:10BBB0008C320748074908A302F0FCFEFF208C30B6
:10BBC000421C034803490C4B02F0F4FE0300FCFF47
:10BBD00041360100093601004473742061646472C7
:10BBE00065737320257820697320696E76616C69AE
:10BBF00064000000081000507F36010080B582B05C
:10BC00000B46014600200092019003200A46FFF7F0
:10BC100029FE02B080BD0000002801D0042100E010
:10BC20000221BD4A5172411E8841800103490A68C0
:10BC300040239A43101808607047C04650A0005037
:10BC4000F0B583B002912E49CD7A0E7B77198742E9
:10BC50004FD908990191182545434126F604BF00A4
:10BC6000BE19745B34490C4057033C199B07D90C2F
:10BC70006418324B1B681B7A745375196C88032641
:10BC8000B60326409B079B0C9B193F2404401819C0
:10BC9000029CA3061B0DC0186880012A184E13D8F9
:10BCA000707B14224243307B5023434324011B19F1
:10BCB0009A18F37AC0181C234343D01880081E4AF0
:10BCC000104007430F432F800198686001F0FAFE8F
:10BCD000A860E8681A4908403030E86028690840E0
:10BCE0002721715C4018286100F08CFE686103B068
:10BCF000F0BDFF228832034803A108A302F05AFED8
:10BD000010D10102D03601006D61635F63735F6320
:10BD10006F6E737472756374000000004353206982
:10BD20006E646578206973206F7665722072616E2B
:10BD300067650D0A00000000FF070000389401024B
:10BD40000000F0FFF0B581B0009314460D460746A1
:10BD500006263046FDF71EFC304602F04DFB26213C
:10BD60001D4847540021017041708171017181703B
:10BD70004171C170C17102224272C16201634163AB
:10BD8000816304734273C572009A561C134A16806D
:10BD900001724120C00401214903F4F7DEF950206B
:10BDA00060432901081861198A00801818224A4343
:10BDB0008018B2B24A43801809494018094988429C
:10BDC00004D200F0ABF8002001B0F0BD064807A196
:10BDD0009A2209A302F0EEFD10D101020CD101025A
:10BDE0002800080201200802D03601006D61635F5F
:10BDF000696E697400000000454D206F76657266BB
:10BE00006C6F770D0A000000F0B583B002912A49EB
:10BE10004B7B834248D9CB7A0C7BE31818245C43D4
:10BE20009B00E3184124E4041A19142401900546E8
:10BE300065430026565100925519EE882E4F0B4649
:10BE40007A1C3240F44E3688497A711A2B4E0E40D5
:10BE5000B618EE803740997BEF80AA88284F1740AC
:10BE60004A424A4191007918264A8918A980264FEA
:10BE70000F402D1D029801280AD124490E400921A6
:10BE8000C902711869800121C9037918298000E06D
:10BE90002F800198444300980019074A918C4182F1
:10BEA000118C018203B0F0BD3520C200034804A10B
:10BEB00009A302F07FFDC04610D10102D036010077
:10BEC0006D61635F6C696E6B5F646573635F636F05
:10BED0006E737472756374004C696E6B2064657365
:10BEE0006320696E646578206973206F76657220BF
:10BEF00072616E67650D0A00FFFBFFFFFF03000024
:10BF000003D0FFFFE80F0000EF1F0000FF830000D9
:10BF1000BD4A50639163704710D10102F0B581B002
:10BF20004348CC21016003214160B7490A7BD30417
:10BF3000404C1B19CC7AA218541E1C43182353439F
:10BF400092009A184B7B14255D43521992012243AB
:10BF5000012463061343436100228262C2620263CA
:10BF600042638263C26342650267334B1A605A6060
:10BF70009A60324B1A601A619A61DC61304C1C6223
:10BF8000304C251D1D6325460C3D5D632546283D2F
:10BF90009D632D4EDE631C645C642C4D2F461C3764
:10BFA0009F642746143FDF64103C1C65284C5C6589
:10BFB000284C9C650C369E67274CA5634035E5638D
:10BFC000DA651A665A669A66DA661A67234DDD677D
:10BFD00002258561224DC561C325AD03CD620A638B
:10BFE000D2435A601F4A1368FF25AB4326254D5D97
:10BFF000AD072D0EEB1813601B4A102313601B4A6C
:10C000001360272260238B5419498160C16001614C
:10C0100021607D210901016641661649C164164906
:10C0200041641649016400F0DDFC01B0F0BDC0467A
:10C0300004A000500000F8FF94A0005034A100506C
:10C04000FF185A0030040040041000401C2000403B
:10C050005430004060400040B8A10050140014006B
:10C06000FF3F3FFF04E400E080E200E000E100E089
:10C07000DC05DC053F0270020133D007D007D00792
:10C080002921C54A50547047F0B58BB007920891EA
:10C090000146C14FB8780991FFF7B6FE78793A7B2F
:10C0A00079790691824200D89FE0FB7A9A1818238A
:10C0B000534392004124E10404915218D2187B7B2F
:10C0C00014214B43D21850246043155801230A937E
:10C0D000DB022E469E4316504E4B2B4005937D7B34
:10C0E00003914D433E7B7443F97A0B011B195B1995
:10C0F00071181C24029461435918A84B1B88069C94
:10C100005C430919C904490D059BC9181150101841
:10C110000799416038787979089A00920322099B3F
:10C12000FFF78EFDF87A397B09183878814263D998
:10C1300083000993049AD45C0894F7212140D154D8
:10C14000D1184D788E7836027619CB781B04F31807
:10C1500007900A9886051E43330CCB70FB7A387B18
:10C16000BC784D709F4D3540039E6643C018029BBE
:10C170004343981940029C4B03405C19200A887085
:10C18000200CC870F023089D2B401B1D3D7B08959B
:10C19000FE7A099D5355C8700620079A50438019AE
:10C1A000089A801848701F22D20222400243100AC7
:10C1B00088707879401C7871387B7979814201D315
:10C1C000002179713978491C3970F97A0818397861
:10C1D000884201D80020387028200A993954387ACA
:10C1E000401C3872387A0BB0F0BDA7204200D2480C
:10C1F0000649074B02F0DEFBA72042007A32CE4808
:10C200007349744B02F0D6FB10D10102F0360100E5
:10C210009936010000F0FFFF0CD101020320000657
:10C2200005490A6882430A600A6802430A600348B3
:10C23000012101607047C0461C0000401CA0005056
:10C2400080B50120FDF7A8FC80BD0000F0B587B0E7
:10C2500006930646504C607A504B1B88181A0C9D6A
:10C26000A84200DC89E00F460592012E06D156480F
:10C270000021C1620169554A89180160A0783146E0
:10C28000FFF7C2FDE078E178069A2B4600F0AEF8A1
:10C290002078E1780097002206923346FFF7D0FC21
:10C2A000E07A217B0818217888426ED94120C204A7
:10C2B00004918800815C0391F7250D40029285541A
:10C2C0004549455C4549465C360276194449475C18
:10C2D0003F04F6190127BF0537433E0C4654E67A62
:10C2E000217BA3783C4A85543E4D3D4014275F4353
:10C2F00089191C234B43D91949023B4B0B405D194B
:10C30000290A364BC1542E0C35494654F02703995F
:10C310000F400599002900D13F1D217BE37A029A45
:10C3200087542F4A86540622049E7243D21851180D
:10C33000294A81541F22D20215400D43290A274A57
:10C340008154E078401CE070E07AE178814201D3CA
:10C350000699E1702178491C2170217B0818217809
:10C36000884201D806982070E079401CE071A07ADC
:10C37000401CA072E07907B0F0BD3920C20016322F
:10C38000074808A109A302F015FB3920C2000448A0
:10C390000F49104B02F00EFB10D101020CD101022B
:10C3A000D03601006D61635F747800004D41432019
:10C3B0005458206C656E206973206F766572207208
:10C3C000616E67650D0A00000804004090D003000C
:10C3D00006370100B736010001000802020008021A
:10C3E00003000802FF07C0FF00F83F00F0B589B066
:10C3F0000893019204914F4DEF7A874200D891E063
:10C40000297B502632464A434124E3040693D2183E
:10C41000CC19A10051181822059254430A19697BBE
:10C4200014230793594353180290000119580446E6
:10C430000390504A0A40A97AC90251180898820507
:10C44000D2088A181A514C4911402A7B009656434B
:10C45000384CE57A2C0106982418A719354E541942
:10C46000A5007D19059844432819747B079D6C43EA
:10C470000519049FD2194148048854432A19089C7D
:10C48000D204520D51181D460398195000F0C4FAF9
:10C490000146707A001902043E460CD080B2C000FA
:10C4A000002900D1801E029FA5214900F3F712FE4A
:10C4B0001F21014001E00021029F38012818427924
:10C4C00083791B029A18C3791B04D2182C4B134092
:10C4D000437109045918090CC171002C20D015486A
:10C4E00035460646007B009B4343F17A0A01069FCE
:10C4F0003A43D21841188B00D218059B4B43D118F0
:10C50000727B079B5343C91840191C4A1288424347
:10C5100088180199884203D001992246F3F704FE56
:10C5200009B0F0BDFF225C32034804A109A302F068
:10C5300041FAC04610D10102D03601006D61635F3F
:10C5400074785F646573635F636F6E737472756331
:10C55000740000005458204445534320696E6465BC
:10C5600078206973206F7665722072616E67650D41
:10C570000A000000FF0700E000F8FFFF0CD10102F5
:10C58000EFFFE00084B0FCF717FE052000252946E8
:10C59000FFF77CF806202946FFF778F80A2029469D
:10C5A000FFF774F809202946FFF770F801242046A8
:10C5B00003F0A2FB284603F09FFBFCF741FE072196
:10C5C0002046FCF733FE01F097FE01F08FFE7F4816
:10C5D00001687F4800688903029408D40321090791
:10C5E00008402107884202D0FCF74EFD06E0FCF728
:10C5F00031F9FCF78FFD0020FDF714FDFCF75CFE20
:10C600000025284604F090FC032672A230463146ED
:10C6100003F02CFA30462946FBF73CFEF8F706FB00
:10C62000FBF716FBFEF7E8FFF8F718FBF7F792FDAC
:10C63000F6F70AFDFAF722FCF6F7F0FC6B4E301D18
:10C64000FCF7C2FB01F034FE002816D1112631049C
:10C65000674D30462A460B46FBF72CF87D208700B5
:10C660003846FDF7B4F83002604E294602462B46A4
:10C67000FBF720F83846FDF7AAF8FAF7C3FD029C4D
:10C68000A2025C495C4B204603F034FE01F0F4FB4F
:10C690005A4A2046214602F0A3F8A00302F0D0F83F
:10C6A000052000273946FAF7BFFBA24D284628305F
:10C6B000534A01902146FCF7F9FA5248FCF7D0FCA6
:10C6C000514800F03BF9FCF77BF8FAF79DFB039724
:10C6D0000DE0029C4D48047034704D48077003F023
:10C6E000F5FA20462146FAF79FFBFBF753FC04F0CE
:10C6F00041F97078002803D1F8F790FA00280ED09D
:10C70000A879012803D10220A871FBF7AFF9F8F747
:10C7100099FAF7F747F8F7F777FAFBF7A7FAE87A05
:10C7200000282BD0EF726879411C69713D2809D32C
:10C730006F7105203946FAF777FB01210198304ADD
:10C74000FCF7B4FAF7F79CFA6A48478F3846F4F7D3
:10C75000ABF80146AE693046F4F768F804467F202E
:10C76000C1053046F3F7D1FD0646781CF4F791F881
:10C77000002C00D13046A8611C4E039F01F0A6FD9D
:10C780000446F7F73DFA002C07D1696A401A0328DE
:10C7900004D302982871F7F733FA686201F088FD34
:10C7A0003178002802D000299FD192E701299CD13D
:10C7B00037705048C78315480770029C14480470AE
:10C7C00003F070FA204639468DE7C0461800004055
:10C7D000300001405557422073696D706C652065CB
:10C7E00078616D706C650D0A000000001C900102FC
:10C7F000111111000CCD01022D050100C1E700004F
:10C80000998B00003DC8000005C900001890010286
:10C8100019900102014800687047C0460C000040B2
:10C8200081B080B581B0039303AB009302F098FD13
:10C8300001B080BC02BC01B0084700003D480021A7
:10C8400081617047F0B581B0002630463146FDF772
:10C850004FFE0125AC022649264F30463A46234674
:10C86000FDF7A6FF3988244881423ED064217E52DC
:10C8700062217E5260217E524422BE52FD87BD87D6
:10C8800078227A8702223A874322FA86BE83FE8183
:10C890001A4ABA817E810A223A81C822FA80184A4D
:10C8A000BA803880FE8306203885F984FF20123054
:10C8B00078848730B88450203E523A83EFF310805A
:10C8C00072B630463146FDF713FE00280CD12A031C
:10C8D00000263046064D2946FDF764FD054A3046E0
:10C8E00029462346FEF73CFA62B601B0F0BDC046C9
:10C8F00000E0020456A80102AA550000E1FF000072
:10C900003412000010B54020094C2146FAF7BEFB56
:10C910006078810602D4C00705D010BD0549002209
:10C920008A61C007F9D103480349C18010BDC046E0
:10C9300004960102609901020103000070B50C4EDB
:10C94000306011240025204629462A46FEF776FE4F
:10C95000032220462946FEF7C1FE32680221204606
:10C96000FEF7E4FD2046294601F00CFB70BDC046F1
:10C97000409601020020704710B50024002809D01D
:10C98000002905D003464A0003481946F3F7CCFBBB
:10C99000204610BDE04310BD309301020146002047
:10C9A0000A2901DAC0437047014A11807047C04626
:10C9B000B89301020020704780B50188064A1180B3
:10C9C0008178064A1170C178054A11700079FCF728
:10C9D000E1FA002080BDC0462294010224940102A5
:10C9E0005CD1010204480549016015210904416038
:10C9F000034981607047C0469C30004041000800F8
:10CA0000340007000748006840697047FD20400077
:10CA100004490968085C7047024800686221405C6C
:10CA20007047C046389401020A491A220A600A492E
:10CA300048704878FF210902084A13688B43800335
:10CA400080B2C018106006482021016005480160CE
:10CA500000207047702000402894010204E400E0A8
:10CA600080E200E000E100E0F0B5A9B016460F4614
:10CA70000546C648002B024600D01A463921CC0094
:10CA80003D21C900511811918242189206D001200F
:10CA90004202BE491898F3F747FB189A6120111912
:10CAA00013910E21119C0A91A170002F0D9501D0B8
:10CAB0000A2100E00921592317938300E17078428D
:10CAC000784113990870307810901070F17AE17401
:10CAD00071785170B7789770F178D1703579157198
:10CAE00074795471B1799171F179D171317A11728E
:10CAF000717A5172B17A91727E1EF0B200210328D0
:10CB0000169106D870B28000A1A210586A00805A0F
:10CB10001690179882001898C0181490F81E0228D2
:10CB200004D3012E084604D89D4800E09D4803190F
:10CB300018781290189DA818179028463030159034
:10CB40002C4656346D2080002950974A974B149EEE
:10CB500033627262B362F2623176F182139B597072
:10CB600009229A70281841608160C16001611098A3
:10CB700080008F490858F3F7FFFE012F10900F91A6
:10CB800004D0022F05D17F217E2004E07C217B2070
:10CB900001E05B215A20159DA984207003200C9090
:10CBA000A080012666701F200B90A8821820A87410
:10CBB0000A46083A179BDA76169B129AD2184A430D
:10CBC0009100189A9163B702791E8B420E9109D990
:10CBD00078486080342068847748288277481399A1
:10CBE000088339E07F2B10DD802B18D031028B4277
:10CBF0001BD071028B4227D16E49618068846F48D7
:10CC000013990883CF20C00025E0202B17D0402B9C
:10CC10001AD1684860800420688469481BE0654830
:10CC2000608006206884674815E0624860801020B4
:10CC30006884624813990883C520C0000BE06248ED
:10CC400060800220688404E0042068848120400021
:10CC50006080FF2002302882104600F0D7FE129834
:10CC6000102806D0402808D108201499C87607203B
:10CC700000E004201799887002E017980C998170E1
:10CC80001898169A8078C11E02290CD3022811D058
:10CC900001280CD12672BA4200D900266672BA4227
:10CCA00013D8F44812E00D200002119908800120E9
:10CCB000800201E00C9800022081BA4201D8EE48BF
:10CCC00000E0FA20179988600EE0FA201799886032
:10CCD000139800780028119901D0E8484880E84866
:10CCE000139A1083E7480880A88CF3F7E5FD002627
:10CCF000E54B3246F3F790FC02460B46E3493046DB
:10CD0000F3F7F2FCE24B3246F3F786FCF3F710FE42
:10CD10000746E080DF493046109A0F9BF3F7E4FCAA
:10CD2000DD4B3246F3F778FCF3F702FE78434042DE
:10CD3000800B608116990E98814208D90C20149FAF
:10CD4000B872D648179988831220189A0EE0480ABC
:10CD5000189A149F01D00D2003E0080A00D1DBE2ED
:10CD60000A98B872CE48179988831220F872D07842
:10CD7000052844D878440079400087440227402C95
:10CD80003339C848B881C8482FE0C046C89001026E
:10CD9000AC1D0100AC1D0100BC1D0100BC1D01004B
:10CDA0009A1A0100A11A0100307500001027000036
:10CDB0005C1B010005020000FF06000004080000E3
:10CDC0000A0400003604000003020000B748F8819E
:10CDD000B748388013E0B748F881B7483882B74879
:10CDE00038600CE0B448B881B5481799C88306E0AC
:10CDF000B4487882B448B8800B9800069064AE4876
:10CE00003881A748F880B14802882A84B048007861
:10CE1000E874B0480078119F7875387D1390002829
:10CE20005ED0AD490A681023DA413A600A794B793D
:10CE3000CF8867801B029A186A840A7A4B7A8F7AA5
:10CE4000C87A0D7B65701B029A183B04D218000645
:10CE50001018179FF860487B8A7BCB7B3B771202C8
:10CE600010186081087C7877487C149A9072887CCE
:10CE7000D072C87C159B1874087D5874487D119039
:10CE80009874C87D0A7E120212181A84887DD8749C
:10CE900018464B7EC375887ECD7E2D022818B8803B
:10CEA000087F4D7F2D022818F880887FB877C87FCB
:10CEB000F8772020085C149D28732120085C687393
:10CEC0002A20085C2A314D782D0228188D782D04EF
:10CED0004019C9780906401818998864119801E02A
:10CEE000EB7DA87C7D498B700A8080001F38C8824A
:10CEF000C883139800281FD022227748825C0346FB
:10CF000022335B781B029A180A842422825C03462F
:10CF100024335B781B029A18CA842622825C03465B
:10CF200026335B781B029A188A832822825C283079
:10CF300040780002801888846948032569A2294640
:10CF400002F094FD189F387814907B78B8780F9091
:10CF5000FA78B8791390F8791190387A1090787A35
:10CF6000B97A0890099100930F980190029216984F
:10CF700003901298049013980590119806901098B9
:10CF80000790FAA2F8482946149B02F06FFD3D462F
:10CF9000643580212846F3F7E0F8B878C11E0229ED
:10CFA0000ED3012800D18FE1022800D0ABE1169109
:10CFB000149078787F225043F7494018F74907E0EA
:10CFC0001691149078785B225043F1494018F1494A
:10CFD00041182846F3F7A8F80D9D1898C6870E3417
:10CFE000324602E0641C0F2A0ADA21780029F9D0BF
:10CFF000491C8907C90F91400E43C687521CF1E7AF
:10D000001699022907D31499491E012900D97DE1F7
:10D010004279D24901E04279CF4989180C78002D34
:10D0200000D177E1C1790E91032900D94AE1427913
:10D03000062A00D979E14921890041181191E4308B
:10D0400010900E98401E129019A800190F900023FE
:10D050001392149403E01898290600D15AE1052A86
:10D060005AD8C0467A44127952009744455C72857A
:10D0700098ABC04688130000E20400000C080000D2
:10D08000060A0000040F00000000104130C1BD413D
:10D09000000070400000F0400000D041120C000081
:10D0A000140B000012120000140E00000E160000F7
:10D0B000130D0000121600000E120000140B0E0AD1
:10D0C00012080000101600000E0B0000229401024E
:10D0D000249401025CD1010268D101029094010202
:10D0E000010800004361736520706172616D6574B1
:10D0F0006572733A200D0A001693DFB2002F04D038
:10D1000019A801223946F3F721F8002C00D191E04B
:10D1100019A8C019BB498AE0E8B2022867D00027E5
:10D12000022867D06BE00E98022872D1E8B202287C
:10D1300000D103461693DFB2002F04D019A80122B4
:10D140003946F3F703F8002C74D019A8C019ACA124
:10D150006DE0E8B2022800D104231693DFB2002F5D
:10D1600004D019A801223946F2F7F0FF002C61D053
:10D1700019A8C0199FA15AE0E8B2022800D10623DD
:10D180001693DFB2002F04D019A801223946F2F716
:10D19000DDFF002C4ED019A8C01992A147E0E8B2DB
:10D1A000022800D10C231693DFB2002F04D019A857
:10D1B00001223946F2F7CAFF002C3BD019A8C0194A
:10D1C000874934E0E8B2811E4A424A41970002286A
:10D1D00004D119A801223946F2F7B8FF002C16D065
:10D1E00019A8C0197CA12246F2F79EFF0FE006277E
:10D1F000022804D119A801223946F2F7A7FF002C12
:10D2000005D019A8C01980492246F2F78DFF16975C
:10D2100010E01693DFB2002F04D019A8012239467E
:10D22000F2F794FF002C05D019A8C01973492246C3
:10D23000F2F77AFF3C193F2C05D80F98C01940210E
:10D24000091BF2F78AFF12980228189801D20020D1
:10D2500002E0C078411E884115990870611E2E4673
:10D26000E8B202280CD1179A517019A9119AB8C9BD
:10D27000B8C2B8C9B8C2B8C9B8C2B8C9B8C20DE056
:10D28000179A117019A9109AB8C9B8C2B8C9B8C20A
:10D29000B8C9B8C2B8C9B8C2C10709D180073546F4
:10D2A000149C139A169B00D4D5E602208543D2E63F
:10D2B000FE20354605401898149C139A169B2906A3
:10D2C00028D0CCE637A231E01691149078780B99EB
:10D2D0004143334808181F386F21C9430D9D7A1800
:10D2E0000378D427D3554378D827D3558378DC27C0
:10D2F000D355002900D170E6C378E027D35510310B
:10D30000001D189FEBE70120404A10E00024002D8B
:10D3100000D087E629B0F0BD80290ED30F20B87267
:10D32000104817998883102020E525A20120014686
:10D3300002F09CFB189829B0F0BD1020402904D3BE
:10D34000B8720849179B998310E5B8720448179979
:10D35000888314200AE5C046A11A01009A1A010028
:10D36000150F0000140B00000108000025642025A3
:10D3700064202564202564202564202564202564FC
:10D380002025642025642025642025640D0A0000E2
:10D390008C4001001DF7FFFFA437010089FBFFFF50
:10D3A000943F01007472785F6D6F646520706172E4
:10D3B000616D65746572206572726F720D0A00008E
:10D3C0004E73666420706172616D6574657220656C
:10D3D00072726F720D0A0000FFFFFFFF01FF000075
:10D3E0005C1E0100FFFFFFFFFF0101FFFF01FF01C6
:10D3F000FFFF01FFFFFFFF01FFFF01FF48240100C6
:10D40000FFFF01FF7C1E0100CC1D0100423701001F
:10D41000002800D10148064908607047C890010201
:10D42000F0B586B0002805D10148006802E0C0468A
:10D43000389401023121C900049141188A791F23CF
:10D440001A40CD79ED06AD0DAA180D7AED066D0CDA
:10D4500052194D7AED062D0B52198D7AED06ED0914
:10D460005219CD7AED06AD0852194D7CED075219CF
:10D47000BD4C22600A7B1A404E7BF606B60DB218F0
:10D480008E7BF606760C9219CE7BF606360B921939
:10D490000E79F606F60992194E79F606B608921933
:10D4A00062604A6AB14D2A40A2608A6A2A40E260FC
:10D4B0002D22D20087183A7E1A4003937E7EF6060C
:10D4C000B60DB218BE7EF606760C9219FE7EF606F2
:10D4D000360B92193E7FF606F60992197E7FF60604
:10D4E000B60892190E7CF60792192261BA7F1A408B
:10D4F0000597FE7FF606B60DB218049BC35CDB06EB
:10D500005B0CD2184B78DB061B0BD2188B78DB0632
:10D51000DB09D218CB78DB069B08D2186261CA6996
:10D520002A40A2610A6A2A40E2618A7C01252A40D7
:10D53000CB7CDB079B0F9A180B7DDB075B0FD218A8
:10D540004B7D9B07DB0ED2188B7DDB079B0ED21821
:10D55000CB7D1B079B0D9A180B7E1B079B0CD218CB
:10D560004B7E5B06DB0A13438A7E520612091A437E
:10D57000CB7E5B075B0813432362CA6A62620A6B55
:10D58000A2624A6BE2628A6B22633922D200835C18
:10D590001E462E4066635E425E41B304AE04744F85
:10D5A0003C68B443E3183B6083185A782A409C785F
:10D5B0002407E40EA2188C8F6401A2186D4C14404D
:10D5C000C98FC905490A0919DA78D207120A8918D8
:10D5D0001A791207120989185A79D207D2088918BC
:10D5E000FB4EB1639968F163997904952940DA7922
:10D5F000D207920F51181A7B5207D20E89185A7B04
:10D60000D206920D51189A7B5207D20C8918DA7BF8
:10D61000D206920B89181A7CD206520A89185A7CB3
:10D62000520792090A43997CC90649085118316486
:10D63000D97C039A11401A7DD206920D51185A7D59
:10D64000D206520C89189A7DD206120B8918DA7DFF
:10D65000D206D20989187164197E0F2421405A7E9E
:10D66000120151189A7E12038918DA7E1207120AE3
:10D6700051181A7F1207120989185A7F1207891840
:10D68000B164997F01942140DA7F1207120E51187C
:10D690003D22D200835C5B075B0D591884186278C9
:10D6A0001207520C8918A278D206120B8918E27858
:10D6B000D206D2098918F164217907220A406179DA
:10D6C000C9008918A2795206920B5118E279920783
:10D6D000120B8918227AD2078A18BF490A60627A27
:10D6E000A37A1B029A18E37A1B04D2184A60E289D3
:10D6F000BA4B13400394228AD2049209D2188A604A
:10D7000003463033598CB64A114002939A8CD205A5
:10D71000D20A51185622825C12068918B14D29602E
:10D72000014656314A788C782402A2188C88640508
:10D730006409A218CC78240712196A60CA880C7A86
:10D74000A407A40BA2184C7A6407E40A1219AA6071
:10D750004989E960492189004118FF22663282180F
:10D7600000921035002207E000300040FFFFFF006C
:10D7700004040040FF3F000084186427E65D03278F
:10D780003E406523E35C9B071B0F9B196626A65D45
:10D79000B607B60EF3186726A65DB601F318DBB21E
:10D7A0006826A65DB607B60DF3186926A65DB6070E
:10D7B000360DF3186A26A65DB607B60CF3186B266D
:10D7C000A65DB607360CF3186C26A65DB607B60B39
:10D7D000F3186D26A65DB607360BF3186E26A65D08
:10D7E000B607B60AF3186F26A65DB607360AF31811
:10D7F0007026A65DB607B609F3187126A65DB607B2
:10D800003609F3187226A65DB607B608F318732614
:10D81000A45DA407E31808C51032802AACD1019A90
:10D82000D243704EB4180B783B404D78AD072D0FA6
:10D83000EB188D78AD07AD0EEB18CD78AD01EB1878
:10D84000DBB20D79AD07AD0DEB184D79AD072D0DA0
:10D85000EB188D79AD07AD0CEB18CD79AD072D0C1C
:10D86000EB180D7AAD07AD0BEB184D7AAD072D0B0C
:10D87000EB188D7AAD07AD0AEB18CD7AAD072D0AFE
:10D88000EB180D7BAD07AD09EB184D7BAD072D09EE
:10D89000EB188D7BAD07AD08EB18CD7BAD07EB1812
:10D8A000A3641031121DBDD1009B19785A7852071C
:10D8B000520D51189A78D207120D8918B164059B40
:10D8C0001968F164D97D5A68120251183165996856
:10D8D000454A0A40998A490589187165D9683D4CBD
:10D8E0002140B16519692140F165029E3178049D9E
:10D8F000294082785207120F5118C2799207920E6E
:10D900008918427A9207920D5118827A9207120D65
:10D910008918C27AD207920C89189A7DD207520CC4
:10D92000891872789207D20B8918B2781207D20A36
:10D930008918F2781207D2098A182C490A60327CB9
:10D94000737C1B071B0D9A18B37C9B069B0BD2188C
:10D95000F37C1B079B0AD218337DDB065B09D218C8
:10D96000737DDB071B09D2184A60B27D2A40C38F42
:10D970005B009A188A60826CCA60C26C22400A619D
:10D98000F27D7F231340328C5204520AD2184A612E
:10D9900002698A614269CA6182690A62C2694A622D
:10D9A000026A8A62426ACA62826A0A63C26A4A6315
:10D9B000039A927CD201121D0A64027A3A40CA6527
:10D9C000808F074A10400866002006B0F0BDC046B0
:10D9D00000300040FFFFFF009C300040FF1F0000B0
:10D9E000FF03000000400040FFFF1F000020004038
:10D9F00004480068806B80080349096849004018A2
:10DA000009307047389401021004004010B52D21F0
:10DA1000C9004118027A032A04D10079002807D0EE
:10DA2000082006E08378DA1E022A05D2032412E0D9
:10DA3000142088601C203DE0012B02D1C8228A609E
:10DA400012E00479042C01D3462404E0032C01D114
:10DA5000322400E014248C605B1E022B04D3022AC3
:10DA600010D24279154B01E04279154B9B181B7877
:10DA7000402B04D0102B06D11423442405E02A2384
:10DA80003E2402E04279342348244B800C80022A51
:10DA900006D0062A08D0052A08D118224C2301E016
:10DAA000142250230B8000E01C224A80C0780428F6
:10DAB00003D1142048806420088010BDA11A010001
:10DAC0009A1A0100134800687047C04610B5104A02
:10DAD000107091700F49002813D05068086104201D
:10DAE00048619078FF2212020B4B1C68944380031C
:10DAF00080B20019186001204007084A1060084AE7
:10DB0000106000200860074901220A6010BDC0466D
:10DB100028940102180400401CE400E080E200E0C8
:10DB200000E100E070000040F0B591B0002801D1A4
:10DB3000C04800688778F91E022913D3012F21D02D
:10DB4000022F3CD11021CA43447821461939914211
:10DB50003DD800970125B94A28462946234601F0B9
:10DB600085FF53E10821CA43447821462139914277
:10DB700018D800970125B14A28462946234601F0C6
:10DB800075FF43E10821CA4344782146093991428F
:10DB900034D800970125A94A28462946234601F092
:10DBA00065FF33E1032F3CD0042F43D1C378012517
:10DBB000042B00D02DE106462A02042343E0012570
:10DBC000A6A2284629463B4601F050FF1EE1C37835
:10DBD0000125052B0AD806462A02284698401B2113
:10DBE000084230D10021052B08462ED0022000909B
:10DBF000914A2846294601F039FF07E10646C378D5
:10DC00000021022B1ED3032B1CD0042B08460A46EE
:10DC10001BD001250095884A2846294601F026FF99
:10DC2000F4E0C3780125032B00D0FAE006462A026F
:10DC3000032308E0012583A2284629463B4601F03C
:10DC400015FFE3E00A46012148020F91592189009E
:10DC50007518FD21490071180291314662313F0566
:10DC6000D219641E1F2727405C013C19144304434A
:10DC700032795207D20C22432B789B065B0BD218C9
:10DC8000B379DB071B0B13436D4D2B60F279032334
:10DC900010931A40737A9B079B0E9A18B37A5B070E
:10DCA000DB0D9A18F37ADB079B0DD218337BDB0769
:10DCB0005B0DD218737B1B075B0CD218AA6032690C
:10DCC000EA6072692A61B2696A61F269AA61326ABC
:10DCD000EA61726A2A62B26A6A620F980870F06A30
:10DCE000A8623F20C4432C353046E4300F903046C4
:10DCF000E5300E903046E6300D903046E7300C901F
:10DD00003046E8300B903046E9300A903046EA3031
:10DD100009903046EB3008903046EC3007903046A2
:10DD2000ED3006903046EE3005903046EF300490EE
:10DD30003046F03003903746F1373046F230F33654
:10DD40000F990A194021525C109B1A400E9B1B1917
:10DD50005B5C9B071B0F9A180D9B1B195B5C9B0759
:10DD60009B0E9A180C9B1B195B5C9B019A18D2B2F4
:10DD70000B9B1B195B5C9B079B0D9A180A9B1B193D
:10DD80005B5C9B071B0D9A18099B1B195B5C9B072F
:10DD90009B0C9A18089B1B195B5C9B071B0C9A1821
:10DDA000079B1B195B5C9B079B0B9A18069B1B1917
:10DDB0005B5C9B071B0B9A18059B1B195B5C9B0705
:10DDC0009B0A9A18049B1B195B5C9B071B0A9A18F9
:10DDD000039B1B195B5C9B079B099A183B195B5CB7
:10DDE0009B071B099A1803195B5C9B079B089A18F1
:10DDF0003319595C8907891802C51034A0D10298DB
:10DE00000078042101430E48C1630025284611B063
:10DE1000F0BD04200090084A2846294601F026FE5D
:10DE2000F4E703200090044A2846294601F01EFE2C
:10DE3000ECE7C04638940102173701005D37010056
:10DE400000100040556E646566696E6564206D65FE
:10DE5000616E205052462025640D0A00496E76619D
:10DE60006C6964206D65616E205052462025640DFA
:10DE70000A0000007047704780B50E490E48024600
:10DE8000083A1268920000D4603142680A43426046
:10DE90000A490A6808239A430A60091F01225204AA
:10DEA0000A600321890402688A430260FBF7F4F9DF
:10DEB00080BDC046200000802800004004020040D1
:10DEC000B0B5032000072D490A6882430125680781
:10DED0001018086000242046FFF7CDFF2046FFF70A
:10DEE000C9FFEFF31080284002D1EFF3108172B622
:10DEF0008021C943224A53680B40536093680B400A
:10DF00009360D3680B40D36013690B40136153696E
:10DF10000B405361002800D162B6B0BD70B50C460D
:10DF200003210907154A13680B4313600122EFF31D
:10DF30001081114002D1EFF3108272B68025EA43BE
:10DF40000F4B5E6816405E609E682E439E60DD68E3
:10DF50001540DD601D6915401D615D6915405D61FD
:10DF6000002900D162B6002802D00120FFF783FF0C
:10DF7000002C02D00120FFF77DFF70BD000400409F
:10DF8000B89501020D4A002907D001290BD10121C2
:10DF9000814010688843106007E0012181401068CB
:10DFA0000843106001E001218140101F02680A430C
:10DFB0000121C907114301607047C0464400004079
:10DFC000032804D840000649085A00B270470020D0
:10DFD00000B27047032802D84000014A115270472E
:10DFE00096D101029E4908707047C04670B58AB04C
:10DFF0000C460546FF20FC30A8490E68315C5920CC
:10E000008000335CB278307808AE069609AE05968B
:10E010000C4E04962126760603960B4E0296012698
:10E0200001960E2600965B1CDBB2F7F79BFF099862
:10E03000F2F750FC28700898F2F74CFC20700AB0F8
:10E0400070BDC0460000204100000443F0B58BB015
:10E050000446457C824800788249002822D000206E
:10E060000880814A1080814B01269E761E830A908B
:10E070007F4800787F4E36786DB205957E4D0495C9
:10E080007E4D03950AAD02957D4D01950096F7F7FB
:10E09000A7FC0A9D112020567A497B4A00F0F2FB2A
:10E0A000064626E000260E806F4A16806F4B012040
:10E0B0009876188309966E4800786E4F3F786DB257
:10E0C00005956D4D04956D4D039509AD02956C4D0B
:10E0D00001950097F7F784FC099D112021567F20B8
:10E0E000C005009001900296664A674B3046F8F7EB
:10E0F000CBFD432001062846F2F760F9F2F7EAFB70
:10E10000089062480078002824D05120800060499F
:10E110004A7D42438D185F480068A8642F46403707
:10E1200050480078B87450480078F8745548007822
:10E13000387555480078787557480078F875504814
:10E140000069F2F7C7FBB87552484069E8644C486B
:10E1500000686864FF20FE3050490968085C392275
:10E16000D2008918022812D303D04E480078012823
:10E170000DD14B480660434800883A4A1080424817
:10E180000088394A108009200790089605E0444825
:10E19000089A02603548C08B07900B780022002B4C
:10E1A00001D0114600E0D1430125002B01D004230A
:10E1B00000E0EB43A67AAD1BEE175B197141656871
:10E1C000AE0F277AAD00ED195641677A3F1FF81759
:10E1D000ED1970414000EE0F80196D00EB184841B9
:10E1E0008001990E4118980127239B02C31A91417F
:10E1F0001D4805881B480088854201D00798421BAE
:10E2000010202056C001194D2D8C032D07D1E46834
:10E21000E5176D0A6419E4150519EC170FE0E468B9
:10E22000E5176D0A6519EC17ED15C6174519744108
:10E2300097B2002F00D03446002F00D00546581B5F
:10E24000A141130409D012B2D2015242D31780184F
:10E250005941089BDA17C01A91410BB0F0BDC04676
:10E26000BA93010260AC01025EAC0102909401021B
:10E27000C5900102C49001024CA201024CA001020F
:10E2800064AC0102AEAC0102ACAC010218A6010202
:10E2900050A30102642000405CAC010238940102EA
:10E2A00058AC0102C0AC0102C10D40028030704781
:10E2B00010B50D4C22463032402000210223F6F7E3
:10E2C00033FB3020205C4007C00F10BD10B5064C5A
:10E2D00022463032402000210223F6F725FB312070
:10E2E000205C0007C00F10BDD49501020120C007BB
:10E2F0001B4908607047C04610B519480068C1073F
:10E3000010D1810711D4410712D4010713D4C106DB
:10E3100014D4810615D4410616D48021084016D0A5
:10E3200031A215E001240FA213E0022411A210E093
:10E33000032414A20DE0042416A20AE0052419A265
:10E3400007E006241CA204E0072421A201E0254ADC
:10E3500004090220032101F089FB204610BDC046BC
:10E360005C000040526573657420627920504F5202
:10E370000D0A0000526573657420627920424F5285
:10E380000D0A000052657365742062792050494E71
:10E390000D0A000052657365742062792057445459
:10E3A0000D0A00005265736574206279204C4F435A
:10E3B0004B55500D0A000000526573657420627958
:10E3C000205357205265626F6F740D0A00000000E1
:10E3D0005265736574206279205359535245510D2B
:10E3E0000A000000262A01005265736574206279D4
:10E3F00020445644440D0A0001218140044A1F284C
:10E4000002D010688843106010680843106070479D
:10E410001C000040F0B583B0029104469949F1F721
:10E4200059FE0546984901942046F1F753FE974955
:10E4300046189749714300956F189649441864210E
:10E440002046F1F747FE3818A108471A924920469E
:10E45000F1F756FE381891494518914F05D46421BB
:10E460003046F1F737FE0C4614E0A6B26421304680
:10E47000F1F730FEB7204000A20701D1002907D1F3
:10E48000884B73430422D341874A934200D3401EF2
:10E490000C4645190098474302980680192001014F
:10E4A0003046F1F717FE2A461F3A284600DB104691
:10E4B000019BFF18B30705D1002C03D01F2D05DAEF
:10E4C0000120C5E01F2D0BDA0120C1E005461D3DEE
:10E4D000034600DB2B461C2808DC02201546B7E06B
:10E4E00000290CD01C21451A0CD50CE019461F3907
:10E4F000184600DB08461F2B1DDA0320A8E01D216B
:10E50000451A00D42846002D08D401461F3902467A
:10E5100000DB0A461F2804DA032099E00220154692
:10E5200096E015461E3D104600DB28461E2A0CDAF2
:10E5300004200D468CE005461E3D024600DB2A46BF
:10E540001E280BDA04200D4682E001461F390246E0
:10E5500000DB0A461F280ADA052079E011461F3938
:10E56000104600DB08461F2A0BDA052070E015462E
:10E570001E3D104600DB28461E2A0CDA06200D46FA
:10E5800066E005461E3D024600DB2A461E280BDAE1
:10E5900006200D465CE001461F39024600DB0A46B4
:10E5A0001F280ADA072053E011461F39104600DB06
:10E5B00008461F2A0BDA07204AE015461F3D13467E
:10E5C00000DB2B461F2A0CDA08200D4640E00546EA
:10E5D0001F3D024600DB2A461F280BDA08200D46A5
:10E5E00036E019461E39184600DB08461E2B0ADAAB
:10E5F00009202DE011461E39104600DB08461E2A70
:10E600000BDA092024E01F28054601DB05461F3DE3
:10E610001F280CDA0A200D461AE01F28054601DBE8
:10E6200005461F3D1F2806DA0A200D4610E01E2D64
:10E6300005DB0C2004E01E2D06DB0C2005E00B2082
:10E640001E2D05DB1E3D03E00B201E2D00DB1E3DB5
:10E65000029EB070681CF070E12001013846F1F7AD
:10E6600039FD3071C0B211494143CC193C212046DB
:10E67000F1F730FD70713B21C94341430819B07176
:10E6800003B0F0BD805101008033E101B20700000A
:10E6900093FEFFFFB107000070FEFFFFA7FA0A001C
:10E6A00080AEFEFF295C8FC20BD7A300F0F1FFFF05
:10E6B000F0B581B00446FFF703FCA08A00280ED015
:10E6C000FFF700FA2749C861274824302CCC2CC01A
:10E6D0002CCC2CC02CCC2CC00020088336E0E08A47
:10E6E000204F3883A1693A8B2048F1F71DFD1E4D5C
:10E6F0002435204629464CC84CC14CC84CC14CC896
:10E700004CC1FFF7DFF9F8611748866AFFF770F927
:10E71000301A78632846FFF799FC06460D461448E0
:10E72000007DFFF74DFC0121B972617CF972F96D32
:10E73000491CF96581B2C90B401800B2C1174010DD
:10E74000301A38678D417D67F4F7BAFC0848426893
:10E750000020014602F094FB0249C8710120887133
:10E7600001B0F0BD68970102E0970102D4D1010227
:10E7700038900102F0B581B0EFF3108072B600203E
:10E780000146FBF7B5FE0446002803D062B62046DA
:10E7900001B0F0BD01273A030025074E2846314657
:10E7A000FBF700FEBB02054A28463146FCF7D8FAC3
:10E7B00062B6204601B0F0BD00E0020456A8010296
:10E7C0000648417B01228A43C272491C4173C179C8
:10E7D000002901D0491EC1717047C04660990102ED
:10E7E00070B514460D4606461120FAF7D3FE2248AE
:10E7F000042101600C4804601E4805608660002EFC
:10E800000DD0FF20000609490A6882430120C00795
:10E8100010180860064808210160064801601A20A7
:10E820000221FFF7AFFB70BDD4D2010200E400E08B
:10E8300080E200E000E100E00C4908607047C0465B
:10E8400010B504460948006860430949F1F758FCCF
:10E8500000190849486008480022026002460C3A44
:10E860004B6813600968016010BDC046D0D2010238
:10E8700040420F000C9001022C100140004800475C
:10E88000C100000080B582B013460A4600900348DC
:10E89000011D0348F8F7A4F902B080BD10D30102AE
:10E8A000849F010210B50C498A1C90420DD2401E73
:10E8B0000D4A50600D4803680B4003218C071B195B
:10E8C000036000209060116010BD04480449E622F6
:10E8D000044B00F06FF8C046FFFFFF00FD29010068
:10E8E000172A0100E329010010E000E020ED00E01C
:10E8F000B0B50120EFF31081014002D1EFF3108297
:10E9000072B6124A1368124C226864688506114870
:10E9100000682840850E5D192923DB006B43002C1D
:10E920001D4606D1002809D11E20684300290AD0BF
:10E93000B0BD121BD218551C0028F5D01D461E2054
:10E9400068430029F4D162B6B0BDC04640DE010282
:10E9500014E000E004ED00E080B50020FBF772F861
:10E96000404280BDB0B586B0104869460A4638C8F6
:10E9700038C238C838C200242046FBF769F803992A
:10E980002046FBF7FFF80198012803D0082400284F
:10E9900004D102E00424002800D104460220FAF742
:10E9A00001FEE0400249086006B0B0BDA81A0100AF
:10E9B00054DE010290B01C4605AB07C3EFF3108094
:10E9C000C00702D1EFF3108072B6EFF310800B9006
:10E9D00068460E907046089010AB0F93CF4F3E1DC7
:10E9E00001200490C50230462946224600F0B8FCBA
:10E9F00000213154EFF303800990EFF308800C906D
:10EA0000EFF309800D90EFF314800A9000F02CFCD6
:10EA10003868012833D80028C14F00D0C14F2A20C0
:10EA2000C1497A69920703D50A783A60401E491CA9
:10EA30000028F6D1B948041D2046F1F7A3FB0028B1
:10EA400007D079698907FAD521783960401E641C9E
:10EA5000F5E70220B5497A69920703D50A783A604A
:10EA6000401E491C0028F6D12A20AF497A69920736
:10EA700003D50A783A60401E491C0028F6D1FFF7FA
:10EA800037FF0346AA4A30462946FDF7C9FE044629
:10EA90003018291B089F3B1F049A9343A5A2FDF73A
:10EAA000BFFE9E490968012966D8001900299C4CBF
:10EAB00000D09C4C00280AD09849091D6269920731
:10EAC00003D50A782260401E491C0028F6D10A208E
:10EAD0009F496269920703D50A782260401E491C4B
:10EAE0000028F6D10598F1F74DFB002809D061699F
:10EAF0008907FAD5059A11782160401E521C0592AB
:10EB0000F3E7022089496269920703D50A782260F7
:10EB1000401E491C0028F6D10A208EA16269920786
:10EB200003D50A782260401E491C0028F6D10698B9
:10EB3000F1F728FB002809D061698907FAD5069A00
:10EB400011782160401E521C0692F3E7022077499B
:10EB50006269920703D50A782260401E491C00288A
:10EB6000F6D10A207EA16269920703D50A78226055
:10EB7000401E491C0028F6D17CA230462946079B3E
:10EB8000FDF74EFE6549096801290E9B1BD8002937
:10EB9000634900D0634900280AD0604A121D4C69BD
:10EBA000A40703D514780C60401E521C0028F6D12F
:10EBB00002205E4A4C69A40703D514780C60401EFD
:10EBC000521C0028F6D16AA230462946FDF728FEDD
:10EBD00004463018291B694A3B46FDF721FE4F4980
:10EBE0000968012911D8001900294D4900D04D4963
:10EBF00000280AD0494A121D4B699B0703D5137898
:10EC00000B60401E521C0028F6D15D4A3046294652
:10EC1000099F3B46FDF704FE0446F800C00FB9000B
:10EC2000C90F7A00D20F0092019102903019291B6E
:10EC3000FB0F544AFDF7F4FD04193019291B3F233B
:10EC40003B40514AFDF7ECFD34490968012911D8D0
:10EC500020180029324900D0324900280AD02F4A12
:10EC6000121D4B699B0703D513780B60401E521C85
:10EC70000028F6D1454A304629460B9BFDF7D0FDCA
:10EC800004463018291B424A0A9BFDF7C9FD234957
:10EC90000968012911D800190029214900D021490A
:10ECA00000280AD01D4A121D4B699B0703D5137813
:10ECB0000B60401E521C0028F6D1364A30462946C9
:10ECC0000C9BFDF7ADFD04463018291B324A0D9B05
:10ECD000FDF7A6FD114909680129114A0DD800194F
:10ECE000002908D00F4A06E05169890703D5317819
:10ECF0001160401E761C0028F6D128490E98091A8A
:10ED0000A94200D32946890800F03AFE2448006849
:10ED1000002800D0804700F045F8C046C0DE010260
:10ED20000090014000A00140572A010081370100F6
:10ED3000402A01000D0A23232320415353455254F6
:10ED4000204020307825303858202323230D0A0016
:10ED50001A2B010046554E4354494F4E3A200000AD
:10ED60004C494E45202020203A2000002564000018
:10ED70000D0A53503D253038580D0A00DF2A010096
:10ED8000F52A0100012B0100E92A01009E2A010059
:10ED9000AD2A0100BC2A0100C72A010000F80202C6
:10EDA000BCDE0102F7480068012811D8002801D014
:10EDB0000B4800E0FC480C210A4A01E0002907D07A
:10EDC00043699B07FAD513780360491E521CF5E787
:10EDD0001E20FFF711FB00BF00BF00BF00BFFAE716
:10EDE00000A001404A2A01008AB00646E448B06605
:10EDF00000F03AFAFFF77CFD0346E248041D0120CB
:10EE00000590C502E04A20462946FDF709FD074660
:10EE100008942018DB4C0995E91BF36C3F220692FD
:10EE20001340DAA2FDF7FCFC2168012910D8C019B3
:10EE30000029DD4900D0DD49002809D0221D4B6999
:10EE40009B0703D513780B60401E521C0028F6D197
:10EE5000F36BD7A2089C2046099D2946FDF7E0FCEC
:10EE60000746291A2018336C069A134007D1D8A2F6
:10EE7000FDF7D6FCC34C2168012907D917E0CEA2C3
:10EE8000FDF7CEFCBF4C2168012910D8C01900291C
:10EE9000C54900D0C549002809D0221D4B699B07F0
:10EEA00003D513780B60401E521C0028F6D10027B2
:10EEB000CBA5B80030580090089809992A463B46DF
:10EEC000FDF7AEFC216801290FD80029B64900D012
:10EED000B649002809D0221D4B699B0703D513783A
:10EEE0000B60401E521C0028F6D17F1C0D2FE0D174
:10EEF000736BBFA2089C2046099D2946FDF790FC34
:10EF0000074620189F4CE91BB36BBC4AFDF788FCF1
:10EF10002168012910D8C0190029A34900D0A349AC
:10EF2000002809D0221D4B699B0703D513780B607D
:10EF3000401E521C0028F6D1336CB14A089C204672
:10EF4000099D2946FDF76CFC0746326CD000C00FC6
:10EF50009100C90F5300DB0F009301910290E0195B
:10EF6000E91BD30FA74AFDF75BFC3246C619A0196F
:10EF7000A91B1546136C069A1340A34AFDF750FCD3
:10EF800080490968012911D880190029864900D0D3
:10EF9000864900280AD07B4A121D4B699B0703D57E
:10EFA00013780B60401E521C0028F6D12E466B6C65
:10EFB000964A089C2046099D2946FDF731FC0746E4
:10EFC0002018E91B0796B36C914AFDF729FC6D4A9E
:10EFD0001168012910D8C0190029734900D073495C
:10EFE000002809D0121D4B699B0703D513780B60CD
:10EFF000401E521C0028F6D10798426E042360215F
:10F000005C2004931A400B4600D003460693002A66
:10F0100000D00846079E33587E4A089C2046099D2A
:10F020002946FDF7FDFB074606983358E019E91B12
:10F03000794AFDF7F5FBC619A019A91B079A536E6B
:10F0400076A2FDF7EDFB4F490968022911D280191C
:10F050000029554900D0554900280AD0494A121DB7
:10F060004B699B0703D513780B60401E521C002888
:10F07000F6D10798C36C06466DA2089C2046099DF0
:10F080002946FDF7CDFB07462018E91B336D6B4A77
:10F09000FDF7C6FBC619A019A91B079F7B6D68A2C7
:10F0A000FDF7BEFB8619A019A91BBB6D67A2FDF772
:10F0B000B7FB344909680129059C11D8801900293A
:10F0C000394900D0394900280AD02E4A121D4B690F
:10F0D0009B0703D513780B60401E521C0028F6D105
:10F0E0000798476B5D4A974237D203208743002633
:10F0F000059CB00039580246049B1A43BA580823AD
:10F100000343FB580C2505437D590091019202935E
:10F1100003953B1808980999514AFDF781FB194955
:10F12000096801290FD800291F4900D01F4900286C
:10F1300009D0089A4B699B0703D513780B60401ED2
:10F14000521C0028F6D11B2E444A06D80798406B63
:10F15000361DB10040189042CBD30798406B111A6E
:10F16000099A914201D8890800E0610200F008FC88
:10F170003C480068002800D08047FFF713FEC046D7
:10F1800022224B4DC0DE0102402A01000D0A0D0A69
:10F1900023232320455843455054494F4E2025648E
:10F1A000202323230D0A00000090014000A001400D
:10F1B00050433D25303858002C20457863657074E5
:10F1C000696F6E4E756D6265723D25640D0A0000B3
:10F1D0002C205468726561644D6F64650D0A0000EF
:10F1E00052252D32643D253038580D0A00000000AC
:10F1F00053503D253038580D0A000000DF2A010029
:10F20000F52A0100012B0100E92A01009E2A0100D4
:10F21000AD2A0100BC2A0100C72A01004558435FFE
:10F2200052455455524E3D253038580D0A000000C5
:10F23000494353523D253038580D0A00D22A010067
:10F240005343523D253038580D0A00004343523D88
:10F25000253038580D0A0D0A0000000000F802029F
:10F26000822A0100BCDE0102F0B583B0344D2C6867
:10F27000012C06D8601E8441204601F037FB00288F
:10F28000FAD10120EFF310810140019102D1EFF397
:10F29000108072B62B48285A2B49695A814245D0B2
:10F2A0002A68002A01D02A4E00E0284E1F23DB02E4
:10F2B0000293284C022A27D205E01046214AA85280
:10F2C00082B2914232D087B2B9420A4600D8621C5B
:10F2D000131A21482B5218040DD0E819001D9FB2B3
:10F2E00001E0002F07D073699B07FAD503783360DC
:10F2F0007F1E401CF5E7A242DFD902981018DDE717
:10F30000304683B299420CD0024680B281420E460A
:10F3100000D8661CA642F3D90298301883B29942ED
:10F32000F2D108496852B01A0B4968520B480021C3
:10F3300029540198002800D162B603B0F0BDC04640
:10F34000C0DE01020A080000080800000090014029
:10F3500000A00140FF0700000C0800000F0800009B
:10F36000F0B58DB00793174600240C9409AA13C278
:10F3700015E006986849F1F721F8F1F7ABFAC117E3
:10F38000401848406549F0F7A5FE009509A80622F7
:10F390003346F9F7BBFABDE0002C00D5BEE1387862
:10F3A0007F1C25280DD0002800D1B7E10B9A511CF5
:10F3B0000A9B9942F0D8099B9854641C0C940B91B9
:10F3C000EAE708940025397823390D2914D801205B
:10F3D0007944097949008F44090F0F0F0F0F0F0F60
:10F3E0000B0F060F0F0D05437F1CECE70820FAE713
:10F3F0000420F8E70220F6E7387801463039002487
:10F40000092902D9264639460BE000260A21714314
:10F410000E18303E791C78780246303A0A2A0F4698
:10F42000F4D32E2817D14A1C4878014630390929CF
:10F4300005D911464F1C2538532811D96AE00024FC
:10F440000A2161430C18303C511C50780246303A76
:10F450000A2A0A46F4D34F1C2538532800D959E00C
:10F460004000C0467844808840008744A000530094
:10F4700053005300530053005300530053005300F4
:10F4800053005300530053005300530053005300E4
:10F4900053005300530053005300530053005300D4
:10F4A00053005300530053005300530053006000B7
:10F4B00053005300530053005300530053005300B4
:10F4C00053005300530053005300530053005300A4
:10F4D000530098005300530053005300530053004F
:10F4E0005300530053005300AD00B60053006000BA
:10F4F0005300590053005300530059005300530068
:10F500005300DE0053005300BD005300D3005300EE
:10F51000530098000C9C3FE70024744940420F00C0
:10F52000791C38780F4625385328F3D898E707997F
:10F53000C91D07208143086807914968F1F730FA2F
:10F5400000210690F1F764F900280BD10B99481CB3
:10F550000A9A904206D8099A2D2353540899491CB7
:10F560000C910B900798083007900698F1F7B2F9C4
:10F570000095C2178118514009A822463346F9F771
:10F58000C5F90B98411C0A9A914200D9F1E6099AF3
:10F590002E2313540B910C98401C0C90E9E607980D
:10F5A00002C807900096019509A8102239E00B982F
:10F5B000411C0A9A9142ADD8099A252313540B9104
:10F5C0000C98401C0C90A5E70B9A511C079C201D21
:10F5D0000A9B994239D907909CE7079802C807907F
:10F5E000009509A82246D3E6079901C90791099910
:10F5F0000A9A089E02E0401C002E8BD40378002B50
:10F6000088D00B9D6C1C9442F5D84B55761C0C96FB
:10F610000B94F0E7079802C807900096019509A897
:10F620000A222346F9F710FA74E7079B10CB102C37
:10F63000079308D300202146401C0A09FF291146E0
:10F64000FAD806280AD8082009E02368099CA354A0
:10F65000089A521C0C920B9107905BE7401C069095
:10F6600009230C980B9D099905910A9E04940DE0BD
:10F67000202104463046059E715506462046049CCE
:10F68000401C15460146089100290AD45B1E0699C4
:10F69000994206D26A1CB242EAD908990891002917
:10F6A000F4D50C900B950898002800D532E7012678
:10F6B000082501E06D1E3601022DFBD220463146A1
:10F6C000F0F708FD0F28F6D80C98059009980390DC
:10F6D0000A9806900B9D20463146F0F7FBFC691C0A
:10F6E000069A914204D90899089100290CD511E095
:10F6F0000C4A125C039B5A55089A521C0D460592FF
:10F7000011460891002905D47043241A3009102E9F
:10F710000646E0D205980C900B95FBE620460DB00E
:10F72000F0BDC0469C1D010070B588B000220328C2
:10F7300003D9D243104608B070BD7F4CC34D2A5147
:10F740000F4B104EEE5081231E010123AB55286054
:10F750002C1962600128EDD80793002206920592C9
:10F76000049203230393029201920091411E884167
:10F77000694600F0EBFC0246104608B070BDC0467A
:10F7800004080000FFC0FFC0F0B583B00C460023A2
:10F79000D943012C56DB074602910126EFF3108571
:10F7A000354002D1EFF3108072B65849584A505C88
:10F7B000002800D0A3E056545E48115A5E48105A03
:10F7C0000196F202161A814240D832465218A242DD
:10F7D00040DB00930295A642354600DB25464C49A6
:10F7E0000818001D39462A46F0F79EFCA642484EEE
:10F7F00004DA7919621B301DF0F796FC4E48305A36
:10F80000001981B24D4A914201D94D494018029DDB
:10F81000009B4949705230464A4E805D002865D1B0
:10F82000EFF310850198054002D1EFF3108072B616
:10F83000374A4048115A4048105A884232D142480B
:10F8400013524FE00C46204603B0F0BD424252181E
:10F85000A242BEDA3B4A2E4EB25C002A0CD03A4A93
:10F86000B25A51188AB2354CA242284C029F01D993
:10F87000334A8918304A02E0244C2F4A029F3355FC
:10F88000B152421A89B2884202D22C488018421CD6
:10F8900093B22F4801212FA200F0E8F83C46002D3A
:10F8A000D1D128E0019F9755884201D82348401CB8
:10F8B000421A90B2800A01D0019882022248144F65
:10F8C0003A52386801280DD8431E9841104B5918F8
:10F8D000091D92B21D4B00F04FFE009B002801D085
:10F8E0000B488355002D029D00D162B60748084998
:10F8F0000B54002DA7D162B6204603B0F0BD2120E5
:10F900000201044804A108A3FFF754F80E08000000
:10F91000C0DE0102962B010074726163655F6F7532
:10F9200074707574000000005452414345204255E4
:10F93000535900000A08000008080000FF070000F3
:10F9400000F8FFFF0F0800000C08000099FB000002
:10F9500002FF00000D0A54726163652062756666DD
:10F9600065722069732066756C6C2C206469736302
:10F97000617264732025752062797465730D0A00C5
:10F98000F0B587B0054600260696059604960396C0
:10F990000296800701D007B0F0BD019102A81421A2
:10F9A00026A2FCF73DFF29490968012911D8002941
:10F9B000274900D0274900280BD002AA01E00028DF
:10F9C00007D04B699B07FAD513780B60401E521C79
:10F9D000F5E701990029DED0204C3746B8002B58B6
:10F9E000D80724D0581EA04204D31B4818181C4A1C
:10F9F00090421CD802A814211AA2FCF711FF134947
:10FA00000968012911D80029114900D0114900289D
:10FA10000BD002AA01E0002807D04B699B07FAD55A
:10FA200013780B60401E521CF5E7761C01997F1C71
:10FA30008F42B0D2322ED1D3ADE7C0460D0A42611B
:10FA4000636B74726163653A200D0A00C0DE0102C7
:10FA50000090014000A00140FFFFFFFCFFFF0200FB
:10FA6000FEFF0100253038580D0A000081B0F0B5C6
:10FA7000C4B00E4607464993812000012F49085C17
:10FA8000002845D002920120050204A82946F0F77B
:10FA900064FBFCB20021C8430C2C3AD8721E032A26
:10FAA00037D82748005DB042084632D3F80535D52F
:10FAB0000021B8050DD404A801904018691AA200CD
:10FAC00022A39B582E4AFCF7ABFE0198F0F75AFB95
:10FAD000014678050ED404AF7818691AB20029A33C
:10FAE000D218121F1368264AFCF79AFE3846F0F720
:10FAF00049FB0146029A04AE70180C46691A49ABDC
:10FB00000393FFF72DFC01193046FFF73DFE00E09F
:10FB1000002044B0F0BC02BC01B00847FEF7E8FE8C
:10FB2000034604A8019007A22946FCF779FE019834
:10FB3000F0F728FB0146B805BDD5CAE7C0DE0102D3
:10FB40006443010025313075207C20003A2B0100F0
:10FB5000902B01008A2B0100692B0100342B01003E
:10FB6000552B0100832B01007C2B0100772B01001A
:10FB70002D2B0100402B0100502B0100252B0100F3
:10FB8000D83301006F2B01005B2B0100622B0100B9
:10FB9000462B010000000000F0B581B00B460120AB
:10FBA000EFF31084044002D1EFF3108172B6990F85
:10FBB00007D0022001212DA2FFF758FF002C3DD1D4
:10FBC00041E02249224D00276F54224AAB5A224A73
:10FBD000AE5AF3189EB2F60A01D0204E9B19AB52D2
:10FBE000EFF31086064002D1EFF3108372B6AA5AE3
:10FBF0001C4BEB5A934202D116482F521AE068541C
:10FC0000934201D8164B5B1C9B1A99B2890A00D00B
:10FC1000830210482B52286801280BD8411E8841C6
:10FC2000A918091D9AB2104B00F0A6FC002801D0BB
:10FC300006482F54002E03D0002C04D001B0F0BD94
:10FC400062B6002CFAD162B601B0F0BD0F08000018
:10FC5000C0DE01020C0800000A08000000F8FFFFE7
:10FC6000FF0700000808000099FB000055415254AE
:10FC7000204572726F722025780D0A0010B5044677
:10FC8000FEF71EF9A08A002800D010BDFDF71AFF6C
:10FC900003498862C861086E401C086610BDC046F2
:10FCA0006897010210B5012400212046FBF7EEFC05
:10FCB0000549204600F04AFAA2020D490D4B2046A4
:10FCC00000F018FB10BDC046D094010210B501240D
:10FCD00004212046FBF7DAFC07212046F9F7A6FAB3
:10FCE000A2020349034B204600F004FB10BDC046AE
:10FCF0000CCD01022D05010070B5012801D90120AC
:10FD000070BD48224243734B9C58A5691F218D4307
:10FD1000A5610625A5600F2525629C18A27C002AF6
:10FD200005D1627C002A02D1227C002A14D06368AB
:10FD3000002B11D4251D0B40012216469E400C4B72
:10FD40001E60BFF34F8FBFF36F8F2B68002B03D460
:10FD50000B409A4007490A60002803D0012804D1CB
:10FD6000092000E00820F9F70DFC0020A06170BD1B
:10FD700080E100E080E200E0F0B585B00D46027859
:10FD8000E348C368934219D0446D944216D0836807
:10FD9000934203D0016D914200D07FE09B1A591E1F
:10FDA0008B41049348215943032D46D14418E169FE
:10FDB00000294ED01C34002020606DE09B1A5A1E92
:10FDC00093410493032D1AD1039548225A43841872
:10FDD000A26B0121EFF310850D4002D1EFF31087E4
:10FDE00072B6A7691026B743A761A669002E01D194
:10FDF00018342160002D00D162B6039D0CE048212B
:10FE00005943421891691832302902D011681029DB
:10FE10004CD1802111600022482159434018002113
:10FE2000816301628162243000210160002A33D0A5
:10FE300004A82946904705B0F0BD421891691832D0
:10FE4000302902D01168202939D180211160002287
:10FE500016E00395E26B0126EFF31085354002D1E1
:10FE6000EFF3108172B6A1692027B943A161A1699E
:10FE7000002901D118342660002D00D162B6039DFF
:10FE80004821594340180021C163C16241633030A9
:10FE900000210160002ACBD105B0F0BD00920E4ACE
:10FEA0002E329C480D490E4BFEF784FD10680093DE
:10FEB000019098480949084A0A4BFEF77BFD1068F3
:10FEC00000930190044A243292480449054BFEF7FE
:10FED00071FDC046F0940102B1020000122C010035
:10FEE000E72B0100CB2B0100F0B585B00490482131
:10FEF0000A464243864B9C58E6690F2535409A18BE
:10FF0000167C002E31D04F2040026169014200D1A1
:10FF100085E0A06904218843A061022020620120BD
:10FF200081076918D161D36BEFF31084044002D1CB
:10FF3000EFF3108572B695692026B54395619569F2
:10FF4000002D00D173E010463C30002C00D162B689
:10FF500000240460D4625463303200201060002B0F
:10FF600063D004A8984705B0F0BD0C2D5DD8C046FD
:10FF70007D442D796D00AF4467586B580658A163D6
:10FF80005858585806009569202D04D01546183544
:10FF90002D68302D49D1156B566B3432AE4217D2D5
:10FFA0006669360714D5646815686E1C1660484388
:10FFB0001818C06A445504980C4644431A19156B26
:10FFC000566B3432AE4203D21C5966693607EAD406
:10FFD0001268AA4229D14143585882690524A24394
:10FFE00082615A18D36B0121EFF31080084002D1CF
:10FFF000EFF3108472B694692025AC439461946940
:020000040001F9
:10000000002C02D114461834216014463C340028D8
:1000100000D162B600212160D16251639CE70C2DB2
:1000200000D176E7012D00D173E705B0F0BD15468C
:100030001835286010463C30002C00D187E787E750
:100040000420206205B0F0BD0120206205B0F0BDA3
:1000500008252562164618369569102D02D0356898
:10006000302D4BD10396566A15462835976AB7420C
:1000700028D1A06902218843A061936B0121EFF38D
:100080001080084002D1EFF3108472B6039E3468EA
:100090001027BC4334603468002C00D13160144612
:1000A0003834002800D162B6002121602960116235
:1000B000243200201060002BB7D052E702202062CB
:1000C00005B0F0BD2A68B242AFD262699207ACD5E2
:1000D0002A68561C2E6048431818006A805C20600D
:1000E00004980A4642439D18AC6A6E6AB4429CD298
:1000F00028359C5862699207EAD496E731680090E7
:100100000191044804A1094A09A3FEF753FCC04623
:10011000F0940102B12B0100756172745F69727114
:100120005F68616E646C6572000000003D03000052
:100130005561727420256420737461746520676F43
:1001400065732077726F6E6720256400F0B585B007
:100150000E460546022804D3002E02D1012005B028
:10016000F0BD002D03D0012D08D1092400E00824A2
:100170002046F9F70FFA2046FEF73EF94821694379
:10018000E74A505883691F240294A34383610623DE
:1001900083600F230193036257180023BB62BB6384
:1001A000FB633B627B62FB623B63317F3974727F2E
:1001B0007A74B27FBA7404937B637368B268F4682C
:1001C000920022435B1E032B0ED8C0467B441B7952
:1001D0005B009F4401050307082304E0282302E095
:1001E000182300E038231A43C260C907090F726957
:1001F0009201D2B28918B2699207920E8918491CED
:10020000816079613169012901D122210161012DCA
:100210005CD831680E2959D2384612300390032435
:10022000002D01D0204600E004204C432D490E193A
:10023000B178F9F73FFA3968CA6880251046284333
:10024000C8602848005D73781B021818C862AA436A
:10025000CA60F9F7C3FA03980078002809D1384634
:1002600011300078002804D138461030007800287A
:1002700027D07868002815D4032102468A431B49F9
:1002800053588407E40EFF26A640B343A5401D4300
:1002900055500299014001208840A2490860144944
:1002A00008600EE08107C90EFF228A40019C0440CD
:1002B000083C032084430C48235893438D401D433E
:1002C00025500120B861049805B0F0BD02480349EB
:1002D000DA22034BFEF76EFBB12B0100242C010048
:1002E000012C0100301B01001CED00E000E400E0E7
:1002F00000E100E0F0B58FB00E900125002900D19B
:100300004BE0039304910592002A00D145E00121BE
:10031000EFF3108201910A4002D1EFF3108172B61F
:100320004827029747437E49CE19B5690023302DEF
:1003300023D831461831C0467D442D796D00AF4435
:100340002024262626262626262626262626262655
:100350005E26262626262626262626262626262605
:10036000182626262626262626262626262626263B
:1003700018000223002A0CD00CE0402D01D0802D63
:1003800005D10123002A04D004E020240C60002AB7
:1003900000D162B61D46002B02D028460FB0F0BD3A
:1003A000002575630399F1630499F162059931633E
:1003B0005B4CE35959691322D202114205D0062140
:1003C00099600F21196271699960317C00290CD004
:1003D000F56109950895079506950D950B950221F0
:1003E0000A91012810D017200FE0717C9A6900292A
:1003F0002CD0952002439A6128460FB0F0BD3024DE
:100400000C60002AC5D0C5E71920049F0C907068C5
:10041000002805D41F21084001998140414801600E
:1004200014209861B06806A9F9F748FA0E98029965
:1004300041436018806861583B4A0092091D3A4662
:10044000059BF9F7ABFA28460FB0F0BD343611061C
:1004500002D580218A439A6131680025059A91422C
:100460002DD205955D694F214A0215421BD1E90540
:1004700002D4029CF24F0AE0596833685C1C346075
:10048000029C6043EE4F3818C06AC1540E98214652
:1004900041437E18736B346BA34238D234367B5899
:1004A0005D691542E3D002211962019EB10729431B
:1004B0003546E34CEFF31082324006D008E029467F
:1004C000019EEFF31082324002D1EFF3108372B637
:1004D000029B4343E01883692024A343836183691B
:1004E000002B05D0002A08D0C26B002A0AD154E79D
:1004F000034618331E60002AF6D162B6C26B002A8A
:1005000000D14AE70EA8904728460FB0F0BD294613
:10051000059D019E3C46EFF310823240D5D0D7E7CF
:10052000F094010280E200E079FD000080B5012036
:1005300082020249024BFFF7DDFE80BD0CCD0102B5
:100540002D050100B0B582B079208400E54D285D0D
:1005500001A90870652080002818F3F765F92F209D
:10056000C000285829190122024BFFF7C3FE02B030
:10057000B0BDC04645050100F0B591B01090012610
:10058000002900D19BE003930591002A00D196E059
:1005900007900121EFF310800291084002D1EFF3A0
:1005A000108172B604924823069307994B43D649AB
:1005B000C9188D690026302D6ED80C461834AD0050
:1005C000374602A675593E46AF46C046A106010011
:1005D000A9060100AD060100AD060100AD0601004F
:1005E000AD060100AD060100AD060100AD0601003B
:1005F000AD060100AD060100AD060100AD0601002B
:10060000AD060100AD060100AD0601009106010036
:10061000AD060100AD060100AD060100AD0601000A
:10062000AD060100AD060100AD060100AD060100FA
:10063000AD060100AD060100AD060100AD060100EA
:10064000AD060100AD060100AD0601003F07010047
:10065000AD060100AD060100AD060100AD060100CA
:10066000AD060100AD060100AD060100AD060100BA
:10067000AD060100AD060100AD060100AD060100AA
:10068000AD060100AD060100AD06010091060100B6
:10069000022600280CD00CE0402D01D0802D05D181
:1006A0000126002804D004E010252560002800D190
:1006B00062B6002E069D944F049C079802D03046E7
:1006C00011B0F0BD00268E62039A8A63059A0A6211
:1006D0004C620A7C002A0BD00C960B960A9609965F
:1006E00008960E9602220D9201282DD018202CE09B
:1006F0008A7C2831002A3BD00A68A24216D22B46B7
:100700004343FA585469A40710D50868441C0C6088
:10071000F918096A085C10601098294641437A1854
:1007200011462831936A526A9342E8D34543785977
:10073000816982220A438261304611B0F0BD3025C2
:1007400025600028B4D0B4E71A200F90C86808A923
:10075000F9F7B4F8109845437A597819C0683949BF
:10076000009105992346F9F719F9304611B0F0BD0B
:10077000FB589A69140602D58024A2439A610A683C
:100780000026049882422ED25D694F225202154201
:1007900007980AD002211962029EB10729431FE07F
:1007A00028315D6915423E46F4D137465C69A4079D
:1007B00002D40699544E0AE00C68661C0E60069935
:1007C0004843514E3018006A005D1860109841434C
:1007D000735871188C6A4E6AB442E1D329463E467A
:1007E000069D494F01E0314607985A6A002AFCD11C
:1007F000EFF31082029B1A4002D1EFF3108372B61E
:100800004543781983691024A34383618369002BCE
:1008100005D0002A09D0826B002A0BD14FE703468E
:100820001833029C1C60002AF5D162B6826B002A44
:1008300000D144E710A89047304611B0F0BDC04643
:10084000F094010279FD0000B0B5264900684A68BD
:10085000824202D10D1D002016E080228A58824279
:1008600003D10D46803501200EE0FC228A588242D9
:1008700003D10D46FC35022006E02F22D2008B5812
:1008800083422ED18D1803207C2242438C18A0680D
:10089000012814D0002824D140342046F3F7B3FBBC
:1008A00001462046F3F785FB2046F3F7ACFB002812
:1008B00017D006C828680C4BFFF75EFEB0BD403469
:1008C0002046F3F7A0FB01462046F3F772FB2046D3
:1008D000F3F799FB002804D006C82868024BFFF7FD
:1008E0004BFEB0BD84BD01024908010048214143CF
:1008F000054842189269D20601D40020704740583A
:100900004169012008407047F094010280B5114808
:100910000078C00110490978890101430F48007827
:10092000400108430E490978090101430D48007848
:10093000C00008430C490978890001430B4800783E
:10094000400008430A4909780143C8B2F4F7C6F8E1
:1009500080BDC046D29E010272960102219401021E
:10096000D4E60102C1AC0102D39E0102D2D1010240
:10097000C6AC0102F0B583B0F3F742F9204CE16B4D
:1009800088423AD0F3F73CF9E0636078002828D039
:100990001C4B32331C4E083600211C4F05E0761CE0
:1009A000401E9B1C3F1D002819D035786A1C3270F0
:1009B000132DF4D83C6801948CB200940291A100EC
:1009C000124D019C6C501049009C09191D880A7237
:1009D00061000C4A51184D860299491CDFE7084C0A
:1009E00000E000216170608A411C61820848808AB1
:1009F00089B2814201D9401C608203B0F0BDC0467B
:100A0000689701025A980102E097010258DE01023C
:100A100056A80102F0B587B0014601270225052836
:100A20003A4600D02A4600200929014600D0114646
:100A3000C900374A54180E210591615EFDF7CAFAC4
:100A40001026A15F3846FDF7C5FA1227E15F284658
:100A5000FDF7C0FA06951425615F03200490FDF7A9
:100A6000B9FA0598235EA05FE15F625F00AD07C53C
:100A700028A2069F3846049D2946FEF7F7FF204628
:100A8000263004263146FBF777FF2620235E2820F8
:100A9000205E2A21615E2C22A25E009001910292CA
:100AA00024A238462946FEF7E1FF27463E3738465E
:100AB0003146FBF77FFF3E20235E06983C5EB95F20
:100AC0000622BA5E00940191029221A207462E46A8
:100AD0002946FEF7CBFF56240D4D285FFBF75EFF3E
:100AE0002B5F2C4621A2384631463546FEF7BEFF25
:100AF000264658363046FBF73DFF5820235EF05F10
:100B000000901FA238462946FEF7B0FF07B0F0BD9F
:100B1000EC9F0102546F4620616E742064656C6125
:100B200079732025642025642025642025640D0A1E
:100B30000000000050446F412064656C61797320AF
:100B400025642025642025642025640D0A0000000A
:100B500050446F41206761696E73202564202564CD
:100B60002025642025640D0A0000000050446F41D8
:100B700020616E742073706163652025640D0A0026
:100B800050446F4120616E676C65206F66667365C7
:100B900074732025642025640D0A0000F0B587B029
:100BA00015467A4B1A680F24A2432F783A431A60ED
:100BB000774C23462C3B774A1A6004900346224622
:100BC000283A12681207FAD5734E092F029306D9F4
:100BD000754A326072600C2F09D175480FE0042FFE
:100BE00007D9704A3260704A7260092F06D3714883
:100BF00005E06A4830607060694800E06B486E4A02
:100C00001060EB7AFF2B039102D10020B0620AE062
:100C100003210B406948C05C40220243B2620220BB
:100C2000674AFEF723FF029F0021384605952A46B2
:100C30000B46FBF719FF06460225032161A2284651
:100C400001913346FEF712FF06963046FCF7E0FBB3
:100C500001210498009108402CD13D4033D16049D6
:100C600000283AD1002D1ED06548A062E0622063C2
:100C700060636448606264480860152085046E1CE7
:100C80008E608D60642420460F46F8F7A7FD3E6015
:100C90003D602046F8F7A2FD281D386003215BA2C5
:100CA0004E48FEF7E3FE0598007BFAF7B5FF06987D
:100CB00007B0F0BD2E4605460698FCF735FF2846DE
:100CC00035463D40CBD02E4605460698FCF7A8FB9E
:100CD0002846354642490028C4D042480861424867
:100CE0004861424888611520C86141480168402236
:100CF0000A43026007210803274B5A698243009880
:100D00004003101858610522039842432A4803689B
:100D10009818334E766B47780F40995C0907490E57
:100D2000C919CA03334B33409A18C9015118324AC2
:100D300089182B4A51632A49896B3822914382785A
:100D40005207920E891804220A4325498A63124BDE
:100D500019690279019E3240C0784007C00E8018A0
:100D60001F2291430818186155204003411C21603F
:100D700020606420F8F732FD204A18483146039B72
:100D8000FEF774FE1649002D8DD06DE70404004077
:100D90002C60004000040080000600400F040F0497
:100DA000B92501000304030400040004EA2601003D
:100DB000882401001B2801003C9401024C290100F9
:100DC000502C010050485920706172616D7320737E
:100DD00065747320253038780D0A00000208000081
:100DE0009060004012A83E009DD79B5AD579BD491E
:100DF000340200403F0080FF40400000322C0100E0
:100E00002008820002D50F00020255007577625F4C
:100E100072785F696E69740D0A000000F0B581B0E8
:100E20001820FDF7E9FA1920FDF7E6FA002420461C
:100E30002146F8F75FF820462146FAF771FE0126B1
:100E400003257F23304629462A46FAF77BFF3046A2
:100E5000FBF716F902273846FBF7E6FD3046314628
:100E6000FCF734FE03A238462946FEF7FFFD204674
:100E700001B0F0BD7577625F6F70656E0D0A00009E
:100E8000F0B581B01646009104460020012739468E
:100E9000FDF744F8EFF310853D4002D1EFF31080E9
:100EA00072B62720400170430A21EFF713F902467A
:100EB000002C02D00020009901E002200021FBF765
:100EC000E3F80446FBF7AAF9002D00D162B62046EC
:100ED00001B0F0BDF0B581B01D460E460446022AB1
:100EE00009D1012738463946FDF718F80096002247
:100EF000384629460FE0174601200021FDF70EF87D
:100F0000012F04D1009600202946024603E00096F6
:100F1000022000210A462346FBF798F90446FBF716
:100F20007DF9204601B0F0BD70B5002801D0012048
:100F300070BD0325A9020F4802680F4B53500024CF
:100F40009460012253030D4E3360BFF34F8FBFF304
:100F50006F8F0B4E336003685A50847204811020E7
:100F6000F8F710FB022007A22946FEF77FFD204676
:100F700070BDC0468095010251E5CC1A80E100E0C9
:100F800080E200E057445420636C6F73650D0A00E3
:100F90000FB47CB50C0009AD01D0611E00E000214A
:100FA00001910090074B6A462946089800F026F9FF
:100FB000002C02D0009A002111707CBC08BC04B047
:100FC00018470000351901000FB410B504A9074BEC
:100FD00002AA039800F012F9044602A9002000F0CA
:100FE000B4FC204610BC08BC04B018474B190100E3
:100FF0007CB51D4616460C0001D0611E00E00021A4
:1010000001910090054B6A462946304600F0F6F8FB
:10101000002C02D0009A002111707CBD351901000E
:101020002021020C01D010211046020A01D01046E6
:101030000839020901D01046091F820801D0104664
:10104000891E420801D0881E7047081A70470000A8
:10105000004870470890010202E008C8121F08C14A
:10106000002AFAD170477047002001E001C1121F29
:10107000002AFBD170470000F0B51FB486B0099874
:10108000089A030D0021024314D05148514A181800
:10109000504305141198012810981AD0281A401CA2
:1010A00000264D4F4D49009601910490002812DA18
:1010B000444211E01198012449A3012801D110985C
:1010C000C1430698119A84600360C26041600BB00E
:1010D000F0BD4042E4E70446210500203F4A001CE1
:1010E00051410391029012E0E00707D032463B469F
:1010F00001990098EFF790FA0191009032463B4633
:1011000010461946EFF788FA06460F466410002C81
:10111000EAD10498039B0028029A0999089806DAF4
:10112000EFF77AFA019B009AEFF776FA05E0EFF70E
:10113000DBFA019B009AEFF7D7FA04460E4600222D
:10114000284BEFF737FE03D80020C043014607E0E5
:101150000022254B20463146EFF7ACF9EFF70AFEA7
:10116000102409E0002C0ADB0A220023EFF734FCEC
:10117000079B30321A55641E02460A43F2D11122EF
:10118000641C079B121B1C19119B012B03D001230C
:1011900008430ED10AE0084304D01120109000202B
:1011A000119077E71098151A6D1E0BE01098824287
:1011B00002DD00236D1C03E0824201DA00236D1E74
:1011C000002BEED0069811998260C16030C07EE796
:1011D00001FCFFFF104D0000000014400000F03F34
:1011E000300000000000F0430000E03F30380A28E3
:1011F00001D201207047002070470000FFB597B072
:101200000646002518E2252877D100242746FD4907
:10121000049400E00443761C32780120203A904088
:101220000842F7D130782A280ED0022230780146C1
:101230003039092916D804990A23594330394018FE
:101240001443761C0490F1E7189802C80491189092
:10125000002904DA0120400304434842049002209C
:101260000443761C30782E2814D10420044370786F
:10127000761C2A2809D11898761C80C8189009E095
:101280000A214F43303FC719761C30780146303968
:101290000929F5D930786C2810D006DC4C281AD0F2
:1012A00068280ED06A2817D104E0742813D07A2851
:1012B00012D110E00120400504430CE00121090592
:1012C00001E0032109050C437178814203D101201B
:1012D00000052418761C761C3078119066280BD0F7
:1012E00013DC58287DD009DC00287BD04528F6D0B7
:1012F0004628F4D047281AD1A5E118E0632835D054
:10130000642870D0652812D19DE170286CD008DC6B
:101310006728F1D069287BD06E280DD06F2806D1C0
:10132000BAE073282ED0752871D0782859D01A9A2F
:10133000199990476D1C7EE16002400F022809D088
:1013400003280DD00428189801680DD00D60001DE9
:10135000189070E11898EA1701680D604A60F6E786
:10136000189801680D80F2E70D70F0E718986A464A
:1013700001781172001D18900020507202A8009090
:10138000012005E0189802C8189000200091C04381
:1013900061070DD5002101E00199491C0191B94275
:1013A00012DA8142F8DB009A515C0029F4D10BE09B
:1013B000002101E00199491C01918142FADB019A67
:1013C0000099895C0029F5D1019904981A9B471A64
:1013D00021463846199A00F097FA019940194518A4
:1013E0000BE04FE02CE113E04EE00098009900780C
:1013F000491C00911A9A199990470198401E019032
:10140000401CF2D1214638461A9B199A10E137E068
:101410000A200021009001916002410F022907D0AB
:10142000189A01CA1892C2179446032908D00AE0F4
:101430001898C01DC108C90005C91891944607E055
:1014400000B2C2179446042902D140B2C1178C469B
:1014500000226146944506DA0A4600214042914145
:101460008C462D2102E0210504D52B216A461173FB
:10147000012103E0E10701D02021F7E7029155E0C7
:101480000A200AE0102008E010200090002104202B
:1014900004430191082703E00820002101910090F6
:1014A0006002410F022907D0189A01CA189200223F
:1014B0009446032908D008E01898C01DC108C90047
:1014C00005C91891944603E080B2042900D1C0B246
:1014D00000210291210729D51199702906D0009A7F
:1014E0001021019B4A401A4305D00EE040216A4674
:1014F0001173012108E06146014306D030216A469C
:1015000011731199517302210291009A0821019BD4
:101510004A401A430AD16146014301D1610705D50A
:1015200030216A46117301217F1E029111995829B9
:1015300004D035A10E910DA90D910DE037A1F9E769
:101540006146019B009AEFF747FA0E9B8C469B5C25
:101550000D9A521E0D92137061460143F0D10D9801
:1015600005A9081A20300190600703D50120000466
:10157000844300E001270198874201DD381A00E02A
:101580000020019900904118029809180498401A07
:101590000490E00306D421461A9B199A049800F09F
:1015A000B3F94519002706E003A81A9AC05D1999F6
:1015B00090476D1C7F1C02988742F5DBE0030CD539
:1015C00021461A9B199A049800F09EF9451904E0E7
:1015D0001A9A3020199990476D1C0099481E009066
:1015E0000029F5DC08E00D980D990078491C0D9153
:1015F0001A9A199990476D1C0199481E019000296B
:10160000F1DC63E1092801003031323334353637FB
:10161000383961626364656600000000303132333E
:1016200034353637383941424344454600000000DE
:1016300000F05AF94519761C3078002800D0E2E510
:1016400028461BB0F0BD600700D406271898C01DBF
:10165000C108C90048680A680831C30FDB07189140
:10166000190001D09CA108E0210501D59BA104E04F
:10167000E10701D09AA100E09AA1430011985B080C
:10168000109165280CD006DC452809D046281DD0CD
:10169000472841D141E0662818D067283CD13CE07A
:1016A0000021112F01DB112000E0781C0191009036
:1016B00008A911A8FFF7E0FC139905910021119AE0
:1016C00015927F1C12980197009150E00120C007ED
:1016D00003900120019008A9009711A8FFF7CCFC06
:1016E000139A149905920022119B00921298159357
:1016F000059A0192002901D0104602E0791C401899
:101700000190381A01D5019804E04042401E009033
:10171000781C0190C01B029043E0012F00DA0127E2
:101720000021112F01DD112000E0384601910090C9
:1017300008A911A8FFF7A0FC13990591119A00219F
:10174000129815920091019721070CD40599B9427E
:1017500001DB019900E00191012904DD159A491E80
:10176000515C302906D0B84201DA011D05DA0121A9
:10177000029115E00199491EEDE7002805DC00996A
:10178000411800910199091A03E0019A411C914204
:1017900000DD01910099401A401C02900120C00711
:1017A0000390200706D402990198814202DB0020B1
:1017B000C043029000206946C87707AF0121039813
:1017C0000337C907884224D0022011902B201290A1
:1017D000039800280CDA404203902D20129007E075
:1017E0000A210398EEF776FC30317F1E03903970A2
:1017F0001199481E11900029F2DC03980028EFD1BE
:10180000791E129808703078202108404530BF1E9C
:10181000387006A8C01BC01D0390109800780028DF
:1018200000D00120019941180298C01709180398A7
:1018300009180498401A401E0490E00306D421467B
:101840001A9B199A049800F05FF8451910980078CF
:10185000002803D01A9A199990476D1CE00324D5EB
:1018600021461A9B199A049800F04EF845191CE07D
:101870000098002807DB00990598884203DD159839
:10188000405C199901E0199930201A9A9047009804
:101890006D1C401C00900298401E0290002804D14C
:1018A0001A9A2E20199990476D1C0199481E019093
:1018B0000029DDDC05E038781A9A7F1C19999047D9
:1018C0006D1C0399481E03900029F4DC21461A9BE5
:1018D000199A0498ACE600002D0000002B000000CF
:1018E0002000000000000000F8B5044600251E4658
:1018F0001746880404D405E039462020B0476D1C03
:10190000641EF9D52846F8BDFFB50446002581B010
:101910001E46C80301D5302700E02027880404D5DF
:1019200005E038460399B0476D1C641EF9D528467A
:1019300005B0F0BD4A68002A06D00A68531C0B6047
:1019400010704868401E486070470A68531C0B605E
:101950001070704700B50A4683B0002100910191D4
:10196000014601236846EFF7F3F80199009803B0A8
:1019700000BD004040404040404040404141414166
:101980004140404040404040404040404040404056
:10199000404040050202020202020202020202026A
:1019A00002020220202020202020202020020202EB
:1019B000020202029090909090901010101010105F
:1019C0001010101010101010101010101010020233
:1019D000020202028888888888880808080808089F
:1019E0000808080808080808080808080808020283
:1019F00002024000731901006A34010088130000DC
:101A0000010000005A3401008813000001000000AA
:101A1000503401008813000001000000643401000C
:101A20008813000001000000133401008813000037
:101A300001000000053401008813000001000000CF
:101A4000203401008813000001000000DB33010096
:101A500060EA0000030000007434010060EA000046
:101A6000030000007F340100E803000005000000CF
:101A7000F03301008813000005000000000084C15D
:101A8000000008C10000C03F000038410000AC4128
:101A90000000D441280004000000084008000008AD
:101AA00010080408102000000000000000000000E2
:101AB00001000000FFFFFFFF000000000000000029
:101AC00000000000B00400000100000060090000F8
:101AD00002000000C012000003000000802500008A
:101AE00004000000004B000005000000009600000C
:101AF0000600000000E100000700000000C2010035
:101B0000080000000084030009000000000807002E
:101B10000A00000000100E000B00000000201C0056
:101B20000C00000040420F000D00000080841E00E9
:101B30005906201403214501288200324100321940
:101B400000411300390300B506002D03002D0200EB
:101B50002201002201003E01002000008009EE4D1C
:101B60005048504F80096E4F58E5854F80096E4FA1
:101B7000B867C14F5048D04FB867C14FE828DF4F12
:101B80008009EE4F18EAFC4F8009EE4F58E50550EA
:101B9000A4550D50F0C51450A4550D50000021104F
:101BA000422063308440A550C660E77008812991C7
:101BB0004AA16BB18CC1ADD1CEE1EFF1311210026F
:101BC00073325222B5529442F772D6623993188317
:101BD0007BB35AA3BDD39CC3FFF3DEE3622443343B
:101BE00020040114E664C774A44485546AA54BB567
:101BF00028850995EEE5CFF5ACC58DD5533672260F
